 FileCase

 Timestamp is 61f9e9f9 (Wed Feb  2 02:18:33 2022)

 Preferred load address is 0000000180000000

 Start         Length     Name                   Class
 0001:00000000 00010510H .text$mn                CODE
 0001:00010510 00000040H .text$mn$00             CODE
 0001:00010550 00000490H .text$x                 CODE
 0002:00000000 00000250H .idata$5                DATA
 0002:00000250 00000028H .00cfg                  DATA
 0002:00000278 00000008H .CRT$XCA                DATA
 0002:00000280 00000008H .CRT$XCZ                DATA
 0002:00000288 00000008H .CRT$XIA                DATA
 0002:00000290 00000018H .CRT$XIC                DATA
 0002:000002a8 00000008H .CRT$XIZ                DATA
 0002:000002b0 00000008H .CRT$XPA                DATA
 0002:000002b8 00000010H .CRT$XPX                DATA
 0002:000002c8 00000008H .CRT$XPXA               DATA
 0002:000002d0 00000008H .CRT$XPZ                DATA
 0002:000002d8 00000008H .CRT$XTA                DATA
 0002:000002e0 00000010H .CRT$XTZ                DATA
 0002:000002e8 00000000H .gehcont$y              DATA
 0002:000002e8 00000000H .gfids$y                DATA
 0002:000002f0 00007890H .rdata                  DATA
 0002:00007b80 00000000H .rdata$CastGuardVftablesA DATA
 0002:00007b80 00000000H .rdata$CastGuardVftablesC DATA
 0002:00007b80 0000054cH .rdata$r                DATA
 0002:000080cc 00000028H .rdata$voltmd           DATA
 0002:000080f4 00000354H .rdata$zzzdbg           DATA
 0002:00008448 00000008H .rtc$IAA                DATA
 0002:00008450 00000008H .rtc$IZZ                DATA
 0002:00008458 00000008H .rtc$TAA                DATA
 0002:00008460 00000008H .rtc$TZZ                DATA
 0002:00008468 00000ff8H .xdata                  DATA
 0002:00009460 000001e0H .xdata$x                DATA
 0002:00009640 00000094H .edata                  DATA
 0002:000096d4 00000014H .idata$2                DATA
 0002:000096e8 00000018H .idata$3                DATA
 0002:00009700 00000250H .idata$4                DATA
 0002:00009950 00000542H .idata$6                DATA
 0003:00000000 000009e0H .data                   DATA
 0003:000009e0 000000f8H .data$r                 DATA
 0003:00000ad8 000000d8H .data$rs                DATA
 0003:00000bb0 000018d0H .bss                    DATA
 0004:00000000 000011b8H .pdata                  DATA
 0005:00000000 000000fcH _RDATA                  DATA
 0006:00000000 00000060H .rsrc$01                DATA
 0006:00000060 00000360H .rsrc$02                DATA

  Address         Publics by Value              Rva+Base               Lib:Object

 0000:00000000       __guard_longjmp_table      0000000000000000     <absolute>
 0000:00000000       ___safe_se_handler_table   0000000000000000     <absolute>
 0000:00000000       __x64_code_ranges_to_entry_points_count 0000000000000000     <absolute>
 0000:00000000       __guard_fids_count         0000000000000000     <absolute>
 0000:00000000       __arm64x_redirection_metadata 0000000000000000     <absolute>
 0000:00000000       __arm64x_extra_rfe_table   0000000000000000     <absolute>
 0000:00000000       __guard_iat_table          0000000000000000     <absolute>
 0000:00000000       __hybrid_code_map          0000000000000000     <absolute>
 0000:00000000       __guard_iat_count          0000000000000000     <absolute>
 0000:00000000       __arm64x_extra_rfe_table_size 0000000000000000     <absolute>
 0000:00000000       __guard_longjmp_count      0000000000000000     <absolute>
 0000:00000000       __x64_code_ranges_to_entry_points 0000000000000000     <absolute>
 0000:00000000       ___safe_se_handler_count   0000000000000000     <absolute>
 0000:00000000       __dynamic_value_reloc_table 0000000000000000     <absolute>
 0000:00000000       __hybrid_auxiliary_iat     0000000000000000     <absolute>
 0000:00000000       __hybrid_auxiliary_iat_copy 0000000000000000     <absolute>
 0000:00000000       __AbsoluteZero             0000000000000000     <absolute>
 0000:00000000       __guard_eh_cont_count      0000000000000000     <absolute>
 0000:00000000       __guard_check_icall_a64n_fptr 0000000000000000     <absolute>
 0000:00000000       __guard_fids_table         0000000000000000     <absolute>
 0000:00000000       __arm64x_redirection_metadata_count 0000000000000000     <absolute>
 0000:00000000       __enclave_config           0000000000000000     <absolute>
 0000:00000000       __guard_eh_cont_table      0000000000000000     <absolute>
 0000:00000000       __arm64x_native_entrypoint 0000000000000000     <absolute>
 0000:00000000       __hybrid_code_map_count    0000000000000000     <absolute>
 0000:00000100       __guard_flags              0000000000000100     <absolute>
 0000:00000000       __ImageBase                0000000180000000     <linker-defined>
 0001:00000000       ??1PluginSettings@@QEAA@XZ 0000000180001000 f i FileCase.obj
 0001:00000020       GetGlobalInfoW             0000000180001020 f   FileCase.obj
 0001:000000a0       SetStartupInfoW            00000001800010a0 f   FileCase.obj
 0001:000003f0       OpenW                      00000001800013f0 f   FileCase.obj
 0001:00000400       GetPluginInfoW             0000000180001400 f   FileCase.obj
 0001:00000450       ??0exception@std@@QEAA@AEBV01@@Z 0000000180001450 f i filecvt.obj
 0001:00000490       ?what@exception@std@@UEBAPEBDXZ 0000000180001490 f i filecvt.obj
 0001:000004b0       ??_Gbad_array_new_length@std@@UEAAPEAXI@Z 00000001800014b0 f i filecvt.obj
 0001:000004b0       ??_Gbad_alloc@std@@UEAAPEAXI@Z 00000001800014b0 f i filecvt.obj
 0001:000004b0       ??_Glength_error@std@@UEAAPEAXI@Z 00000001800014b0 f i libcpmt:xthrow.obj
 0001:000004b0       ??_Glogic_error@std@@UEAAPEAXI@Z 00000001800014b0 f i libcpmt:xthrow.obj
 0001:000004b0       ??_Ebad_exception@std@@UEAAPEAXI@Z 00000001800014b0 f i libvcruntime:frame.obj
 0001:000004b0       ??_Ebad_alloc@std@@UEAAPEAXI@Z 00000001800014b0 f i * CIL library *:* CIL module *
 0001:000004b0       ??_Elogic_error@std@@UEAAPEAXI@Z 00000001800014b0 f i libcpmt:xthrow.obj
 0001:000004b0       ??_Gexception@std@@UEAAPEAXI@Z 00000001800014b0 f i filecvt.obj
 0001:000004b0       ??_Gbad_exception@std@@UEAAPEAXI@Z 00000001800014b0 f i libvcruntime:frame.obj
 0001:000004b0       ??_Ebad_array_new_length@std@@UEAAPEAXI@Z 00000001800014b0 f i * CIL library *:* CIL module *
 0001:000004b0       ??_Elength_error@std@@UEAAPEAXI@Z 00000001800014b0 f i libcpmt:xthrow.obj
 0001:000004b0       ??_Eexception@std@@UEAAPEAXI@Z 00000001800014b0 f i * CIL library *:* CIL module *
 0001:00000500       ??1bad_exception@std@@UEAA@XZ 0000000180001500 f i libvcruntime:frame.obj
 0001:00000500       ??1bad_array_new_length@std@@UEAA@XZ 0000000180001500 f i filecvt.obj
 0001:00000500       ??1bad_alloc@std@@UEAA@XZ  0000000180001500 f i filecvt.obj
 0001:00000500       ??1length_error@std@@UEAA@XZ 0000000180001500 f i libcpmt:xthrow.obj
 0001:00000520       ??0bad_array_new_length@std@@QEAA@XZ 0000000180001520 f i filecvt.obj
 0001:00000550       ?_Throw_bad_array_new_length@std@@YAXXZ 0000000180001550 f i filecvt.obj
 0001:00000550       ?__scrt_throw_std_bad_array_new_length@@YAXXZ 0000000180001550 f i LIBCMT:throw_bad_alloc.obj
 0001:00000570       ??0bad_array_new_length@std@@QEAA@AEBV01@@Z 0000000180001570 f i filecvt.obj
 0001:000005b0       ??0bad_alloc@std@@QEAA@AEBV01@@Z 00000001800015b0 f i filecvt.obj
 0001:000005f0       ?_Xlen_string@std@@YAXXZ   00000001800015f0 f i filecvt.obj
 0001:00000610       ?SaveValue@PluginCheckBoxBinding@@UEAAXPEBUFarDialogItem@@H@Z 0000000180001610 f i filecvt.obj
 0001:00000680       ??_GPluginEditFieldBinding@@UEAAPEAXI@Z 0000000180001680 f i filecvt.obj
 0001:00000680       ??_EPluginCheckBoxBinding@@UEAAPEAXI@Z 0000000180001680 f i * CIL library *:* CIL module *
 0001:00000680       ??_EPluginEditFieldBinding@@UEAAPEAXI@Z 0000000180001680 f i * CIL library *:* CIL module *
 0001:00000680       ??_GPluginCheckBoxBinding@@UEAAPEAXI@Z 0000000180001680 f i filecvt.obj
 0001:000006b0       ?SaveValue@PluginRadioButtonBinding@@UEAAXPEBUFarDialogItem@@H@Z 00000001800016b0 f i filecvt.obj
 0001:00000700       ??_GPluginRadioButtonBinding@@UEAAPEAXI@Z 0000000180001700 f i filecvt.obj
 0001:00000700       ??_EPluginRadioButtonBinding@@UEAAPEAXI@Z 0000000180001700 f i * CIL library *:* CIL module *
 0001:00000730       ?SaveValue@PluginEditFieldBinding@@UEAAXPEBUFarDialogItem@@H@Z 0000000180001730 f i filecvt.obj
 0001:000007a0       ??0PluginDialogBuilder@@QEAA@AEBUPluginStartupInfo@@AEBU_GUID@@1HPEB_WP6A_JPEAX_J43@Z3_K@Z 00000001800017a0 f i filecvt.obj
 0001:000009e0       ??1PluginDialogBuilder@@QEAA@XZ 00000001800019e0 f i filecvt.obj
 0001:00000a60       ?AddRadioButtons@PluginDialogBuilder@@QEAAPEAUFarDialogItem@@PEAHHQEBH_N@Z 0000000180001a60 f i filecvt.obj
 0001:00000da0       ?AddButtons@PluginDialogBuilder@@QEAAXHPEBHHH@Z 0000000180001da0 f i filecvt.obj
 0001:000010a0       ?ShowDialogEx@PluginDialogBuilder@@QEAA_JXZ 00000001800020a0 f i filecvt.obj
 0001:000013f0       ?AddDialogItem@PluginDialogBuilder@@AEAAPEAUFarDialogItem@@W4FARDIALOGITEMTYPES@@PEB_W@Z 00000001800023f0 f i filecvt.obj
 0001:000015a0       ?ItemWidth@PluginDialogBuilder@@CA_JAEBUFarDialogItem@@@Z 00000001800025a0 f i filecvt.obj
 0001:00001680       ?CaseConvertion@@YAXXZ     0000000180002680 f   filecvt.obj
 0001:00002640       ?assign@?$basic_string@_WU?$char_traits@_W@std@@V?$allocator@_W@2@@std@@QEAAAEAV12@QEB_W_K@Z 0000000180003640 f i filecvt.obj
 0001:000027e0       ?IsCaseMixed@@YAHPEB_W@Z   00000001800037e0 f   FileMix.obj
 0001:00002880       ?CaseWord@@YAXPEA_WH@Z     0000000180003880 f   FileMix.obj
 0001:00002990       ?ProcessName@@YAXPEB_WK@Z  0000000180003990 f   ProcessName.obj
 0001:00002c70       __security_check_cookie    0000000180003c70 f   LIBCMT:amdsecgs.obj
 0001:00002c90       ??_V@YAXPEAX@Z             0000000180003c90 f   LIBCMT:delete_array.obj
 0001:00002c90       ??3@YAXPEAX_K@Z            0000000180003c90 f   LIBCMT:delete_scalar_size.obj
 0001:00002c98       ??2@YAPEAX_K@Z             0000000180003c98 f   LIBCMT:new_scalar.obj
 0001:00002cd4       ??3@YAXPEAX@Z              0000000180003cd4 f   LIBCMT:delete_scalar.obj
 0001:00002cdc       ??_U@YAPEAX_K@Z            0000000180003cdc f   LIBCMT:new_array.obj
 0001:00002ce4       ??_Etype_info@@UEAAPEAXI@Z 0000000180003ce4 f i LIBCMT:std_type_info_static.obj
 0001:00002ce4       ??_Gtype_info@@UEAAPEAXI@Z 0000000180003ce4 f i LIBCMT:std_type_info_static.obj
 0001:00003030       _DllMainCRTStartup         0000000180004030 f   LIBCMT:dll_dllmain.obj
 0001:00003070       __raise_securityfailure    0000000180004070 f   LIBCMT:gs_report.obj
 0001:000030a4       __report_gsfailure         00000001800040a4 f   LIBCMT:gs_report.obj
 0001:00003178       __report_rangecheckfailure 0000000180004178 f   LIBCMT:gs_report.obj
 0001:0000318c       __report_securityfailure   000000018000418c f   LIBCMT:gs_report.obj
 0001:0000330c       ??0bad_alloc@std@@QEAA@XZ  000000018000430c f i LIBCMT:throw_bad_alloc.obj
 0001:0000332c       ?__scrt_throw_std_bad_alloc@@YAXXZ 000000018000432c f   LIBCMT:throw_bad_alloc.obj
 0001:0000334c       __security_init_cookie     000000018000434c f   LIBCMT:gs_support.obj
 0001:000033f8       _get_startup_argv_mode     00000001800043f8 f   LIBCMT:argv_mode.obj
 0001:000033f8       DllMain                    00000001800043f8 f   LIBCMT:dll_dllmain_stub.obj
 0001:00003400       ?__scrt_initialize_type_info@@YAXXZ 0000000180004400 f   LIBCMT:tncleanup.obj
 0001:00003410       ?__scrt_uninitialize_type_info@@YAXXZ 0000000180004410 f   LIBCMT:tncleanup.obj
 0001:0000341c       __local_stdio_printf_options 000000018000441c f i LIBCMT:default_local_stdio_options.obj
 0001:00003424       __local_stdio_scanf_options 0000000180004424 f i LIBCMT:default_local_stdio_options.obj
 0001:0000342c       __scrt_initialize_default_local_stdio_options 000000018000442c f   LIBCMT:default_local_stdio_options.obj
 0001:00003448       __scrt_acquire_startup_lock 0000000180004448 f   LIBCMT:utility.obj
 0001:00003484       __scrt_dllmain_after_initialize_c 0000000180004484 f   LIBCMT:utility.obj
 0001:000034b8       __scrt_dllmain_before_initialize_c 00000001800044b8 f   LIBCMT:utility.obj
 0001:000034d0       __scrt_dllmain_crt_thread_attach 00000001800044d0 f   LIBCMT:utility.obj
 0001:000034f8       __scrt_dllmain_crt_thread_detach 00000001800044f8 f   LIBCMT:utility.obj
 0001:00003510       __scrt_dllmain_exception_filter 0000000180004510 f   LIBCMT:utility.obj
 0001:00003570       __scrt_dllmain_uninitialize_c 0000000180004570 f   LIBCMT:utility.obj
 0001:000035a0       __scrt_dllmain_uninitialize_critical 00000001800045a0 f   LIBCMT:utility.obj
 0001:000035b4       __scrt_initialize_crt      00000001800045b4 f   LIBCMT:utility.obj
 0001:00003600       __scrt_initialize_onexit_tables 0000000180004600 f   LIBCMT:utility.obj
 0001:0000368c       __scrt_is_nonwritable_in_current_image 000000018000468c f   LIBCMT:utility.obj
 0001:00003724       __scrt_release_startup_lock 0000000180004724 f   LIBCMT:utility.obj
 0001:00003748       __scrt_uninitialize_crt    0000000180004748 f   LIBCMT:utility.obj
 0001:00003774       __scrt_get_dyn_tls_init_callback 0000000180004774 f   LIBCMT:dyn_tls_init.obj
 0001:0000377c       __crt_debugger_hook        000000018000477c f   LIBCMT:utility_desktop.obj
 0001:00003784       __scrt_fastfail            0000000180004784 f   LIBCMT:utility_desktop.obj
 0001:000038d0       _RTC_Initialize            00000001800048d0 f   LIBCMT:initsect.obj
 0001:0000390c       _RTC_Terminate             000000018000490c f   LIBCMT:initsect.obj
 0001:00003948       _guard_check_icall_nop     0000000180004948 f i LIBCMT:guard_support.obj
 0001:0000394c       __isa_available_init       000000018000494c f   LIBCMT:cpu_disp.obj
 0001:00003af0       __scrt_is_ucrt_dll_in_use  0000000180004af0 f   LIBCMT:ucrt_detection.obj
 0001:00003b00       ??0length_error@std@@QEAA@AEBV01@@Z 0000000180004b00 f i libcpmt:xthrow.obj
 0001:00003b3c       ??0length_error@std@@QEAA@PEBD@Z 0000000180004b3c f i libcpmt:xthrow.obj
 0001:00003b84       ??0logic_error@std@@QEAA@AEBV01@@Z 0000000180004b84 f i libcpmt:xthrow.obj
 0001:00003bc0       ?_Xlength_error@std@@YAXPEBD@Z 0000000180004bc0 f   libcpmt:xthrow.obj
 0001:00003be4       ??$_CallSETranslator@V__FrameHandler4@@@@YAHPEAUEHExceptionRecord@@PEA_KPEAU_CONTEXT@@PEAU_xDISPATCHER_CONTEXT@@PEAUFuncInfo4@FH4@@K1H@Z 0000000180004be4 f i libvcruntime:risctrnsctrl.obj
 0001:00003c38       ?DecompFuncInfo@FH4@@YA_JPEAEAEAUFuncInfo4@1@_KH_N@Z 0000000180004c38 f i libvcruntime:risctrnsctrl.obj
 0001:00003d5c       ?ExecutionInCatch@__FrameHandler4@@SA_NPEAU_xDISPATCHER_CONTEXT@@PEAUFuncInfo4@FH4@@@Z 0000000180004d5c f   libvcruntime:risctrnsctrl.obj
 0001:00003d64       ?FrameUnwindToEmptyState@__FrameHandler4@@SAXPEA_KPEAU_xDISPATCHER_CONTEXT@@PEAUFuncInfo4@FH4@@@Z 0000000180004d64 f   libvcruntime:risctrnsctrl.obj
 0001:00003d98       ?GetEstablisherFrame@__FrameHandler4@@SAPEA_KPEA_KPEAU_xDISPATCHER_CONTEXT@@PEAUFuncInfo4@FH4@@0@Z 0000000180004d98 f   libvcruntime:risctrnsctrl.obj
 0001:00003dbc       ?GetRangeOfTrysToCheck@__FrameHandler4@@SA?AU?$pair@Viterator@TryBlockMap4@FH4@@V123@@std@@AEAVTryBlockMap4@FH4@@HPEAU_xDISPATCHER_CONTEXT@@PEAUFuncInfo4@5@H@Z 0000000180004dbc f   libvcruntime:risctrnsctrl.obj
 0001:00003f24       ?UnwindNestedFrames@__FrameHandler4@@SAXPEA_KPEAUEHExceptionRecord@@PEAU_CONTEXT@@0PEAXPEAUFuncInfo4@FH4@@HHPEAUHandlerType4@5@PEAU_xDISPATCHER_CONTEXT@@E@Z 0000000180004f24 f   libvcruntime:risctrnsctrl.obj
 0001:00004044       ?setBuffer@TryBlockMap4@FH4@@QEAAXViterator@12@@Z 0000000180005044 f i libvcruntime:risctrnsctrl.obj
 0001:00004204       _CreateFrameInfo           0000000180005204 f   libvcruntime:risctrnsctrl.obj
 0001:00004240       _FindAndUnlinkFrame        0000000180005240 f   libvcruntime:risctrnsctrl.obj
 0001:00004294       _GetImageBase              0000000180005294 f   libvcruntime:risctrnsctrl.obj
 0001:000042a8       _GetThrowImageBase         00000001800052a8 f   libvcruntime:risctrnsctrl.obj
 0001:000042bc       _SetImageBase              00000001800052bc f   libvcruntime:risctrnsctrl.obj
 0001:000042d4       _SetThrowImageBase         00000001800052d4 f   libvcruntime:risctrnsctrl.obj
 0001:000042ec       __CxxFrameHandler4         00000001800052ec f   libvcruntime:risctrnsctrl.obj
 0001:000043ac       __DestructExceptionObject  00000001800053ac f   libvcruntime:ehhelpers.obj
 0001:0000441c       ?_CallMemberFunction0@@YAXQEAX0@Z 000000018000541c f i libvcruntime:ehhelpers.obj
 0001:00004420       _IsExceptionObjectToBeDestroyed 0000000180005420 f   libvcruntime:ehhelpers.obj
 0001:00004450       __AdjustPointer            0000000180005450 f   libvcruntime:ehhelpers.obj
 0001:00004474       __FrameUnwindFilter        0000000180005474 f   libvcruntime:ehhelpers.obj
 0001:000044dc       __std_terminate            00000001800054dc f   libvcruntime:ehhelpers.obj
 0001:000044e8       __std_exception_copy       00000001800054e8 f   libvcruntime:std_exception.obj
 0001:00004578       __std_exception_destroy    0000000180005578 f   libvcruntime:std_exception.obj
 0001:000045a0       wcsrchr                    00000001800055a0 f   libvcruntime:wcsrchr.obj
 0001:00004650       __C_specific_handler       0000000180005650 f   libvcruntime:riscchandler.obj
 0001:0000485c       _CxxThrowException         000000018000585c f   libvcruntime:throw.obj
 0001:000048fc       __std_type_info_compare    00000001800058fc f   libvcruntime:std_type_info.obj
 0001:00004924       __std_type_info_destroy_list 0000000180005924 f   libvcruntime:std_type_info.obj
 0001:00004950       __vcrt_initialize          0000000180005950 f   libvcruntime:initialization.obj
 0001:00004978       __vcrt_thread_attach       0000000180005978 f   libvcruntime:initialization.obj
 0001:0000498c       __vcrt_thread_detach       000000018000598c f   libvcruntime:initialization.obj
 0001:000049a0       __vcrt_uninitialize        00000001800059a0 f   libvcruntime:initialization.obj
 0001:000049bc       __vcrt_uninitialize_critical 00000001800059bc f   libvcruntime:initialization.obj
 0001:000049e0       memset_repmovs             00000001800059e0 f   libvcruntime:memset.obj
 0001:00004a00       memset                     0000000180005a00 f   libvcruntime:memset.obj
 0001:00004b90       __vcrt_freefls             0000000180005b90 f   libvcruntime:per_thread_data.obj
 0001:00004bb0       __vcrt_freeptd             0000000180005bb0 f   libvcruntime:per_thread_data.obj
 0001:00004c00       __vcrt_getptd              0000000180005c00 f   libvcruntime:per_thread_data.obj
 0001:00004c1c       __vcrt_getptd_noexit       0000000180005c1c f   libvcruntime:per_thread_data.obj
 0001:00004cdc       __vcrt_initialize_ptd      0000000180005cdc f   libvcruntime:per_thread_data.obj
 0001:00004d24       __vcrt_uninitialize_ptd    0000000180005d24 f   libvcruntime:per_thread_data.obj
 0001:00004d48       ?StateFromControlPc@__FrameHandler4@@SAHPEAUFuncInfo4@FH4@@PEAU_xDISPATCHER_CONTEXT@@@Z 0000000180005d48 f   libvcruntime:ehstate.obj
 0001:00004d50       ?StateFromIp@__FrameHandler4@@SAHPEAUFuncInfo4@FH4@@PEAU_xDISPATCHER_CONTEXT@@_K@Z 0000000180005d50 f   libvcruntime:ehstate.obj
 0001:000059c0       ??$TypeMatchHelper@V__FrameHandler3@@@@YAHPEBU_s_HandlerType@@PEBU_s_CatchableType@@PEBU_s_ThrowInfo@@@Z 00000001800069c0 f i libvcruntime:frame.obj
 0001:00005b00       ??$TypeMatchHelper@V__FrameHandler4@@@@YAHPEAUHandlerType4@FH4@@PEBU_s_CatchableType@@PEBU_s_ThrowInfo@@@Z 0000000180006b00 f i libvcruntime:frame.obj
 0001:00005c44       ??$__InternalCxxFrameHandler@V__FrameHandler4@@@@YA?AW4_EXCEPTION_DISPOSITION@@PEAUEHExceptionRecord@@PEA_KPEAU_CONTEXT@@PEAU_xDISPATCHER_CONTEXT@@PEAUFuncInfo4@FH4@@H1E@Z 0000000180006c44 f i libvcruntime:frame.obj
 0001:00005ed8       ??0HandlerMap4@FH4@@QEAA@PEBUTryBlockMapEntry4@1@_KH@Z 0000000180006ed8 f i libvcruntime:frame.obj
 0001:00005f54       ??0TryBlockMap4@FH4@@QEAA@PEBUFuncInfo4@1@_K@Z 0000000180006f54 f i libvcruntime:frame.obj
 0001:0000602c       ??0bad_exception@std@@QEAA@AEBV01@@Z 000000018000702c f i libvcruntime:frame.obj
 0001:00006068       ??0bad_exception@std@@QEAA@XZ 0000000180007068 f i libvcruntime:frame.obj
 0001:00006088       ?CxxCallCatchBlock@__FrameHandler4@@SAPEAXPEAU_EXCEPTION_RECORD@@@Z 0000000180007088 f   libvcruntime:frame.obj
 0001:000062d8       ?DecompHandler@HandlerMap4@FH4@@AEAAXXZ 00000001800072d8 f i libvcruntime:frame.obj
 0001:00006518       ?FrameUnwindToState@__FrameHandler4@@SAXPEA_KPEAU_xDISPATCHER_CONTEXT@@PEAUFuncInfo4@FH4@@H@Z 0000000180007518 f   libvcruntime:frame.obj
 0001:00006978       ?ReadEntry@UWMap4@FH4@@AEAAXPEAPEAE@Z 0000000180007978 f i libvcruntime:frame.obj
 0001:00006a18       ?_CallMemberFunction1@@YAXQEAX00@Z 0000000180007a18 f i libvcruntime:frame.obj
 0001:00006a24       ?_CallMemberFunction2@@YAXQEAX00H@Z 0000000180007a24 f i libvcruntime:frame.obj
 0001:00006a34       ?getStartStop@UWMap4@FH4@@QEAAXHHAEAViterator@12@0@Z 0000000180007a34 f i libvcruntime:frame.obj
 0001:00006b04       ?getStateFromIterators@UWMap4@FH4@@SAHAEBViterator@12@H0H0@Z 0000000180007b04 f i libvcruntime:frame.obj
 0001:00006be0       _NLG_Notify                0000000180007be0 f   libvcruntime:notify.obj
 0001:00006c00       __NLG_Dispatch2            0000000180007c00 f   libvcruntime:notify.obj
 0001:00006c10       __NLG_Return2              0000000180007c10 f   libvcruntime:notify.obj
 0001:00006c14       __except_validate_context_record 0000000180007c14 f   libvcruntime:jbcxrval.obj
 0001:00006c4c       __vcrt_initialize_locks    0000000180007c4c f   libvcruntime:locks.obj
 0001:00006c80       __vcrt_uninitialize_locks  0000000180007c80 f   libvcruntime:locks.obj
 0001:00006e08       __vcrt_FlsAlloc            0000000180007e08 f   libvcruntime:winapi_downlevel.obj
 0001:00006e50       __vcrt_FlsFree             0000000180007e50 f   libvcruntime:winapi_downlevel.obj
 0001:00006e98       __vcrt_FlsGetValue         0000000180007e98 f   libvcruntime:winapi_downlevel.obj
 0001:00006ee0       __vcrt_FlsSetValue         0000000180007ee0 f   libvcruntime:winapi_downlevel.obj
 0001:00006f34       __vcrt_InitializeCriticalSectionEx 0000000180007f34 f   libvcruntime:winapi_downlevel.obj
 0001:00006fb0       _CallSettingFrame          0000000180007fb0 f   libvcruntime:handlers.obj
 0001:00007000       _CallSettingFrame_LookupContinuationIndex 0000000180008000 f   libvcruntime:handlers.obj
 0001:00007030       _CallSettingFrame_NotifyContinuationAddr 0000000180008030 f   libvcruntime:handlers.obj
 0001:00007060       _CallSettingFrameEncoded   0000000180008060 f   libvcruntime:handlers.obj
 0001:000070c0       memcpy_repmovs             00000001800080c0 f   libvcruntime:memcpy.obj
 0001:000070e0       memcpy                     00000001800080e0 f   libvcruntime:memcpy.obj
 0001:000070e0       memmove                    00000001800080e0 f   libvcruntime:memcpy.obj
 0001:00007758       free                       0000000180008758 f   libucrt:free.obj
 0001:0000776c       __acrt_call_reportfault    000000018000876c f   libucrt:invalid_parameter.obj
 0001:000078c8       __acrt_initialize_invalid_parameter_handler 00000001800088c8 f   libucrt:invalid_parameter.obj
 0001:000078d0       _invalid_parameter         00000001800088d0 f   libucrt:invalid_parameter.obj
 0001:00007980       _invalid_parameter_noinfo  0000000180008980 f   libucrt:invalid_parameter.obj
 0001:000079a0       _invalid_parameter_noinfo_noreturn 00000001800089a0 f   libucrt:invalid_parameter.obj
 0001:000079d0       _invoke_watson             00000001800089d0 f   libucrt:invalid_parameter.obj
 0001:00007a18       malloc                     0000000180008a18 f   libucrt:malloc.obj
 0001:00007a20       __acrt_initialize_new_handler 0000000180008a20 f   libucrt:new_handler.obj
 0001:00007a28       _callnewh                  0000000180008a28 f   libucrt:new_handler.obj
 0001:00007a58       _query_new_handler         0000000180008a58 f   libucrt:new_handler.obj
 0001:00007a8c       _initterm                  0000000180008a8c f   libucrt:initterm.obj
 0001:00007af0       _initterm_e                0000000180008af0 f   libucrt:initterm.obj
 0001:00007b30       _seh_filter_dll            0000000180008b30 f   libucrt:exception_filter.obj
 0001:00007b44       _seh_filter_exe            0000000180008b44 f   libucrt:exception_filter.obj
 0001:00007f34       __acrt_initialize_thread_local_exit_callback 0000000180008f34 f   libucrt:exit.obj
 0001:00007f3c       _cexit                     0000000180008f3c f   libucrt:exit.obj
 0001:00007f4c       _exit                      0000000180008f4c f   libucrt:exit.obj
 0001:00007f58       _is_c_termination_complete 0000000180008f58 f   libucrt:exit.obj
 0001:00008124       __acrt_allocate_buffer_for_argv 0000000180009124 f   libucrt:argv_parsing.obj
 0001:00008184       _configure_narrow_argv     0000000180009184 f   libucrt:argv_parsing.obj
 0001:000084fc       __dcrt_uninitialize_environments_nolock 00000001800094fc f   libucrt:environment_initialization.obj
 0001:00008534       _initialize_narrow_environment 0000000180009534 f   libucrt:environment_initialization.obj
 0001:00008690       _execute_onexit_table      0000000180009690 f   libucrt:onexit.obj
 0001:000086cc       _initialize_onexit_table   00000001800096cc f   libucrt:onexit.obj
 0001:0000872c       __acrt_uninitialize_command_line 000000018000972c f   libucrt:argv_data.obj
 0001:00008824       __acrt_initialize          0000000180009824 f   libucrt:initialization.obj
 0001:00008838       __acrt_thread_attach       0000000180009838 f   libucrt:initialization.obj
 0001:0000884c       __acrt_thread_detach       000000018000984c f   libucrt:initialization.obj
 0001:0000885c       __acrt_uninitialize        000000018000985c f   libucrt:initialization.obj
 0001:00008894       __acrt_uninitialize_critical 0000000180009894 f   libucrt:initialization.obj
 0001:000088a4       terminate                  00000001800098a4 f   libucrt:terminate.obj
 0001:000088c4       abort                      00000001800098c4 f   libucrt:abort.obj
 0001:0000891c       strcpy_s                   000000018000991c f   libucrt:strcpy_s.obj
 0001:0000897c       calloc                     000000018000997c f   libucrt:calloc.obj
 0001:00008984       ??0_LocaleUpdate@@QEAA@QEAU__crt_locale_pointers@@@Z 0000000180009984 f i libucrt:output.obj
 0001:00008a30       strncmp                    0000000180009a30 f   libucrt:strncmp.obj
 0001:00008ab0       wcsncmp                    0000000180009ab0 f   libucrt:wcsncmp.obj
 0001:00008adc       _free_base                 0000000180009adc f   libucrt:free_base.obj
 0001:00008e94       __acrt_freeptd             0000000180009e94 f   libucrt:per_thread_data.obj
 0001:00008ed8       __acrt_getptd              0000000180009ed8 f   libucrt:per_thread_data.obj
 0001:00008fac       __acrt_getptd_head         0000000180009fac f   libucrt:per_thread_data.obj
 0001:00009054       __acrt_getptd_noexit       000000018000a054 f   libucrt:per_thread_data.obj
 0001:00009120       __acrt_initialize_ptd      000000018000a120 f   libucrt:per_thread_data.obj
 0001:0000915c       __acrt_uninitialize_ptd    000000018000a15c f   libucrt:per_thread_data.obj
 0001:00009180       _malloc_base               000000018000a180 f   libucrt:malloc_base.obj
 0001:000091e0       __acrt_initialize_locks    000000018000a1e0 f   libucrt:locks.obj
 0001:00009228       __acrt_lock                000000018000a228 f   libucrt:locks.obj
 0001:00009244       __acrt_uninitialize_locks  000000018000a244 f   libucrt:locks.obj
 0001:0000927c       __acrt_unlock              000000018000a27c f   libucrt:locks.obj
 0001:00009298       __acrt_get_process_end_policy 000000018000a298 f   libucrt:win_policies.obj
 0001:000092d4       __acrt_errno_from_os_error 000000018000a2d4 f   libucrt:errno.obj
 0001:0000931c       __acrt_errno_map_os_error  000000018000a31c f   libucrt:errno.obj
 0001:0000936c       __doserrno                 000000018000a36c f   libucrt:errno.obj
 0001:0000938c       _errno                     000000018000a38c f   libucrt:errno.obj
 0001:000093ac       _calloc_base               000000018000a3ac f   libucrt:calloc_base.obj
 0001:00009438       ??$__acrt_mbs_to_wcs_cp@U__crt_win32_buffer_internal_dynamic_resizing@@@@YAHQEBDAEAV?$__crt_win32_buffer@_WU__crt_win32_buffer_internal_dynamic_resizing@@@@I@Z 000000018000a438 f i libucrt:argv_wildcards.obj
 0001:000095b0       ??$__acrt_wcs_to_mbs_cp@U__crt_win32_buffer_internal_dynamic_resizing@@@@YAHQEB_WAEAV?$__crt_win32_buffer@DU__crt_win32_buffer_internal_dynamic_resizing@@@@I@Z 000000018000a5b0 f i libucrt:argv_wildcards.obj
 0001:00009de0       __acrt_expand_narrow_argv_wildcards 000000018000ade0 f   libucrt:argv_wildcards.obj
 0001:00009de8       ??$__acrt_wcs_to_mbs_cp@U__crt_win32_buffer_no_resizing@@@@YAHQEB_WAEAV?$__crt_win32_buffer@DU__crt_win32_buffer_no_resizing@@@@I@Z 000000018000ade8 f i libucrt:getmodulefilenamea.obj
 0001:00009efc       __acrt_GetModuleFileNameA  000000018000aefc f   libucrt:getmodulefilenamea.obj
 0001:0000a748       __acrt_initialize_multibyte 000000018000b748 f   libucrt:mbctype.obj
 0001:0000a7a8       __acrt_update_thread_multibyte_data 000000018000b7a8 f   libucrt:mbctype.obj
 0001:0000a7c4       _setmbcp_nolock            000000018000b7c4 f   libucrt:mbctype.obj
 0001:0000aaf8       _ismbblead                 000000018000baf8 f   libucrt:ismbbyte.obj
 0001:0000ab0c       __acrt_initialize_command_line 000000018000bb0c f   libucrt:argv_data.obj
 0001:0000ab34       __acrt_MultiByteToWideChar 000000018000bb34 f   libucrt:multibytetowidechar.obj
 0001:0000ab90       __acrt_WideCharToMultiByte 000000018000bb90 f   libucrt:widechartomultibyte.obj
 0001:0000ac28       __dcrt_get_narrow_environment_from_os 000000018000bc28 f   libucrt:get_environment_from_os.obj
 0001:0000ad2c       _recalloc_base             000000018000bd2c f   libucrt:recalloc.obj
 0001:0000af9c       __acrt_AppPolicyGetProcessTerminationMethodInternal 000000018000bf9c f   libucrt:winapi_thunks.obj
 0001:0000afec       __acrt_AreFileApisANSI     000000018000bfec f   libucrt:winapi_thunks.obj
 0001:0000b028       __acrt_FlsAlloc            000000018000c028 f   libucrt:winapi_thunks.obj
 0001:0000b070       __acrt_FlsFree             000000018000c070 f   libucrt:winapi_thunks.obj
 0001:0000b0b8       __acrt_FlsGetValue         000000018000c0b8 f   libucrt:winapi_thunks.obj
 0001:0000b100       __acrt_FlsSetValue         000000018000c100 f   libucrt:winapi_thunks.obj
 0001:0000b154       __acrt_InitializeCriticalSectionEx 000000018000c154 f   libucrt:winapi_thunks.obj
 0001:0000b1b8       __acrt_LCMapStringEx       000000018000c1b8 f   libucrt:winapi_thunks.obj
 0001:0000b294       __acrt_LocaleNameToLCID    000000018000c294 f   libucrt:winapi_thunks.obj
 0001:0000b2e4       __acrt_initialize_winapi_thunks 000000018000c2e4 f   libucrt:winapi_thunks.obj
 0001:0000b318       __acrt_uninitialize_winapi_thunks 000000018000c318 f   libucrt:winapi_thunks.obj
 0001:0000b35c       __acrt_initialize_heap     000000018000c35c f   libucrt:heap_handle.obj
 0001:0000b378       __acrt_uninitialize_heap   000000018000c378 f   libucrt:heap_handle.obj
 0001:0000b580       __acrt_initialize_lowio    000000018000c580 f   libucrt:ioinit.obj
 0001:0000b5bc       __acrt_uninitialize_lowio  000000018000c5bc f   libucrt:ioinit.obj
 0001:0000b5fc       __acrt_execute_initializers 000000018000c5fc f   libucrt:shared_initialization.obj
 0001:0000b67c       __acrt_execute_uninitializers 000000018000c67c f   libucrt:shared_initialization.obj
 0001:0000b700       __acrt_get_sigabrt_handler 000000018000c700 f   libucrt:signal.obj
 0001:0000b730       __acrt_initialize_signal_handlers 000000018000c730 f   libucrt:signal.obj
 0001:0000b750       raise                      000000018000c750 f   libucrt:signal.obj
 0001:0000b9bc       __acrt_has_user_matherr    000000018000c9bc f   libucrt:matherr.obj
 0001:0000b9dc       __acrt_initialize_user_matherr 000000018000c9dc f   libucrt:matherr.obj
 0001:0000b9e4       __acrt_invoke_user_matherr 000000018000c9e4 f   libucrt:matherr.obj
 0001:0000bbf0       __acrt_stdio_flush_nolock  000000018000cbf0 f   libucrt:fflush.obj
 0001:0000bc6c       _fflush_nolock             000000018000cc6c f   libucrt:fflush.obj
 0001:0000bcb8       _flushall                  000000018000ccb8 f   libucrt:fflush.obj
 0001:0000bcc0       __acrt_initialize_stdio    000000018000ccc0 f   libucrt:_file.obj
 0001:0000bde0       __acrt_uninitialize_stdio  000000018000cde0 f   libucrt:_file.obj
 0001:0000be3c       _lock_file                 000000018000ce3c f   libucrt:_file.obj
 0001:0000be48       _unlock_file               000000018000ce48 f   libucrt:_file.obj
 0001:0000be54       _mbtowc_l                  000000018000ce54 f   libucrt:mbtowc.obj
 0001:0000bfd4       mbtowc                     000000018000cfd4 f   libucrt:mbtowc.obj
 0001:0000bfdc       __acrt_update_locale_info  000000018000cfdc f   libucrt:locale_update.obj
 0001:0000c010       __acrt_update_multibyte_info 000000018000d010 f   libucrt:locale_update.obj
 0001:0000c044       _fileno                    000000018000d044 f   libucrt:fileno.obj
 0001:0000c0dc       __acrt_set_locale_changed  000000018000d0dc f   libucrt:wsetlocale.obj
 0001:0000c0e8       __acrt_uninitialize_locale 000000018000d0e8 f   libucrt:wsetlocale.obj
 0001:0000c118       __pctype_func              000000018000d118 f   libucrt:ctype.obj
 0001:0000c148       __acrt_add_locale_ref      000000018000d148 f   libucrt:locale_refcounting.obj
 0001:0000c1d4       __acrt_free_locale         000000018000d1d4 f   libucrt:locale_refcounting.obj
 0001:0000c34c       __acrt_locale_add_lc_time_reference 000000018000d34c f   libucrt:locale_refcounting.obj
 0001:0000c374       __acrt_locale_free_lc_time_if_unreferenced 000000018000d374 f   libucrt:locale_refcounting.obj
 0001:0000c3ac       __acrt_locale_release_lc_time_reference 000000018000d3ac f   libucrt:locale_refcounting.obj
 0001:0000c3d4       __acrt_release_locale_ref  000000018000d3d4 f   libucrt:locale_refcounting.obj
 0001:0000c47c       __acrt_update_thread_locale_data 000000018000d47c f   libucrt:locale_refcounting.obj
 0001:0000c4e8       _updatetlocinfoEx_nolock   000000018000d4e8 f   libucrt:locale_refcounting.obj
 0001:0000c550       _query_new_mode            000000018000d550 f   libucrt:new_mode.obj
 0001:0000c560       qsort                      000000018000d560 f   libucrt:qsort.obj
 0001:0000c910       strncpy_s                  000000018000d910 f   libucrt:strncpy_s.obj
 0001:0000ca90       strpbrk                    000000018000da90 f   libucrt:strpbrk.obj
 0001:0000ce70       _mbsdec                    000000018000de70 f   libucrt:mbsdec.obj
 0001:0000ce78       _mbsdec_l                  000000018000de78 f   libucrt:mbsdec.obj
 0001:0000cf0c       __acrt_GetStringTypeA      000000018000df0c f   libucrt:getstringtypea.obj
 0001:0000d3b4       __acrt_LCMapStringA        000000018000e3b4 f   libucrt:lcmapstringa.obj
 0001:0000d464       _msize_base                000000018000e464 f   libucrt:msize.obj
 0001:0000d4a0       _realloc_base              000000018000e4a0 f   libucrt:realloc_base.obj
 0001:0000d51c       __acrt_DownlevelLocaleNameToLCID 000000018000e51c f   libucrt:lcidtoname_downlevel.obj
 0001:0000d5cc       __acrt_lowio_create_handle_array 000000018000e5cc f   libucrt:osfinfo.obj
 0001:0000d674       __acrt_lowio_destroy_handle_array 000000018000e674 f   libucrt:osfinfo.obj
 0001:0000d6c4       __acrt_lowio_ensure_fh_exists 000000018000e6c4 f   libucrt:osfinfo.obj
 0001:0000d76c       __acrt_lowio_lock_fh       000000018000e76c f   libucrt:osfinfo.obj
 0001:0000d794       __acrt_lowio_unlock_fh     000000018000e794 f   libucrt:osfinfo.obj
 0001:0000d7bc       _free_osfhnd               000000018000e7bc f   libucrt:osfinfo.obj
 0001:0000d878       _get_osfhandle             000000018000e878 f   libucrt:osfinfo.obj
 0001:0000d97c       _commit                    000000018000e97c f   libucrt:commit.obj
 0001:0000e270       _write                     000000018000f270 f   libucrt:write.obj
 0001:0000e35c       _write_nolock              000000018000f35c f   libucrt:write.obj
 0001:0000e638       _fcloseall                 000000018000f638 f   libucrt:closeall.obj
 0001:0000e6ec       __acrt_stdio_free_buffer_nolock 000000018000f6ec f   libucrt:_freebuf.obj
 0001:0000e72c       _isatty                    000000018000f72c f   libucrt:isatty.obj
 0001:0000e78c       _isleadbyte_l              000000018000f78c f i libucrt:_wctype.obj
 0001:0000e7d8       ?__mbrtowc_utf8@__crt_mbstring@@YA_KPEA_WPEBD_KPEAU_Mbstatet@@@Z 000000018000f7d8 f   libucrt:mbrtowc.obj
 0001:0000e814       ?__mbsrtowcs_utf8@__crt_mbstring@@YA_KPEA_WPEAPEBD_KPEAU_Mbstatet@@@Z 000000018000f814 f   libucrt:mbrtowc.obj
 0001:0000e98c       __acrt_locale_free_monetary 000000018000f98c f   libucrt:initmon.obj
 0001:0000ea98       __acrt_locale_free_numeric 000000018000fa98 f   libucrt:initnum.obj
 0001:0000eb5c       __acrt_locale_free_time    000000018000fb5c f   libucrt:inittime.obj
 0001:0000ec64       __strncnt                  000000018000fc64 f   libucrt:strncnt.obj
 0001:0000ec7c       __ascii_wcsnicmp           000000018000fc7c f   libucrt:wcsnicmp.obj
 0001:0000ecc8       _query_app_type            000000018000fcc8 f   libucrt:report_runtime_error.obj
 0001:0000ed6c       _lseeki64_nolock           000000018000fd6c f   libucrt:lseek.obj
 0001:0000ed74       _putwch_nolock             000000018000fd74 f   libucrt:putwch.obj
 0001:0000edb0       _fclose_nolock             000000018000fdb0 f   libucrt:fclose.obj
 0001:0000ee34       fclose                     000000018000fe34 f   libucrt:fclose.obj
 0001:0000ee98       ?__mbrtoc32_utf8@__crt_mbstring@@YA_KPEA_UPEBD_KPEAU_Mbstatet@@@Z 000000018000fe98 f   libucrt:mbrtoc32.obj
 0001:0000f080       log10                      0000000180010080 f   libucrt:log10.obj
 0001:0000f62c       __dcrt_lowio_ensure_console_output_initialized 000000018001062c f   libucrt:initcon.obj
 0001:0000f680       __dcrt_terminate_console_output 0000000180010680 f   libucrt:initcon.obj
 0001:0000f69c       __dcrt_write_console       000000018001069c f   libucrt:initcon.obj
 0001:0000f7d0       _close                     00000001800107d0 f   libucrt:close.obj
 0001:0000f874       _close_nolock              0000000180010874 f   libucrt:close.obj
 0001:0000f934       ?__acrt_stdio_free_stream@@YAXV__crt_stdio_stream@@@Z 0000000180010934 f   libucrt:stream.obj
 0001:0000fa74       _handle_error              0000000180010a74 f   libucrt:libm_error.obj
 0001:0000fba0       __acrt_initialize_fma3     0000000180010ba0 f   libucrt:fma3_available.obj
 0001:0000fc10       _log10_special             0000000180010c10 f   libucrt:log_special.obj
 0001:0000fce0       _get_fpsr                  0000000180010ce0 f   libucrt:fpsr.obj
 0001:0000fcf0       _set_fpsr                  0000000180010cf0 f   libucrt:fpsr.obj
 0001:0000fcfa       _fclrf                     0000000180010cfa f   libucrt:fpsr.obj
 0001:0000fd0e       _frnd                      0000000180010d0e f   libucrt:fpsr.obj
 0001:0000fd30       _raise_exc                 0000000180010d30 f   libucrt:fpexcept.obj
 0001:0000fd58       _raise_exc_ex              0000000180010d58 f   libucrt:fpexcept.obj
 0001:00010068       _set_errno_from_matherr    0000000180011068 f   libucrt:fpexcept.obj
 0001:00010098       _clrfp                     0000000180011098 f   libucrt:fpctrl.obj
 0001:000100b8       _ctrlfp                    00000001800110b8 f   libucrt:fpctrl.obj
 0001:00010134       _set_statfp                0000000180011134 f   libucrt:fpctrl.obj
 0001:00010154       _statfp                    0000000180011154 f   libucrt:fpctrl.obj
 0001:00010168       __GSHandlerCheck           0000000180011168 f   LIBCMT:gshandler.obj
 0001:00010188       __GSHandlerCheckCommon     0000000180011188 f   LIBCMT:gshandler.obj
 0001:000101f0       _FindPESection             00000001800111f0 f   LIBCMT:pesect.obj
 0001:00010240       _IsNonwritableInCurrentImage 0000000180011240 f   LIBCMT:pesect.obj
 0001:00010290       _ValidateImageBase         0000000180011290 f   LIBCMT:pesect.obj
 0001:000102c0       __GSHandlerCheck_SEH       00000001800112c0 f   LIBCMT:gshandlerseh.obj
 0001:00010360       __chkstk                   0000000180011360 f   LIBCMT:chkstk.obj
 0001:00010360       _alloca_probe              0000000180011360 f   LIBCMT:chkstk.obj
 0001:000103c0       memcmp                     00000001800113c0 f   libvcruntime:memcmp.obj
 0001:00010488       __GSHandlerCheck_EH4       0000000180011488 f   LIBCMT:gshandlereh4.obj
 0001:00010520       _guard_dispatch_icall_nop  0000000180011520 f   LIBCMT:guard_dispatch.obj
 0001:00010540       _guard_xfg_dispatch_icall_nop 0000000180011540 f   LIBCMT:guard_xfg_dispatch.obj
 0002:00000000       __imp_lstrlenW             0000000180012000     kernel32:KERNEL32.dll
 0002:00000008       __imp_lstrcpynW            0000000180012008     kernel32:KERNEL32.dll
 0002:00000010       __imp_lstrcatW             0000000180012010     kernel32:KERNEL32.dll
 0002:00000018       __imp_lstrcpyW             0000000180012018     kernel32:KERNEL32.dll
 0002:00000020       __imp_MoveFileW            0000000180012020     kernel32:KERNEL32.dll
 0002:00000028       __imp_WriteConsoleW        0000000180012028     kernel32:KERNEL32.dll
 0002:00000030       __imp_RtlCaptureContext    0000000180012030     kernel32:KERNEL32.dll
 0002:00000038       __imp_RtlLookupFunctionEntry 0000000180012038     kernel32:KERNEL32.dll
 0002:00000040       __imp_RtlVirtualUnwind     0000000180012040     kernel32:KERNEL32.dll
 0002:00000048       __imp_UnhandledExceptionFilter 0000000180012048     kernel32:KERNEL32.dll
 0002:00000050       __imp_SetUnhandledExceptionFilter 0000000180012050     kernel32:KERNEL32.dll
 0002:00000058       __imp_GetCurrentProcess    0000000180012058     kernel32:KERNEL32.dll
 0002:00000060       __imp_TerminateProcess     0000000180012060     kernel32:KERNEL32.dll
 0002:00000068       __imp_IsProcessorFeaturePresent 0000000180012068     kernel32:KERNEL32.dll
 0002:00000070       __imp_QueryPerformanceCounter 0000000180012070     kernel32:KERNEL32.dll
 0002:00000078       __imp_GetCurrentProcessId  0000000180012078     kernel32:KERNEL32.dll
 0002:00000080       __imp_GetCurrentThreadId   0000000180012080     kernel32:KERNEL32.dll
 0002:00000088       __imp_GetSystemTimeAsFileTime 0000000180012088     kernel32:KERNEL32.dll
 0002:00000090       __imp_InitializeSListHead  0000000180012090     kernel32:KERNEL32.dll
 0002:00000098       __imp_IsDebuggerPresent    0000000180012098     kernel32:KERNEL32.dll
 0002:000000a0       __imp_GetStartupInfoW      00000001800120a0     kernel32:KERNEL32.dll
 0002:000000a8       __imp_GetModuleHandleW     00000001800120a8     kernel32:KERNEL32.dll
 0002:000000b0       __imp_RtlUnwindEx          00000001800120b0     kernel32:KERNEL32.dll
 0002:000000b8       __imp_RtlPcToFileHeader    00000001800120b8     kernel32:KERNEL32.dll
 0002:000000c0       __imp_RaiseException       00000001800120c0     kernel32:KERNEL32.dll
 0002:000000c8       __imp_InterlockedFlushSList 00000001800120c8     kernel32:KERNEL32.dll
 0002:000000d0       __imp_GetLastError         00000001800120d0     kernel32:KERNEL32.dll
 0002:000000d8       __imp_SetLastError         00000001800120d8     kernel32:KERNEL32.dll
 0002:000000e0       __imp_EncodePointer        00000001800120e0     kernel32:KERNEL32.dll
 0002:000000e8       __imp_EnterCriticalSection 00000001800120e8     kernel32:KERNEL32.dll
 0002:000000f0       __imp_LeaveCriticalSection 00000001800120f0     kernel32:KERNEL32.dll
 0002:000000f8       __imp_DeleteCriticalSection 00000001800120f8     kernel32:KERNEL32.dll
 0002:00000100       __imp_InitializeCriticalSectionAndSpinCount 0000000180012100     kernel32:KERNEL32.dll
 0002:00000108       __imp_TlsAlloc             0000000180012108     kernel32:KERNEL32.dll
 0002:00000110       __imp_TlsGetValue          0000000180012110     kernel32:KERNEL32.dll
 0002:00000118       __imp_TlsSetValue          0000000180012118     kernel32:KERNEL32.dll
 0002:00000120       __imp_TlsFree              0000000180012120     kernel32:KERNEL32.dll
 0002:00000128       __imp_FreeLibrary          0000000180012128     kernel32:KERNEL32.dll
 0002:00000130       __imp_GetProcAddress       0000000180012130     kernel32:KERNEL32.dll
 0002:00000138       __imp_LoadLibraryExW       0000000180012138     kernel32:KERNEL32.dll
 0002:00000140       __imp_ExitProcess          0000000180012140     kernel32:KERNEL32.dll
 0002:00000148       __imp_GetModuleHandleExW   0000000180012148     kernel32:KERNEL32.dll
 0002:00000150       __imp_GetModuleFileNameW   0000000180012150     kernel32:KERNEL32.dll
 0002:00000158       __imp_HeapFree             0000000180012158     kernel32:KERNEL32.dll
 0002:00000160       __imp_HeapAlloc            0000000180012160     kernel32:KERNEL32.dll
 0002:00000168       __imp_FindClose            0000000180012168     kernel32:KERNEL32.dll
 0002:00000170       __imp_FindFirstFileExW     0000000180012170     kernel32:KERNEL32.dll
 0002:00000178       __imp_FindNextFileW        0000000180012178     kernel32:KERNEL32.dll
 0002:00000180       __imp_IsValidCodePage      0000000180012180     kernel32:KERNEL32.dll
 0002:00000188       __imp_GetACP               0000000180012188     kernel32:KERNEL32.dll
 0002:00000190       __imp_GetOEMCP             0000000180012190     kernel32:KERNEL32.dll
 0002:00000198       __imp_GetCPInfo            0000000180012198     kernel32:KERNEL32.dll
 0002:000001a0       __imp_GetCommandLineA      00000001800121a0     kernel32:KERNEL32.dll
 0002:000001a8       __imp_GetCommandLineW      00000001800121a8     kernel32:KERNEL32.dll
 0002:000001b0       __imp_MultiByteToWideChar  00000001800121b0     kernel32:KERNEL32.dll
 0002:000001b8       __imp_WideCharToMultiByte  00000001800121b8     kernel32:KERNEL32.dll
 0002:000001c0       __imp_GetEnvironmentStringsW 00000001800121c0     kernel32:KERNEL32.dll
 0002:000001c8       __imp_FreeEnvironmentStringsW 00000001800121c8     kernel32:KERNEL32.dll
 0002:000001d0       __imp_LCMapStringW         00000001800121d0     kernel32:KERNEL32.dll
 0002:000001d8       __imp_GetProcessHeap       00000001800121d8     kernel32:KERNEL32.dll
 0002:000001e0       __imp_GetStdHandle         00000001800121e0     kernel32:KERNEL32.dll
 0002:000001e8       __imp_GetFileType          00000001800121e8     kernel32:KERNEL32.dll
 0002:000001f0       __imp_GetStringTypeW       00000001800121f0     kernel32:KERNEL32.dll
 0002:000001f8       __imp_HeapSize             00000001800121f8     kernel32:KERNEL32.dll
 0002:00000200       __imp_HeapReAlloc          0000000180012200     kernel32:KERNEL32.dll
 0002:00000208       __imp_SetStdHandle         0000000180012208     kernel32:KERNEL32.dll
 0002:00000210       __imp_FlushFileBuffers     0000000180012210     kernel32:KERNEL32.dll
 0002:00000218       __imp_WriteFile            0000000180012218     kernel32:KERNEL32.dll
 0002:00000220       __imp_GetConsoleCP         0000000180012220     kernel32:KERNEL32.dll
 0002:00000228       __imp_GetConsoleMode       0000000180012228     kernel32:KERNEL32.dll
 0002:00000230       __imp_SetFilePointerEx     0000000180012230     kernel32:KERNEL32.dll
 0002:00000238       __imp_CreateFileW          0000000180012238     kernel32:KERNEL32.dll
 0002:00000240       __imp_CloseHandle          0000000180012240     kernel32:KERNEL32.dll
 0002:00000248       \177KERNEL32_NULL_THUNK_DATA 0000000180012248     kernel32:KERNEL32.dll
 0002:00000250       __guard_check_icall_fptr   0000000180012250     LIBCMT:guard_support.obj
 0002:00000258       __guard_xfg_check_icall_fptr 0000000180012258     LIBCMT:guard_support.obj
 0002:00000260       __guard_dispatch_icall_fptr 0000000180012260     LIBCMT:guard_support.obj
 0002:00000268       __guard_xfg_dispatch_icall_fptr 0000000180012268     LIBCMT:guard_support.obj
 0002:00000270       __guard_xfg_table_dispatch_icall_fptr 0000000180012270     LIBCMT:guard_support.obj
 0002:00000278       __xc_a                     0000000180012278     LIBCMT:initializers.obj
 0002:00000280       __xc_z                     0000000180012280     LIBCMT:initializers.obj
 0002:00000288       __xi_a                     0000000180012288     LIBCMT:initializers.obj
 0002:00000290       __acrt_multibyte_initializer 0000000180012290     libucrt:multibyte_initializer.obj
 0002:00000298       __acrt_stdio_initializer   0000000180012298     libucrt:stdio_initializer.obj
 0002:000002a0       __acrt_tran_fma3_initializer 00000001800122a0     libucrt:fma3_initializer.obj
 0002:000002a8       __xi_z                     00000001800122a8     LIBCMT:initializers.obj
 0002:000002b0       __xp_a                     00000001800122b0     LIBCMT:initializers.obj
 0002:000002b8       __acrt_locale_terminator   00000001800122b8     libucrt:locale_initializer.obj
 0002:000002c0       __dcrt_console_output_terminator 00000001800122c0     libucrt:console_output_initializer.obj
 0002:000002c8       __acrt_stdio_terminator    00000001800122c8     libucrt:stdio_initializer.obj
 0002:000002d0       __xp_z                     00000001800122d0     LIBCMT:initializers.obj
 0002:000002d8       __xt_a                     00000001800122d8     LIBCMT:initializers.obj
 0002:000002e0       __xt_z                     00000001800122e0     LIBCMT:initializers.obj
 0002:000002f8       ??_7type_info@@6B@         00000001800122f8     LIBCMT:std_type_info_static.obj
 0002:00000300       _pRawDllMain               0000000180012300     LIBCMT:dll_dllmain.obj
 0002:00000300       _pDefaultRawDllMain        0000000180012300     LIBCMT:dll_dllmain.obj
 0002:00000320       ??_7exception@std@@6B@     0000000180012320     LIBCMT:throw_bad_alloc.obj
 0002:00000338       ??_7bad_alloc@std@@6B@     0000000180012338     LIBCMT:throw_bad_alloc.obj
 0002:00000348       ??_C@_0P@GHFPNOJB@bad?5allocation@ 0000000180012348     LIBCMT:throw_bad_alloc.obj
 0002:00000360       ??_7bad_array_new_length@std@@6B@ 0000000180012360     LIBCMT:throw_bad_alloc.obj
 0002:00000370       __xmm@ffffffffffffffffffffffffffffffff 0000000180012370     LIBCMT:utility.obj
 0002:00000388       ??_7logic_error@std@@6B@   0000000180012388     libcpmt:xthrow.obj
 0002:000003a0       ??_7length_error@std@@6B@  00000001800123a0     libcpmt:xthrow.obj
 0002:000003b0       ?s_negLengthTab@FH4@@3QBCB 00000001800123b0     libvcruntime:risctrnsctrl.obj
 0002:000003c0       ?s_shiftTab@FH4@@3QBEB     00000001800123c0     libvcruntime:risctrnsctrl.obj
 0002:00000468       _pDestructExceptionObject  0000000180012468     libvcruntime:ehhelpers.obj
 0002:00000478       ??_7bad_exception@std@@6B@ 0000000180012478     libvcruntime:frame.obj
 0002:00000488       ??_C@_0O@DPKOEFFH@bad?5exception@ 0000000180012488     libvcruntime:frame.obj
 0002:00000ba0       ??_C@_08EHJDFFNH@__based?$CI@ 0000000180012ba0     libvcruntime:undname.obj
 0002:00000bb0       ??_C@_07KOLFKCDI@__cdecl@  0000000180012bb0     libvcruntime:undname.obj
 0002:00000bb8       ??_C@_08GHMPAG@__pascal@   0000000180012bb8     libvcruntime:undname.obj
 0002:00000bc8       ??_C@_09IFJBGAPI@__stdcall@ 0000000180012bc8     libvcruntime:undname.obj
 0002:00000bd8       ??_C@_0L@NPHFGOKO@__thiscall@ 0000000180012bd8     libvcruntime:undname.obj
 0002:00000be8       ??_C@_0L@JMKHOMEK@__fastcall@ 0000000180012be8     libvcruntime:undname.obj
 0002:00000bf8       ??_C@_0N@BCKKPABJ@__vectorcall@ 0000000180012bf8     libvcruntime:undname.obj
 0002:00000c08       ??_C@_09HIJEGCPM@__clrcall@ 0000000180012c08     libvcruntime:undname.obj
 0002:00000c14       ??_C@_06GHPCKEAG@__eabi@   0000000180012c14     libvcruntime:undname.obj
 0002:00000c20       ??_C@_09IOPIDJLG@__swift_1@ 0000000180012c20     libvcruntime:undname.obj
 0002:00000c30       ??_C@_09KFNFGKHF@__swift_2@ 0000000180012c30     libvcruntime:undname.obj
 0002:00000c40       ??_C@_07JOMMBBKO@__ptr64@  0000000180012c40     libvcruntime:undname.obj
 0002:00000c48       ??_C@_0L@PILCLIHE@__restrict@ 0000000180012c48     libvcruntime:undname.obj
 0002:00000c58       ??_C@_0M@GFIIJFMG@__unaligned@ 0000000180012c58     libvcruntime:undname.obj
 0002:00000c68       ??_C@_09DHDLOLLB@restrict?$CI@ 0000000180012c68     libvcruntime:undname.obj
 0002:00000c72       ??_C@_00CNPNBAHC@@         0000000180012c72     libvcruntime:undname.obj
 0002:00000c74       ??_C@_04NIHEBCM@?5new@     0000000180012c74     libvcruntime:undname.obj
 0002:00000c80       ??_C@_07FPCDHGMM@?5delete@ 0000000180012c80     libvcruntime:undname.obj
 0002:00000c88       ??_C@_01NEMOKFLO@?$DN@     0000000180012c88     libvcruntime:undname.obj
 0002:00000c8c       ??_C@_02GPIOPFAK@?$DO?$DO@ 0000000180012c8c     libvcruntime:undname.obj
 0002:00000c90       ??_C@_02FODMEDOG@?$DM?$DM@ 0000000180012c90     libvcruntime:undname.obj
 0002:00000c94       ??_C@_01DCLJPIOD@?$CB@     0000000180012c94     libvcruntime:undname.obj
 0002:00000c98       ??_C@_02EGOFBIJA@?$DN?$DN@ 0000000180012c98     libvcruntime:undname.obj
 0002:00000c9c       ??_C@_02FDNJECIE@?$CB?$DN@ 0000000180012c9c     libvcruntime:undname.obj
 0002:00000ca0       ??_C@_02GPECMEKF@?$FL?$FN@ 0000000180012ca0     libvcruntime:undname.obj
 0002:00000ca8       ??_C@_08LHJFAFGD@operator@ 0000000180012ca8     libvcruntime:undname.obj
 0002:00000cb4       ??_C@_02HBOOOICD@?9?$DO@   0000000180012cb4     libvcruntime:undname.obj
 0002:00000cb8       ??_C@_01NBENCBCI@?$CK@     0000000180012cb8     libvcruntime:undname.obj
 0002:00000cbc       ??_C@_02ECNGHCIF@?$CL?$CL@ 0000000180012cbc     libvcruntime:undname.obj
 0002:00000cc0       ??_C@_02BAABKJLB@?9?9@     0000000180012cc0     libvcruntime:undname.obj
 0002:00000cc4       ??_C@_01JOAMLHOP@?9@       0000000180012cc4     libvcruntime:undname.obj
 0002:00000cc8       ??_C@_01MIFGBAGJ@?$CL@     0000000180012cc8     libvcruntime:undname.obj
 0002:00000ccc       ??_C@_01HNPIGOCE@?$CG@     0000000180012ccc     libvcruntime:undname.obj
 0002:00000cd0       ??_C@_03MNHNFDLC@?9?$DO?$CK@ 0000000180012cd0     libvcruntime:undname.obj
 0002:00000cd4       ??_C@_01KMDKNFGN@?1@       0000000180012cd4     libvcruntime:undname.obj
 0002:00000cd8       ??_C@_01FGNFDNOH@?$CF@     0000000180012cd8     libvcruntime:undname.obj
 0002:00000cdc       ??_C@_01MNNFJEPP@?$DM@     0000000180012cdc     libvcruntime:undname.obj
 0002:00000ce0       ??_C@_02EHCHHCKH@?$DM?$DN@ 0000000180012ce0     libvcruntime:undname.obj
 0002:00000ce4       ??_C@_01PPODPGHN@?$DO@     0000000180012ce4     libvcruntime:undname.obj
 0002:00000ce8       ??_C@_02EEKDKGMJ@?$DO?$DN@ 0000000180012ce8     libvcruntime:undname.obj
 0002:00000cec       ??_C@_01IHBHIGKO@?0@       0000000180012cec     libvcruntime:undname.obj
 0002:00000cf0       ??_C@_02HCKGKOFO@?$CI?$CJ@ 0000000180012cf0     libvcruntime:undname.obj
 0002:00000cf4       ??_C@_01PJKLJHI@?$HO@      0000000180012cf4     libvcruntime:undname.obj
 0002:00000cf8       ??_C@_01JKBOJNNK@?$FO@     0000000180012cf8     libvcruntime:undname.obj
 0002:00000cfc       ??_C@_01DNKMNLPK@?$HM@     0000000180012cfc     libvcruntime:undname.obj
 0002:00000d00       ??_C@_02PPKAJPJL@?$CG?$CG@ 0000000180012d00     libvcruntime:undname.obj
 0002:00000d04       ??_C@_02NONPIBCD@?$HM?$HM@ 0000000180012d04     libvcruntime:undname.obj
 0002:00000d08       ??_C@_02FPIMKNGF@?$CK?$DN@ 0000000180012d08     libvcruntime:undname.obj
 0002:00000d0c       ??_C@_02FOEOMHFC@?$CL?$DN@ 0000000180012d0c     libvcruntime:undname.obj
 0002:00000d10       ??_C@_02FKMDLLOA@?9?$DN@   0000000180012d10     libvcruntime:undname.obj
 0002:00000d14       ??_C@_02FJEHGPIO@?1?$DN@   0000000180012d14     libvcruntime:undname.obj
 0002:00000d18       ??_C@_02FENAOKFI@?$CF?$DN@ 0000000180012d18     libvcruntime:undname.obj
 0002:00000d1c       ??_C@_03IKFCCPFF@?$DO?$DO?$DN@ 0000000180012d1c     libvcruntime:undname.obj
 0002:00000d20       ??_C@_03CDNPDDLA@?$DM?$DM?$DN@ 0000000180012d20     libvcruntime:undname.obj
 0002:00000d24       ??_C@_02FGJGFEAB@?$CG?$DN@ 0000000180012d24     libvcruntime:undname.obj
 0002:00000d28       ??_C@_02DHLNPPGH@?$HM?$DN@ 0000000180012d28     libvcruntime:undname.obj
 0002:00000d2c       ??_C@_02MHEGNOJ@?$FO?$DN@  0000000180012d2c     libvcruntime:undname.obj
 0002:00000d30       ??_C@_09IFPLHPGF@?$GAvftable?8@ 0000000180012d30     libvcruntime:undname.obj
 0002:00000d40       ??_C@_09BLBHBJP@?$GAvbtable?8@ 0000000180012d40     libvcruntime:undname.obj
 0002:00000d50       ??_C@_07FEEIOKP@?$GAvcall?8@ 0000000180012d50     libvcruntime:undname.obj
 0002:00000d58       ??_C@_08LLFFHHDJ@?$GAtypeof?8@ 0000000180012d58     libvcruntime:undname.obj
 0002:00000d68       ??_C@_0BF@KDPPACIK@?$GAlocal?5static?5guard?8@ 0000000180012d68     libvcruntime:undname.obj
 0002:00000d80       ??_C@_08OBABFOLI@?$GAstring?8@ 0000000180012d80     libvcruntime:undname.obj
 0002:00000d90       ??_C@_0BD@JDLKDPAB@?$GAvbase?5destructor?8@ 0000000180012d90     libvcruntime:undname.obj
 0002:00000da8       ??_C@_0BN@DEGPLNFK@?$GAvector?5deleting?5destructor?8@ 0000000180012da8     libvcruntime:undname.obj
 0002:00000dc8       ??_C@_0BO@OBMKPJIG@?$GAdefault?5constructor?5closure?8@ 0000000180012dc8     libvcruntime:undname.obj
 0002:00000de8       ??_C@_0BN@IMDCHIKM@?$GAscalar?5deleting?5destructor?8@ 0000000180012de8     libvcruntime:undname.obj
 0002:00000e08       ??_C@_0BO@PFGOCPJJ@?$GAvector?5constructor?5iterator?8@ 0000000180012e08     libvcruntime:undname.obj
 0002:00000e28       ??_C@_0BN@LFPFMEDL@?$GAvector?5destructor?5iterator?8@ 0000000180012e28     libvcruntime:undname.obj
 0002:00000e48       ??_C@_0CE@IKBNEHA@?$GAvector?5vbase?5constructor?5itera@ 0000000180012e48     libvcruntime:undname.obj
 0002:00000e70       ??_C@_0BL@NILFHHPC@?$GAvirtual?5displacement?5map?8@ 0000000180012e70     libvcruntime:undname.obj
 0002:00000e90       ??_C@_0CB@JONCMFFK@?$GAeh?5vector?5constructor?5iterator@ 0000000180012e90     libvcruntime:undname.obj
 0002:00000eb8       ??_C@_0CA@GCEOPDGL@?$GAeh?5vector?5destructor?5iterator?8@ 0000000180012eb8     libvcruntime:undname.obj
 0002:00000ed8       ??_C@_0CH@OOJPLCPH@?$GAeh?5vector?5vbase?5constructor?5it@ 0000000180012ed8     libvcruntime:undname.obj
 0002:00000f00       ??_C@_0BL@LLKPOHJI@?$GAcopy?5constructor?5closure?8@ 0000000180012f00     libvcruntime:undname.obj
 0002:00000f20       ??_C@_0BA@KBCDOMBN@?$GAudt?5returning?8@ 0000000180012f20     libvcruntime:undname.obj
 0002:00000f30       ??_C@_03KLGMFNMG@?$GAEH@   0000000180012f30     libvcruntime:undname.obj
 0002:00000f34       ??_C@_05KHLCHHI@?$GARTTI@  0000000180012f34     libvcruntime:undname.obj
 0002:00000f40       ??_C@_0BA@KKLDJDLB@?$GAlocal?5vftable?8@ 0000000180012f40     libvcruntime:undname.obj
 0002:00000f50       ??_C@_0CE@IIHCMGGL@?$GAlocal?5vftable?5constructor?5clos@ 0000000180012f50     libvcruntime:undname.obj
 0002:00000f74       ??_C@_06FHBGPFGH@?5new?$FL?$FN@ 0000000180012f74     libvcruntime:undname.obj
 0002:00000f80       ??_C@_09LBNFPBCA@?5delete?$FL?$FN@ 0000000180012f80     libvcruntime:undname.obj
 0002:00000f90       ??_C@_0P@HJKNJFNN@?$GAomni?5callsig?8@ 0000000180012f90     libvcruntime:undname.obj
 0002:00000fa0       ??_C@_0BL@CNOONJFP@?$GAplacement?5delete?5closure?8@ 0000000180012fa0     libvcruntime:undname.obj
 0002:00000fc0       ??_C@_0BN@CKNJLHMB@?$GAplacement?5delete?$FL?$FN?5closure?8@ 0000000180012fc0     libvcruntime:undname.obj
 0002:00000fe0       ??_C@_0CG@CFDHKGGD@?$GAmanaged?5vector?5constructor?5ite@ 0000000180012fe0     libvcruntime:undname.obj
 0002:00001008       ??_C@_0CF@IMGKMJNO@?$GAmanaged?5vector?5destructor?5iter@ 0000000180013008     libvcruntime:undname.obj
 0002:00001030       ??_C@_0CG@HLDDJMAG@?$GAeh?5vector?5copy?5constructor?5ite@ 0000000180013030     libvcruntime:undname.obj
 0002:00001058       ??_C@_0CM@FCBBDIGB@?$GAeh?5vector?5vbase?5copy?5construct@ 0000000180013058     libvcruntime:undname.obj
 0002:00001088       ??_C@_0BL@CLIPGLGB@?$GAdynamic?5initializer?5for?5?8@ 0000000180013088     libvcruntime:undname.obj
 0002:000010a8       ??_C@_0CB@PDBIFEP@?$GAdynamic?5atexit?5destructor?5for?5@ 00000001800130a8     libvcruntime:undname.obj
 0002:000010d0       ??_C@_0CD@CGAJBKEJ@?$GAvector?5copy?5constructor?5iterat@ 00000001800130d0     libvcruntime:undname.obj
 0002:000010f8       ??_C@_0CJ@GJELGAMM@?$GAvector?5vbase?5copy?5constructor?5@ 00000001800130f8     libvcruntime:undname.obj
 0002:00001128       ??_C@_0CL@FGIJHLCE@?$GAmanaged?5vector?5copy?5constructo@ 0000000180013128     libvcruntime:undname.obj
 0002:00001158       ??_C@_0BM@PMGGMLDN@?$GAlocal?5static?5thread?5guard?8@ 0000000180013158     libvcruntime:undname.obj
 0002:00001178       ??_C@_0N@BDNMDMOL@operator?5?$CC?$CC?5@ 0000000180013178     libvcruntime:undname.obj
 0002:00001188       ??_C@_0BC@GGEBGALA@operator?5co_await@ 0000000180013188     libvcruntime:undname.obj
 0002:000011a0       ??_C@_0M@GAAIMMOH@operator?$DM?$DN?$DO@ 00000001800131a0     libvcruntime:undname.obj
 0002:000011b0       ??_C@_0BC@DAFEJGAK@?5Type?5Descriptor?8@ 00000001800131b0     libvcruntime:undname.obj
 0002:000011c8       ??_C@_0BM@LDKODKLH@?5Base?5Class?5Descriptor?5at?5?$CI@ 00000001800131c8     libvcruntime:undname.obj
 0002:000011e8       ??_C@_0BD@LGICGFMM@?5Base?5Class?5Array?8@ 00000001800131e8     libvcruntime:undname.obj
 0002:00001200       ??_C@_0BN@MECKDCOJ@?5Class?5Hierarchy?5Descriptor?8@ 0000000180013200     libvcruntime:undname.obj
 0002:00001220       ??_C@_0BK@CFCOFLF@?5Complete?5Object?5Locator?8@ 0000000180013220     libvcruntime:undname.obj
 0002:00001240       ??_C@_0BG@JNJLAMPM@?$GAanonymous?5namespace?8@ 0000000180013240     libvcruntime:undname.obj
 0002:00001270       ??_C@_1DM@KHCHBNEB@?$AAa?$AAp?$AAi?$AA?9?$AAm?$AAs?$AA?9?$AAw?$AAi?$AAn?$AA?9?$AAc?$AAo?$AAr?$AAe@ 0000000180013270     libvcruntime:winapi_downlevel.obj
 0002:000012b0       ??_C@_1DK@LPPGFMPP@?$AAa?$AAp?$AAi?$AA?9?$AAm?$AAs?$AA?9?$AAw?$AAi?$AAn?$AA?9?$AAc?$AAo?$AAr?$AAe@ 00000001800132b0     libvcruntime:winapi_downlevel.obj
 0002:000012f0       ??_C@_1BC@GDMECMAK@?$AAk?$AAe?$AAr?$AAn?$AAe?$AAl?$AA3?$AA2@ 00000001800132f0     libvcruntime:winapi_downlevel.obj
 0002:00001308       ??_C@_1BA@PFFKHIOG@?$AAa?$AAp?$AAi?$AA?9?$AAm?$AAs?$AA?9@ 0000000180013308     libvcruntime:winapi_downlevel.obj
 0002:00001320       ??_C@_08KNHFBNJ@FlsAlloc@  0000000180013320     libvcruntime:winapi_downlevel.obj
 0002:00001338       ??_C@_07PEJMOBNF@FlsFree@  0000000180013338     libvcruntime:winapi_downlevel.obj
 0002:00001348       ??_C@_0M@GDNOONDI@FlsGetValue@ 0000000180013348     libvcruntime:winapi_downlevel.obj
 0002:00001360       ??_C@_0M@JCPCPOEF@FlsSetValue@ 0000000180013360     libvcruntime:winapi_downlevel.obj
 0002:00001378       ??_C@_0BM@HCFOFFN@InitializeCriticalSectionEx@ 0000000180013378     libvcruntime:winapi_downlevel.obj
 0002:000013a0       __acrt_exception_action_table 00000001800133a0     libucrt:exception_filter.obj
 0002:00001460       __acrt_signal_action_table_count 0000000180013460     libucrt:exception_filter.obj
 0002:00001468       __acrt_signal_action_first_fpe_index 0000000180013468     libucrt:exception_filter.obj
 0002:00001470       __acrt_signal_action_fpe_count 0000000180013470     libucrt:exception_filter.obj
 0002:00001478       ??_C@_1BI@BGOHAHKC@?$AAm?$AAs?$AAc?$AAo?$AAr?$AAe?$AAe?$AA?4?$AAd?$AAl?$AAl@ 0000000180013478     libucrt:exit.obj
 0002:00001490       ??_C@_0P@MIGLKIOC@CorExitProcess@ 0000000180013490     libucrt:exit.obj
 0002:00001728       ??_C@_1M@HPNHIDJI@?$AAj?$AAa?$AA?9?$AAJ?$AAP@ 0000000180013728     libucrt:mbctype.obj
 0002:00001738       ??_C@_1M@BIBDDEMK@?$AAz?$AAh?$AA?9?$AAC?$AAN@ 0000000180013738     libucrt:mbctype.obj
 0002:00001748       ??_C@_1M@JLOOOEGK@?$AAk?$AAo?$AA?9?$AAK?$AAR@ 0000000180013748     libucrt:mbctype.obj
 0002:00001758       ??_C@_1M@CLNBBOPM@?$AAz?$AAh?$AA?9?$AAT?$AAW@ 0000000180013758     libucrt:mbctype.obj
 0002:00001810       ??_C@_1EA@JGEFHKEI@?$AAa?$AAp?$AAi?$AA?9?$AAm?$AAs?$AA?9?$AAw?$AAi?$AAn?$AA?9?$AAc?$AAo?$AAr?$AAe@ 0000000180013810     libucrt:winapi_thunks.obj
 0002:00001850       ??_C@_1DI@IJCEHOCB@?$AAa?$AAp?$AAi?$AA?9?$AAm?$AAs?$AA?9?$AAw?$AAi?$AAn?$AA?9?$AAc?$AAo?$AAr?$AAe@ 0000000180013850     libucrt:winapi_thunks.obj
 0002:00001890       ??_C@_1EI@MPIAOHOC@?$AAa?$AAp?$AAi?$AA?9?$AAm?$AAs?$AA?9?$AAw?$AAi?$AAn?$AA?9?$AAc?$AAo?$AAr?$AAe@ 0000000180013890     libucrt:winapi_thunks.obj
 0002:000018e0       ??_C@_1FK@FPHCKFIE@?$AAa?$AAp?$AAi?$AA?9?$AAm?$AAs?$AA?9?$AAw?$AAi?$AAn?$AA?9?$AAc?$AAo?$AAr?$AAe@ 00000001800138e0     libucrt:winapi_thunks.obj
 0002:00001940       ??_C@_1EM@DILCGIIO@?$AAa?$AAp?$AAi?$AA?9?$AAm?$AAs?$AA?9?$AAw?$AAi?$AAn?$AA?9?$AAc?$AAo?$AAr?$AAe@ 0000000180013940     libucrt:winapi_thunks.obj
 0002:00001990       ??_C@_1DM@LNCGDDPN@?$AAa?$AAp?$AAi?$AA?9?$AAm?$AAs?$AA?9?$AAw?$AAi?$AAn?$AA?9?$AAc?$AAo?$AAr?$AAe@ 0000000180013990     libucrt:winapi_thunks.obj
 0002:000019d0       ??_C@_1DO@FPAPJEMD@?$AAa?$AAp?$AAi?$AA?9?$AAm?$AAs?$AA?9?$AAw?$AAi?$AAn?$AA?9?$AAc?$AAo?$AAr?$AAe@ 00000001800139d0     libucrt:winapi_thunks.obj
 0002:00001a10       ??_C@_1DK@NDHNAHIO@?$AAa?$AAp?$AAi?$AA?9?$AAm?$AAs?$AA?9?$AAw?$AAi?$AAn?$AA?9?$AAc?$AAo?$AAr?$AAe@ 0000000180013a10     libucrt:winapi_thunks.obj
 0002:00001a50       ??_C@_1DM@KGHDGBCM@?$AAa?$AAp?$AAi?$AA?9?$AAm?$AAs?$AA?9?$AAw?$AAi?$AAn?$AA?9?$AAc?$AAo?$AAr?$AAe@ 0000000180013a50     libucrt:winapi_thunks.obj
 0002:00001a90       ??_C@_1EO@IJIOEFOH@?$AAa?$AAp?$AAi?$AA?9?$AAm?$AAs?$AA?9?$AAw?$AAi?$AAn?$AA?9?$AAr?$AAt?$AAc?$AAo@ 0000000180013a90     libucrt:winapi_thunks.obj
 0002:00001ae0       ??_C@_1FG@HHGEKANL@?$AAa?$AAp?$AAi?$AA?9?$AAm?$AAs?$AA?9?$AAw?$AAi?$AAn?$AA?9?$AAs?$AAe?$AAc?$AAu@ 0000000180013ae0     libucrt:winapi_thunks.obj
 0002:00001b40       ??_C@_1EG@DBIOJECG@?$AAe?$AAx?$AAt?$AA?9?$AAm?$AAs?$AA?9?$AAw?$AAi?$AAn?$AA?9?$AAn?$AAt?$AAu?$AAs@ 0000000180013b40     libucrt:winapi_thunks.obj
 0002:00001b90       ??_C@_1EO@FIHMJCLF@?$AAe?$AAx?$AAt?$AA?9?$AAm?$AAs?$AA?9?$AAw?$AAi?$AAn?$AA?9?$AAn?$AAt?$AAu?$AAs@ 0000000180013b90     libucrt:winapi_thunks.obj
 0002:00001be0       ??_C@_1BC@DNHGCMLG@?$AAa?$AAd?$AAv?$AAa?$AAp?$AAi?$AA3?$AA2@ 0000000180013be0     libucrt:winapi_thunks.obj
 0002:00001bf8       ??_C@_1M@OAIMIKLP@?$AAn?$AAt?$AAd?$AAl?$AAl@ 0000000180013bf8     libucrt:winapi_thunks.obj
 0002:00001c10       ??_C@_1EG@DPGNFKGC@?$AAa?$AAp?$AAi?$AA?9?$AAm?$AAs?$AA?9?$AAw?$AAi?$AAn?$AA?9?$AAa?$AAp?$AAp?$AAm@ 0000000180013c10     libucrt:winapi_thunks.obj
 0002:00001c58       ??_C@_1O@BCCLBEOE@?$AAu?$AAs?$AAe?$AAr?$AA3?$AA2@ 0000000180013c58     libucrt:winapi_thunks.obj
 0002:00001c68       ??_C@_1BA@IAIFMGEF@?$AAe?$AAx?$AAt?$AA?9?$AAm?$AAs?$AA?9@ 0000000180013c68     libucrt:winapi_thunks.obj
 0002:00001c80       ??_C@_0BA@FHFNEAED@AreFileApisANSI@ 0000000180013c80     libucrt:winapi_thunks.obj
 0002:00001cc0       ??_C@_0O@KKBNKAPF@LCMapStringEx@ 0000000180013cc0     libucrt:winapi_thunks.obj
 0002:00001cd8       ??_C@_0BB@HBDEELFH@LocaleNameToLCID@ 0000000180013cd8     libucrt:winapi_thunks.obj
 0002:00001cf0       ??_C@_0CF@OJOFEIGO@AppPolicyGetProcessTerminationM@ 0000000180013cf0     libucrt:winapi_thunks.obj
 0002:00001d20       __lc_time_c                0000000180013d20     libucrt:nlsdata.obj
 0002:00001fe0       ??_C@_03KOEHGMDN@Sun@      0000000180013fe0     libucrt:nlsdata.obj
 0002:00001fe4       ??_C@_03PDAGKDH@Mon@       0000000180013fe4     libucrt:nlsdata.obj
 0002:00001fe8       ??_C@_03NAGEINEP@Tue@      0000000180013fe8     libucrt:nlsdata.obj
 0002:00001fec       ??_C@_03MHOMLAJA@Wed@      0000000180013fec     libucrt:nlsdata.obj
 0002:00001ff0       ??_C@_03IOFIKPDN@Thu@      0000000180013ff0     libucrt:nlsdata.obj
 0002:00001ff4       ??_C@_03IDIOELNC@Fri@      0000000180013ff4     libucrt:nlsdata.obj
 0002:00001ff8       ??_C@_03FEFJNEK@Sat@       0000000180013ff8     libucrt:nlsdata.obj
 0002:00001ffc       ??_C@_06OOPIFAJ@Sunday@    0000000180013ffc     libucrt:nlsdata.obj
 0002:00002004       ??_C@_06JLEDEDGH@Monday@   0000000180014004     libucrt:nlsdata.obj
 0002:00002010       ??_C@_07BAAGCFCM@Tuesday@  0000000180014010     libucrt:nlsdata.obj
 0002:00002018       ??_C@_09DLIGFAKA@Wednesday@ 0000000180014018     libucrt:nlsdata.obj
 0002:00002028       ??_C@_08HACCIKIA@Thursday@ 0000000180014028     libucrt:nlsdata.obj
 0002:00002034       ??_C@_06JECMNKMI@Friday@   0000000180014034     libucrt:nlsdata.obj
 0002:00002040       ??_C@_08INBOOONO@Saturday@ 0000000180014040     libucrt:nlsdata.obj
 0002:0000204c       ??_C@_03JIHJHPIE@Jan@      000000018001404c     libucrt:nlsdata.obj
 0002:00002050       ??_C@_03HJBDCHOM@Feb@      0000000180014050     libucrt:nlsdata.obj
 0002:00002054       ??_C@_03ODNJBKGA@Mar@      0000000180014054     libucrt:nlsdata.obj
 0002:00002058       ??_C@_03LEOLGMJP@Apr@      0000000180014058     libucrt:nlsdata.obj
 0002:0000205c       ??_C@_03CNMDKL@May@        000000018001405c     libucrt:nlsdata.obj
 0002:00002060       ??_C@_03IDFGHECI@Jun@      0000000180014060     libucrt:nlsdata.obj
 0002:00002064       ??_C@_03LBGABGKK@Jul@      0000000180014064     libucrt:nlsdata.obj
 0002:00002068       ??_C@_03IFJFEIGA@Aug@      0000000180014068     libucrt:nlsdata.obj
 0002:0000206c       ??_C@_03GGCAPAJC@Sep@      000000018001406c     libucrt:nlsdata.obj
 0002:00002070       ??_C@_03BMAOKBAD@Oct@      0000000180014070     libucrt:nlsdata.obj
 0002:00002074       ??_C@_03JPJOFNIA@Nov@      0000000180014074     libucrt:nlsdata.obj
 0002:00002078       ??_C@_03MKABNOCG@Dec@      0000000180014078     libucrt:nlsdata.obj
 0002:00002080       ??_C@_07CGJPFGJA@January@  0000000180014080     libucrt:nlsdata.obj
 0002:00002088       ??_C@_08GNJGEPFN@February@ 0000000180014088     libucrt:nlsdata.obj
 0002:00002094       ??_C@_05HPCKOFNC@March@    0000000180014094     libucrt:nlsdata.obj
 0002:0000209c       ??_C@_05DMJDNLEJ@April@    000000018001409c     libucrt:nlsdata.obj
 0002:000020a4       ??_C@_04CNLMGBGM@June@     00000001800140a4     libucrt:nlsdata.obj
 0002:000020ac       ??_C@_04MIEPOIFP@July@     00000001800140ac     libucrt:nlsdata.obj
 0002:000020b4       ??_C@_06LBBHFDDG@August@   00000001800140b4     libucrt:nlsdata.obj
 0002:000020c0       ??_C@_09BHHEALKD@September@ 00000001800140c0     libucrt:nlsdata.obj
 0002:000020d0       ??_C@_07JJNFCEND@October@  00000001800140d0     libucrt:nlsdata.obj
 0002:000020d8       ??_C@_08HCHEGEOA@November@ 00000001800140d8     libucrt:nlsdata.obj
 0002:000020e8       ??_C@_08EDHMEBNP@December@ 00000001800140e8     libucrt:nlsdata.obj
 0002:000020f4       ??_C@_02DEDBPAFC@AM@       00000001800140f4     libucrt:nlsdata.obj
 0002:000020f8       ??_C@_02CJNFDJBF@PM@       00000001800140f8     libucrt:nlsdata.obj
 0002:00002100       ??_C@_08BPBNCDIB@MM?1dd?1yy@ 0000000180014100     libucrt:nlsdata.obj
 0002:00002110       ??_C@_0BE@CKGJFCPC@dddd?0?5MMMM?5dd?0?5yyyy@ 0000000180014110     libucrt:nlsdata.obj
 0002:00002128       ??_C@_08JCCMCCIL@HH?3mm?3ss@ 0000000180014128     libucrt:nlsdata.obj
 0002:00002138       ??_C@_17MBGCMIPB@?$AAS?$AAu?$AAn@ 0000000180014138     libucrt:nlsdata.obj
 0002:00002140       ??_C@_17KBOMKBF@?$AAM?$AAo?$AAn@ 0000000180014140     libucrt:nlsdata.obj
 0002:00002148       ??_C@_17BMKGEGOJ@?$AAT?$AAu?$AAe@ 0000000180014148     libucrt:nlsdata.obj
 0002:00002150       ??_C@_17CJEDCEPE@?$AAW?$AAe?$AAd@ 0000000180014150     libucrt:nlsdata.obj
 0002:00002158       ??_C@_17PDPHAADD@?$AAT?$AAh?$AAu@ 0000000180014158     libucrt:nlsdata.obj
 0002:00002160       ??_C@_17HFOLPPLP@?$AAF?$AAr?$AAi@ 0000000180014160     libucrt:nlsdata.obj
 0002:00002168       ??_C@_17GGIBDPIH@?$AAS?$AAa?$AAt@ 0000000180014168     libucrt:nlsdata.obj
 0002:00002170       ??_C@_1O@IHNHDHPB@?$AAS?$AAu?$AAn?$AAd?$AAa?$AAy@ 0000000180014170     libucrt:nlsdata.obj
 0002:00002180       ??_C@_1O@MMNBFLIA@?$AAM?$AAo?$AAn?$AAd?$AAa?$AAy@ 0000000180014180     libucrt:nlsdata.obj
 0002:00002190       ??_C@_1BA@ENFBFFEK@?$AAT?$AAu?$AAe?$AAs?$AAd?$AAa?$AAy@ 0000000180014190     libucrt:nlsdata.obj
 0002:000021a0       ??_C@_1BE@EBOGMDOH@?$AAW?$AAe?$AAd?$AAn?$AAe?$AAs?$AAd?$AAa?$AAy@ 00000001800141a0     libucrt:nlsdata.obj
 0002:000021b8       ??_C@_1BC@HHMNLIHE@?$AAT?$AAh?$AAu?$AAr?$AAs?$AAd?$AAa?$AAy@ 00000001800141b8     libucrt:nlsdata.obj
 0002:000021d0       ??_C@_1O@PDICJHAG@?$AAF?$AAr?$AAi?$AAd?$AAa?$AAy@ 00000001800141d0     libucrt:nlsdata.obj
 0002:000021e0       ??_C@_1BC@ENMNNPAJ@?$AAS?$AAa?$AAt?$AAu?$AAr?$AAd?$AAa?$AAy@ 00000001800141e0     libucrt:nlsdata.obj
 0002:000021f8       ??_C@_17DKNBKCHM@?$AAJ?$AAa?$AAn@ 00000001800141f8     libucrt:nlsdata.obj
 0002:00002200       ??_C@_17LMDJEKJN@?$AAF?$AAe?$AAb@ 0000000180014200     libucrt:nlsdata.obj
 0002:00002208       ??_C@_17CKNLEDEC@?$AAM?$AAa?$AAr@ 0000000180014208     libucrt:nlsdata.obj
 0002:00002210       ??_C@_17LFPOIHDD@?$AAA?$AAp?$AAr@ 0000000180014210     libucrt:nlsdata.obj
 0002:00002218       ??_C@_17PNNKMEED@?$AAM?$AAa?$AAy@ 0000000180014218     libucrt:nlsdata.obj
 0002:00002220       ??_C@_17KCJGOCPB@?$AAJ?$AAu?$AAn@ 0000000180014220     libucrt:nlsdata.obj
 0002:00002228       ??_C@_17IJPCKHK@?$AAJ?$AAu?$AAl@ 0000000180014228     libucrt:nlsdata.obj
 0002:00002230       ??_C@_17ICPELBCN@?$AAA?$AAu?$AAg@ 0000000180014230     libucrt:nlsdata.obj
 0002:00002238       ??_C@_17HCHCOKMG@?$AAS?$AAe?$AAp@ 0000000180014238     libucrt:nlsdata.obj
 0002:00002240       ??_C@_17FNLKOI@?$AAO?$AAc?$AAt@ 0000000180014240     libucrt:nlsdata.obj
 0002:00002248       ??_C@_17BBDMLCIG@?$AAN?$AAo?$AAv@ 0000000180014248     libucrt:nlsdata.obj
 0002:00002250       ??_C@_17EGKACKIF@?$AAD?$AAe?$AAc@ 0000000180014250     libucrt:nlsdata.obj
 0002:00002258       ??_C@_1BA@EFMEIEBA@?$AAJ?$AAa?$AAn?$AAu?$AAa?$AAr?$AAy@ 0000000180014258     libucrt:nlsdata.obj
 0002:00002268       ??_C@_1BC@JGDDFFAM@?$AAF?$AAe?$AAb?$AAr?$AAu?$AAa?$AAr?$AAy@ 0000000180014268     libucrt:nlsdata.obj
 0002:00002280       ??_C@_1M@IKEENEDF@?$AAM?$AAa?$AAr?$AAc?$AAh@ 0000000180014280     libucrt:nlsdata.obj
 0002:00002290       ??_C@_1M@GJNLMHFD@?$AAA?$AAp?$AAr?$AAi?$AAl@ 0000000180014290     libucrt:nlsdata.obj
 0002:000022a0       ??_C@_19EPFLPGAP@?$AAJ?$AAu?$AAn?$AAe@ 00000001800142a0     libucrt:nlsdata.obj
 0002:000022b0       ??_C@_19BIFMLPCD@?$AAJ?$AAu?$AAl?$AAy@ 00000001800142b0     libucrt:nlsdata.obj
 0002:000022c0       ??_C@_1O@PAHLKOAC@?$AAA?$AAu?$AAg?$AAu?$AAs?$AAt@ 00000001800142c0     libucrt:nlsdata.obj
 0002:000022d0       ??_C@_1BE@DKAAMBJL@?$AAS?$AAe?$AAp?$AAt?$AAe?$AAm?$AAb?$AAe?$AAr@ 00000001800142d0     libucrt:nlsdata.obj
 0002:000022e8       ??_C@_1BA@EPANDLNG@?$AAO?$AAc?$AAt?$AAo?$AAb?$AAe?$AAr@ 00000001800142e8     libucrt:nlsdata.obj
 0002:000022f8       ??_C@_1BC@BGLIFPF@?$AAN?$AAo?$AAv?$AAe?$AAm?$AAb?$AAe?$AAr@ 00000001800142f8     libucrt:nlsdata.obj
 0002:00002310       ??_C@_1BC@FEMKIFH@?$AAD?$AAe?$AAc?$AAe?$AAm?$AAb?$AAe?$AAr@ 0000000180014310     libucrt:nlsdata.obj
 0002:00002324       ??_C@_15ODEHAHHF@?$AAA?$AAM@ 0000000180014324     libucrt:nlsdata.obj
 0002:0000232c       ??_C@_15CLMNNGEL@?$AAP?$AAM@ 000000018001432c     libucrt:nlsdata.obj
 0002:00002338       ??_C@_1BC@IEBCMHCM@?$AAM?$AAM?$AA?1?$AAd?$AAd?$AA?1?$AAy?$AAy@ 0000000180014338     libucrt:nlsdata.obj
 0002:00002350       ??_C@_1CI@KNAKOEBC@?$AAd?$AAd?$AAd?$AAd?$AA?0?$AA?5?$AAM?$AAM?$AAM?$AAM?$AA?5?$AAd?$AAd?$AA?0?$AA?5@ 0000000180014350     libucrt:nlsdata.obj
 0002:00002378       ??_C@_1BC@GDGBMEMK@?$AAH?$AAH?$AA?3?$AAm?$AAm?$AA?3?$AAs?$AAs@ 0000000180014378     libucrt:nlsdata.obj
 0002:00002390       ??_C@_1M@BMHNFIME@?$AAe?$AAn?$AA?9?$AAU?$AAS@ 0000000180014390     libucrt:nlsdata.obj
 0002:000023a0       __newctype                 00000001800143a0     libucrt:ctype.obj
 0002:000026a0       __newclmap                 00000001800146a0     libucrt:ctype.obj
 0002:00002820       __newcumap                 0000000180014820     libucrt:ctype.obj
 0002:000037e0       ??_C@_15EMKDOKLE@?$AAa?$AAr@ 00000001800157e0     libucrt:lcidtoname_downlevel.obj
 0002:000037e8       ??_C@_15KNPADPLH@?$AAb?$AAg@ 00000001800157e8     libucrt:lcidtoname_downlevel.obj
 0002:000037f0       ??_C@_15EDMHLDMO@?$AAc?$AAa@ 00000001800157f0     libucrt:lcidtoname_downlevel.obj
 0002:000037f8       ??_C@_1O@BPEAJADD@?$AAz?$AAh?$AA?9?$AAC?$AAH?$AAS@ 00000001800157f8     libucrt:lcidtoname_downlevel.obj
 0002:00003808       ??_C@_15LJNHCMNK@?$AAc?$AAs@ 0000000180015808     libucrt:lcidtoname_downlevel.obj
 0002:00003810       ??_C@_15FOMCIDHG@?$AAd?$AAa@ 0000000180015810     libucrt:lcidtoname_downlevel.obj
 0002:00003818       ??_C@_15NBKABECB@?$AAd?$AAe@ 0000000180015818     libucrt:lcidtoname_downlevel.obj
 0002:00003820       ??_C@_15GHPEIIAO@?$AAe?$AAl@ 0000000180015820     libucrt:lcidtoname_downlevel.obj
 0002:00003828       ??_C@_15MNPNEAIF@?$AAe?$AAn@ 0000000180015828     libucrt:lcidtoname_downlevel.obj
 0002:00003830       ??_C@_15GPIOMPMH@?$AAe?$AAs@ 0000000180015830     libucrt:lcidtoname_downlevel.obj
 0002:00003838       ??_C@_15NGLOAKJC@?$AAf?$AAi@ 0000000180015838     libucrt:lcidtoname_downlevel.obj
 0002:00003840       ??_C@_15FBKGNKAM@?$AAf?$AAr@ 0000000180015840     libucrt:lcidtoname_downlevel.obj
 0002:00003848       ??_C@_15KGGCNEFK@?$AAh?$AAe@ 0000000180015848     libucrt:lcidtoname_downlevel.obj
 0002:00003850       ??_C@_15PGHLIDMF@?$AAh?$AAu@ 0000000180015850     libucrt:lcidtoname_downlevel.obj
 0002:00003858       ??_C@_15BIEMAPLM@?$AAi?$AAs@ 0000000180015858     libucrt:lcidtoname_downlevel.obj
 0002:00003860       ??_C@_15IFJLDHAF@?$AAi?$AAt@ 0000000180015860     libucrt:lcidtoname_downlevel.obj
 0002:00003868       ??_C@_15GEMIOCAG@?$AAj?$AAa@ 0000000180015868     libucrt:lcidtoname_downlevel.obj
 0002:00003870       ??_C@_15EPELEGJA@?$AAk?$AAo@ 0000000180015870     libucrt:lcidtoname_downlevel.obj
 0002:00003878       ??_C@_15NDDHIMN@?$AAn?$AAl@ 0000000180015878     libucrt:lcidtoname_downlevel.obj
 0002:00003880       ??_C@_15BPIGNHCD@?$AAn?$AAo@ 0000000180015880     libucrt:lcidtoname_downlevel.obj
 0002:00003888       ??_C@_15DEOPBLCG@?$AAp?$AAl@ 0000000180015888     libucrt:lcidtoname_downlevel.obj
 0002:00003890       ??_C@_15KBECGEFG@?$AAp?$AAt@ 0000000180015890     libucrt:lcidtoname_downlevel.obj
 0002:00003898       ??_C@_15GLJCBFMD@?$AAr?$AAo@ 0000000180015898     libucrt:lcidtoname_downlevel.obj
 0002:000038a0       ??_C@_15FEDGKCDI@?$AAr?$AAu@ 00000001800158a0     libucrt:lcidtoname_downlevel.obj
 0002:000038a8       ??_C@_15GLKMLLHM@?$AAh?$AAr@ 00000001800158a8     libucrt:lcidtoname_downlevel.obj
 0002:000038b0       ??_C@_15CPKMFBDB@?$AAs?$AAk@ 00000001800158b0     libucrt:lcidtoname_downlevel.obj
 0002:000038b8       ??_C@_15BAAIOGMK@?$AAs?$AAq@ 00000001800158b8     libucrt:lcidtoname_downlevel.obj
 0002:000038c0       ??_C@_15INNPNOHD@?$AAs?$AAv@ 00000001800158c0     libucrt:lcidtoname_downlevel.obj
 0002:000038c8       ??_C@_15CABMMOGH@?$AAt?$AAh@ 00000001800158c8     libucrt:lcidtoname_downlevel.obj
 0002:000038d0       ??_C@_15BPLIHJJM@?$AAt?$AAr@ 00000001800158d0     libucrt:lcidtoname_downlevel.obj
 0002:000038d8       ??_C@_15NEOEKKDJ@?$AAu?$AAr@ 00000001800158d8     libucrt:lcidtoname_downlevel.obj
 0002:000038e0       ??_C@_15NFICGAJK@?$AAi?$AAd@ 00000001800158e0     libucrt:lcidtoname_downlevel.obj
 0002:000038e8       ??_C@_15PJPFLCCM@?$AAu?$AAk@ 00000001800158e8     libucrt:lcidtoname_downlevel.obj
 0002:000038f0       ??_C@_15HPJPHDM@?$AAb?$AAe@ 00000001800158f0     libucrt:lcidtoname_downlevel.obj
 0002:000038f8       ??_C@_15LCHLGJII@?$AAs?$AAl@ 00000001800158f8     libucrt:lcidtoname_downlevel.obj
 0002:00003900       ??_C@_15PCFJPHHO@?$AAe?$AAt@ 0000000180015900     libucrt:lcidtoname_downlevel.obj
 0002:00003908       ??_C@_15HPFPGODN@?$AAl?$AAv@ 0000000180015908     libucrt:lcidtoname_downlevel.obj
 0002:00003910       ??_C@_15NFFGKGLG@?$AAl?$AAt@ 0000000180015910     libucrt:lcidtoname_downlevel.obj
 0002:00003918       ??_C@_15BDAKCCHN@?$AAf?$AAa@ 0000000180015918     libucrt:lcidtoname_downlevel.obj
 0002:00003920       ??_C@_15NFGIAIAJ@?$AAv?$AAi@ 0000000180015920     libucrt:lcidtoname_downlevel.obj
 0002:00003928       ??_C@_15LMKNDMHN@?$AAh?$AAy@ 0000000180015928     libucrt:lcidtoname_downlevel.obj
 0002:00003930       ??_C@_15IJBHMCFL@?$AAa?$AAz@ 0000000180015930     libucrt:lcidtoname_downlevel.obj
 0002:00003938       ??_C@_15EKOFJABL@?$AAe?$AAu@ 0000000180015938     libucrt:lcidtoname_downlevel.obj
 0002:00003940       ??_C@_15BGHADCNK@?$AAm?$AAk@ 0000000180015940     libucrt:lcidtoname_downlevel.obj
 0002:00003948       ??_C@_15JDNICKHM@?$AAa?$AAf@ 0000000180015948     libucrt:lcidtoname_downlevel.obj
 0002:00003950       ??_C@_15KPJEDBKD@?$AAk?$AAa@ 0000000180015950     libucrt:lcidtoname_downlevel.obj
 0002:00003958       ??_C@_15PDNFFFEO@?$AAf?$AAo@ 0000000180015958     libucrt:lcidtoname_downlevel.obj
 0002:00003960       ??_C@_15OMLEGLOC@?$AAh?$AAi@ 0000000180015960     libucrt:lcidtoname_downlevel.obj
 0002:00003968       ??_C@_15IDNNENKK@?$AAm?$AAs@ 0000000180015968     libucrt:lcidtoname_downlevel.obj
 0002:00003970       ??_C@_15MACJNBMH@?$AAk?$AAk@ 0000000180015970     libucrt:lcidtoname_downlevel.obj
 0002:00003978       ??_C@_15DKDJEOND@?$AAk?$AAy@ 0000000180015978     libucrt:lcidtoname_downlevel.obj
 0002:00003980       ??_C@_15DFGDLJBG@?$AAs?$AAw@ 0000000180015980     libucrt:lcidtoname_downlevel.obj
 0002:00003988       ??_C@_15BBFAICNG@?$AAu?$AAz@ 0000000180015988     libucrt:lcidtoname_downlevel.obj
 0002:00003990       ??_C@_15DKNDCGEA@?$AAt?$AAt@ 0000000180015990     libucrt:lcidtoname_downlevel.obj
 0002:00003998       ??_C@_15MGIFMDPL@?$AAp?$AAa@ 0000000180015998     libucrt:lcidtoname_downlevel.obj
 0002:000039a0       ??_C@_15HCNDBBA@?$AAg?$AAu@ 00000001800159a0     libucrt:lcidtoname_downlevel.obj
 0002:000039a8       ??_C@_15FNBEIBON@?$AAt?$AAa@ 00000001800159a8     libucrt:lcidtoname_downlevel.obj
 0002:000039b0       ??_C@_15NCHGBGLK@?$AAt?$AAe@ 00000001800159b0     libucrt:lcidtoname_downlevel.obj
 0002:000039b8       ??_C@_15PHPHCBPF@?$AAk?$AAn@ 00000001800159b8     libucrt:lcidtoname_downlevel.obj
 0002:000039c0       ??_C@_15DLGBCKMP@?$AAm?$AAr@ 00000001800159c0     libucrt:lcidtoname_downlevel.obj
 0002:000039c8       ??_C@_15EABBLBFF@?$AAs?$AAa@ 00000001800159c8     libucrt:lcidtoname_downlevel.obj
 0002:000039d0       ??_C@_15CBKOMCOI@?$AAm?$AAn@ 00000001800159d0     libucrt:lcidtoname_downlevel.obj
 0002:000039d8       ??_C@_15CKDMCJAF@?$AAg?$AAl@ 00000001800159d8     libucrt:lcidtoname_downlevel.obj
 0002:000039e0       ??_C@_17CNJFBPG@?$AAk?$AAo?$AAk@ 00000001800159e0     libucrt:lcidtoname_downlevel.obj
 0002:000039e8       ??_C@_17FFBJICPL@?$AAs?$AAy?$AAr@ 00000001800159e8     libucrt:lcidtoname_downlevel.obj
 0002:000039f0       ??_C@_17KPNDCPAF@?$AAd?$AAi?$AAv@ 00000001800159f0     libucrt:lcidtoname_downlevel.obj
 0002:000039f8       ??_C@_1M@OKAHONE@?$AAa?$AAr?$AA?9?$AAS?$AAA@ 00000001800159f8     libucrt:lcidtoname_downlevel.obj
 0002:00003a08       ??_C@_1M@FFFIGIGK@?$AAb?$AAg?$AA?9?$AAB?$AAG@ 0000000180015a08     libucrt:lcidtoname_downlevel.obj
 0002:00003a18       ??_C@_1M@BJNKEDC@?$AAc?$AAa?$AA?9?$AAE?$AAS@ 0000000180015a18     libucrt:lcidtoname_downlevel.obj
 0002:00003a28       ??_C@_1M@IJJHFJHA@?$AAc?$AAs?$AA?9?$AAC?$AAZ@ 0000000180015a28     libucrt:lcidtoname_downlevel.obj
 0002:00003a38       ??_C@_1M@CLPEOBGI@?$AAd?$AAa?$AA?9?$AAD?$AAK@ 0000000180015a38     libucrt:lcidtoname_downlevel.obj
 0002:00003a48       ??_C@_1M@MCMADGCB@?$AAd?$AAe?$AA?9?$AAD?$AAE@ 0000000180015a48     libucrt:lcidtoname_downlevel.obj
 0002:00003a58       ??_C@_1M@OOCKEMAM@?$AAe?$AAl?$AA?9?$AAG?$AAR@ 0000000180015a58     libucrt:lcidtoname_downlevel.obj
 0002:00003a68       ??_C@_1M@DDNJFGID@?$AAf?$AAi?$AA?9?$AAF?$AAI@ 0000000180015a68     libucrt:lcidtoname_downlevel.obj
 0002:00003a78       ??_C@_1M@GLIPPMAC@?$AAf?$AAr?$AA?9?$AAF?$AAR@ 0000000180015a78     libucrt:lcidtoname_downlevel.obj
 0002:00003a88       ??_C@_1M@GFMCHPE@?$AAh?$AAe?$AA?9?$AAI?$AAL@ 0000000180015a88     libucrt:lcidtoname_downlevel.obj
 0002:00003a98       ??_C@_1M@MHLPGNKM@?$AAh?$AAu?$AA?9?$AAH?$AAU@ 0000000180015a98     libucrt:lcidtoname_downlevel.obj
 0002:00003aa8       ??_C@_1M@LPDDNNPN@?$AAi?$AAs?$AA?9?$AAI?$AAS@ 0000000180015aa8     libucrt:lcidtoname_downlevel.obj
 0002:00003ab8       ??_C@_1M@MADIPODN@?$AAi?$AAt?$AA?9?$AAI?$AAT@ 0000000180015ab8     libucrt:lcidtoname_downlevel.obj
 0002:00003ac8       ??_C@_1M@IHBJJGG@?$AAn?$AAl?$AA?9?$AAN?$AAL@ 0000000180015ac8     libucrt:lcidtoname_downlevel.obj
 0002:00003ad8       ??_C@_1M@EANAGDL@?$AAn?$AAb?$AA?9?$AAN?$AAO@ 0000000180015ad8     libucrt:lcidtoname_downlevel.obj
 0002:00003ae8       ??_C@_1M@NEIEMEGP@?$AAp?$AAl?$AA?9?$AAP?$AAL@ 0000000180015ae8     libucrt:lcidtoname_downlevel.obj
 0002:00003af8       ??_C@_1M@BOCFIGEP@?$AAp?$AAt?$AA?9?$AAB?$AAR@ 0000000180015af8     libucrt:lcidtoname_downlevel.obj
 0002:00003b08       ??_C@_1M@IMPFOPBG@?$AAr?$AAo?$AA?9?$AAR?$AAO@ 0000000180015b08     libucrt:lcidtoname_downlevel.obj
 0002:00003b18       ??_C@_1M@IDNNEJMM@?$AAr?$AAu?$AA?9?$AAR?$AAU@ 0000000180015b18     libucrt:lcidtoname_downlevel.obj
 0002:00003b28       ??_C@_1M@LILEEOGM@?$AAh?$AAr?$AA?9?$AAH?$AAR@ 0000000180015b28     libucrt:lcidtoname_downlevel.obj
 0002:00003b38       ??_C@_1M@FKIFEHPB@?$AAs?$AAk?$AA?9?$AAS?$AAK@ 0000000180015b38     libucrt:lcidtoname_downlevel.obj
 0002:00003b48       ??_C@_1M@LJMAMNPJ@?$AAs?$AAq?$AA?9?$AAA?$AAL@ 0000000180015b48     libucrt:lcidtoname_downlevel.obj
 0002:00003b58       ??_C@_1M@GIAKDKJK@?$AAs?$AAv?$AA?9?$AAS?$AAE@ 0000000180015b58     libucrt:lcidtoname_downlevel.obj
 0002:00003b68       ??_C@_1M@MKJKIKCL@?$AAt?$AAh?$AA?9?$AAT?$AAH@ 0000000180015b68     libucrt:lcidtoname_downlevel.obj
 0002:00003b78       ??_C@_1M@MFLCCMPB@?$AAt?$AAr?$AA?9?$AAT?$AAR@ 0000000180015b78     libucrt:lcidtoname_downlevel.obj
 0002:00003b88       ??_C@_1M@OIJHDKJN@?$AAu?$AAr?$AA?9?$AAP?$AAK@ 0000000180015b88     libucrt:lcidtoname_downlevel.obj
 0002:00003b98       ??_C@_1M@LHIPCIEK@?$AAi?$AAd?$AA?9?$AAI?$AAD@ 0000000180015b98     libucrt:lcidtoname_downlevel.obj
 0002:00003ba8       ??_C@_1M@MFMOBGI@?$AAu?$AAk?$AA?9?$AAU?$AAA@ 0000000180015ba8     libucrt:lcidtoname_downlevel.obj
 0002:00003bb8       ??_C@_1M@OBGLJIPL@?$AAb?$AAe?$AA?9?$AAB?$AAY@ 0000000180015bb8     libucrt:lcidtoname_downlevel.obj
 0002:00003bc8       ??_C@_1M@BCFAJEAD@?$AAs?$AAl?$AA?9?$AAS?$AAI@ 0000000180015bc8     libucrt:lcidtoname_downlevel.obj
 0002:00003bd8       ??_C@_1M@FKFFEDDN@?$AAe?$AAt?$AA?9?$AAE?$AAE@ 0000000180015bd8     libucrt:lcidtoname_downlevel.obj
 0002:00003be8       ??_C@_1M@KGKKAACI@?$AAl?$AAv?$AA?9?$AAL?$AAV@ 0000000180015be8     libucrt:lcidtoname_downlevel.obj
 0002:00003bf8       ??_C@_1M@IFGBIJO@?$AAl?$AAt?$AA?9?$AAL?$AAT@ 0000000180015bf8     libucrt:lcidtoname_downlevel.obj
 0002:00003c08       ??_C@_1M@FGEAHEDM@?$AAf?$AAa?$AA?9?$AAI?$AAR@ 0000000180015c08     libucrt:lcidtoname_downlevel.obj
 0002:00003c18       ??_C@_1M@KBMAIBFN@?$AAv?$AAi?$AA?9?$AAV?$AAN@ 0000000180015c18     libucrt:lcidtoname_downlevel.obj
 0002:00003c28       ??_C@_1M@GPCBKDJK@?$AAh?$AAy?$AA?9?$AAA?$AAM@ 0000000180015c28     libucrt:lcidtoname_downlevel.obj
 0002:00003c38       ??_C@_1BG@BECMDDJB@?$AAa?$AAz?$AA?9?$AAA?$AAZ?$AA?9?$AAL?$AAa?$AAt?$AAn@ 0000000180015c38     libucrt:lcidtoname_downlevel.obj
 0002:00003c50       ??_C@_1M@MAOFCAEA@?$AAe?$AAu?$AA?9?$AAE?$AAS@ 0000000180015c50     libucrt:lcidtoname_downlevel.obj
 0002:00003c60       ??_C@_1M@IGHABKPI@?$AAm?$AAk?$AA?9?$AAM?$AAK@ 0000000180015c60     libucrt:lcidtoname_downlevel.obj
 0002:00003c70       ??_C@_1M@IAIGNEJG@?$AAt?$AAn?$AA?9?$AAZ?$AAA@ 0000000180015c70     libucrt:lcidtoname_downlevel.obj
 0002:00003c80       ??_C@_1M@IIJCOJFA@?$AAx?$AAh?$AA?9?$AAZ?$AAA@ 0000000180015c80     libucrt:lcidtoname_downlevel.obj
 0002:00003c90       ??_C@_1M@LGPJHNJH@?$AAz?$AAu?$AA?9?$AAZ?$AAA@ 0000000180015c90     libucrt:lcidtoname_downlevel.obj
 0002:00003ca0       ??_C@_1M@HOKAOIO@?$AAa?$AAf?$AA?9?$AAZ?$AAA@ 0000000180015ca0     libucrt:lcidtoname_downlevel.obj
 0002:00003cb0       ??_C@_1M@DPCLHLIE@?$AAk?$AAa?$AA?9?$AAG?$AAE@ 0000000180015cb0     libucrt:lcidtoname_downlevel.obj
 0002:00003cc0       ??_C@_1M@BLKMHJBI@?$AAf?$AAo?$AA?9?$AAF?$AAO@ 0000000180015cc0     libucrt:lcidtoname_downlevel.obj
 0002:00003cd0       ??_C@_1M@LGGJAPPB@?$AAh?$AAi?$AA?9?$AAI?$AAN@ 0000000180015cd0     libucrt:lcidtoname_downlevel.obj
 0002:00003ce0       ??_C@_1M@FIKPIHFE@?$AAm?$AAt?$AA?9?$AAM?$AAT@ 0000000180015ce0     libucrt:lcidtoname_downlevel.obj
 0002:00003cf0       ??_C@_1M@HEGGPBFA@?$AAs?$AAe?$AA?9?$AAN?$AAO@ 0000000180015cf0     libucrt:lcidtoname_downlevel.obj
 0002:00003d00       ??_C@_1M@EIBJEEPA@?$AAm?$AAs?$AA?9?$AAM?$AAY@ 0000000180015d00     libucrt:lcidtoname_downlevel.obj
 0002:00003d10       ??_C@_1M@FHLBGMPP@?$AAk?$AAk?$AA?9?$AAK?$AAZ@ 0000000180015d10     libucrt:lcidtoname_downlevel.obj
 0002:00003d20       ??_C@_1M@NGJJLCGI@?$AAk?$AAy?$AA?9?$AAK?$AAG@ 0000000180015d20     libucrt:lcidtoname_downlevel.obj
 0002:00003d30       ??_C@_1M@GIENNBFC@?$AAs?$AAw?$AA?9?$AAK?$AAE@ 0000000180015d30     libucrt:lcidtoname_downlevel.obj
 0002:00003d40       ??_C@_1BG@NDGMJIMJ@?$AAu?$AAz?$AA?9?$AAU?$AAZ?$AA?9?$AAL?$AAa?$AAt?$AAn@ 0000000180015d40     libucrt:lcidtoname_downlevel.obj
 0002:00003d58       ??_C@_1M@IDCCIHBC@?$AAt?$AAt?$AA?9?$AAR?$AAU@ 0000000180015d58     libucrt:lcidtoname_downlevel.obj
 0002:00003d68       ??_C@_1M@LOICPMOJ@?$AAb?$AAn?$AA?9?$AAI?$AAN@ 0000000180015d68     libucrt:lcidtoname_downlevel.obj
 0002:00003d78       ??_C@_1M@KPKKNEAH@?$AAp?$AAa?$AA?9?$AAI?$AAN@ 0000000180015d78     libucrt:lcidtoname_downlevel.obj
 0002:00003d88       ??_C@_1M@PJGPPBOG@?$AAg?$AAu?$AA?9?$AAI?$AAN@ 0000000180015d88     libucrt:lcidtoname_downlevel.obj
 0002:00003d98       ??_C@_1M@KMKMOPHI@?$AAt?$AAa?$AA?9?$AAI?$AAN@ 0000000180015d98     libucrt:lcidtoname_downlevel.obj
 0002:00003da8       ??_C@_1M@KFEHEPAC@?$AAt?$AAe?$AA?9?$AAI?$AAN@ 0000000180015da8     libucrt:lcidtoname_downlevel.obj
 0002:00003db8       ??_C@_1M@CDCLMGHI@?$AAk?$AAn?$AA?9?$AAI?$AAN@ 0000000180015db8     libucrt:lcidtoname_downlevel.obj
 0002:00003dc8       ??_C@_1M@MIODLDKF@?$AAm?$AAl?$AA?9?$AAI?$AAN@ 0000000180015dc8     libucrt:lcidtoname_downlevel.obj
 0002:00003dd8       ??_C@_1M@PBIEACPO@?$AAm?$AAr?$AA?9?$AAI?$AAN@ 0000000180015dd8     libucrt:lcidtoname_downlevel.obj
 0002:00003de8       ??_C@_1M@NIDEAGPH@?$AAs?$AAa?$AA?9?$AAI?$AAN@ 0000000180015de8     libucrt:lcidtoname_downlevel.obj
 0002:00003df8       ??_C@_1M@FHIHCBIO@?$AAm?$AAn?$AA?9?$AAM?$AAN@ 0000000180015df8     libucrt:lcidtoname_downlevel.obj
 0002:00003e08       ??_C@_1M@JAIJPENP@?$AAc?$AAy?$AA?9?$AAG?$AAB@ 0000000180015e08     libucrt:lcidtoname_downlevel.obj
 0002:00003e18       ??_C@_1M@PHGFBEPN@?$AAg?$AAl?$AA?9?$AAE?$AAS@ 0000000180015e18     libucrt:lcidtoname_downlevel.obj
 0002:00003e28       ??_C@_1O@KPIPDNCP@?$AAk?$AAo?$AAk?$AA?9?$AAI?$AAN@ 0000000180015e28     libucrt:lcidtoname_downlevel.obj
 0002:00003e38       ??_C@_1O@KNHJLDJA@?$AAs?$AAy?$AAr?$AA?9?$AAS?$AAY@ 0000000180015e38     libucrt:lcidtoname_downlevel.obj
 0002:00003e48       ??_C@_1O@MKEKBLAH@?$AAd?$AAi?$AAv?$AA?9?$AAM?$AAV@ 0000000180015e48     libucrt:lcidtoname_downlevel.obj
 0002:00003e58       ??_C@_1O@OHDCKDDF@?$AAq?$AAu?$AAz?$AA?9?$AAB?$AAO@ 0000000180015e58     libucrt:lcidtoname_downlevel.obj
 0002:00003e68       ??_C@_1M@LEPJNLFD@?$AAn?$AAs?$AA?9?$AAZ?$AAA@ 0000000180015e68     libucrt:lcidtoname_downlevel.obj
 0002:00003e78       ??_C@_1M@OMLEIIJB@?$AAm?$AAi?$AA?9?$AAN?$AAZ@ 0000000180015e78     libucrt:lcidtoname_downlevel.obj
 0002:00003e88       ??_C@_1M@PMPEAILG@?$AAa?$AAr?$AA?9?$AAI?$AAQ@ 0000000180015e88     libucrt:lcidtoname_downlevel.obj
 0002:00003e98       ??_C@_1M@CNKPNOEE@?$AAd?$AAe?$AA?9?$AAC?$AAH@ 0000000180015e98     libucrt:lcidtoname_downlevel.obj
 0002:00003ea8       ??_C@_1M@LKMGMLKO@?$AAe?$AAn?$AA?9?$AAG?$AAB@ 0000000180015ea8     libucrt:lcidtoname_downlevel.obj
 0002:00003eb8       ??_C@_1M@PGKJFFGL@?$AAe?$AAs?$AA?9?$AAM?$AAX@ 0000000180015eb8     libucrt:lcidtoname_downlevel.obj
 0002:00003ec8       ??_C@_1M@DNNANBDC@?$AAf?$AAr?$AA?9?$AAB?$AAE@ 0000000180015ec8     libucrt:lcidtoname_downlevel.obj
 0002:00003ed8       ??_C@_1M@HLGMDFHM@?$AAi?$AAt?$AA?9?$AAC?$AAH@ 0000000180015ed8     libucrt:lcidtoname_downlevel.obj
 0002:00003ee8       ??_C@_1M@CLLBGJH@?$AAn?$AAl?$AA?9?$AAB?$AAE@ 0000000180015ee8     libucrt:lcidtoname_downlevel.obj
 0002:00003ef8       ??_C@_1M@BODBOGLF@?$AAn?$AAn?$AA?9?$AAN?$AAO@ 0000000180015ef8     libucrt:lcidtoname_downlevel.obj
 0002:00003f08       ??_C@_1M@HFFAHKAD@?$AAp?$AAt?$AA?9?$AAP?$AAT@ 0000000180015f08     libucrt:lcidtoname_downlevel.obj
 0002:00003f18       ??_C@_1BG@LNOAKHIE@?$AAs?$AAr?$AA?9?$AAS?$AAP?$AA?9?$AAL?$AAa?$AAt?$AAn@ 0000000180015f18     libucrt:lcidtoname_downlevel.obj
 0002:00003f30       ??_C@_1M@HBMHBGAK@?$AAs?$AAv?$AA?9?$AAF?$AAI@ 0000000180015f30     libucrt:lcidtoname_downlevel.obj
 0002:00003f40       ??_C@_1BG@DGCJGJBE@?$AAa?$AAz?$AA?9?$AAA?$AAZ?$AA?9?$AAC?$AAy?$AAr?$AAl@ 0000000180015f40     libucrt:lcidtoname_downlevel.obj
 0002:00003f58       ??_C@_1M@KEJDAAHB@?$AAs?$AAe?$AA?9?$AAS?$AAE@ 0000000180015f58     libucrt:lcidtoname_downlevel.obj
 0002:00003f68       ??_C@_1M@HEIBJJAD@?$AAm?$AAs?$AA?9?$AAB?$AAN@ 0000000180015f68     libucrt:lcidtoname_downlevel.obj
 0002:00003f78       ??_C@_1BG@PBGJMCEM@?$AAu?$AAz?$AA?9?$AAU?$AAZ?$AA?9?$AAC?$AAy?$AAr?$AAl@ 0000000180015f78     libucrt:lcidtoname_downlevel.obj
 0002:00003f90       ??_C@_1O@LAOBCMDF@?$AAq?$AAu?$AAz?$AA?9?$AAE?$AAC@ 0000000180015f90     libucrt:lcidtoname_downlevel.obj
 0002:00003fa0       ??_C@_1M@POEEMAIO@?$AAa?$AAr?$AA?9?$AAE?$AAG@ 0000000180015fa0     libucrt:lcidtoname_downlevel.obj
 0002:00003fb0       ??_C@_1M@EFAKDEDL@?$AAz?$AAh?$AA?9?$AAH?$AAK@ 0000000180015fb0     libucrt:lcidtoname_downlevel.obj
 0002:00003fc0       ??_C@_1M@HKKIJHGI@?$AAd?$AAe?$AA?9?$AAA?$AAT@ 0000000180015fc0     libucrt:lcidtoname_downlevel.obj
 0002:00003fd0       ??_C@_1M@KBFBEHJF@?$AAe?$AAn?$AA?9?$AAA?$AAU@ 0000000180015fd0     libucrt:lcidtoname_downlevel.obj
 0002:00003fe0       ??_C@_1M@MNPLFAAH@?$AAe?$AAs?$AA?9?$AAE?$AAS@ 0000000180015fe0     libucrt:lcidtoname_downlevel.obj
 0002:00003ff0       ??_C@_1M@HJOOJFMA@?$AAf?$AAr?$AA?9?$AAC?$AAA@ 0000000180015ff0     libucrt:lcidtoname_downlevel.obj
 0002:00004000       ??_C@_1BG@JPOFPNAB@?$AAs?$AAr?$AA?9?$AAS?$AAP?$AA?9?$AAC?$AAy?$AAr?$AAl@ 0000000180016000     libucrt:lcidtoname_downlevel.obj
 0002:00004018       ??_C@_1M@LNFOCMOB@?$AAs?$AAe?$AA?9?$AAF?$AAI@ 0000000180016018     libucrt:lcidtoname_downlevel.obj
 0002:00004028       ??_C@_1O@MGJBOAMB@?$AAq?$AAu?$AAz?$AA?9?$AAP?$AAE@ 0000000180016028     libucrt:lcidtoname_downlevel.obj
 0002:00004038       ??_C@_1M@GJINLBOK@?$AAa?$AAr?$AA?9?$AAL?$AAY@ 0000000180016038     libucrt:lcidtoname_downlevel.obj
 0002:00004048       ??_C@_1M@GGMNHJNL@?$AAz?$AAh?$AA?9?$AAS?$AAG@ 0000000180016048     libucrt:lcidtoname_downlevel.obj
 0002:00004058       ??_C@_1M@HOIKODND@?$AAd?$AAe?$AA?9?$AAL?$AAU@ 0000000180016058     libucrt:lcidtoname_downlevel.obj
 0002:00004068       ??_C@_1M@DDOCCGFG@?$AAe?$AAn?$AA?9?$AAC?$AAA@ 0000000180016068     libucrt:lcidtoname_downlevel.obj
 0002:00004078       ??_C@_1M@BNOEMJLF@?$AAe?$AAs?$AA?9?$AAG?$AAT@ 0000000180016078     libucrt:lcidtoname_downlevel.obj
 0002:00004088       ??_C@_1M@EOGNKEK@?$AAf?$AAr?$AA?9?$AAC?$AAH@ 0000000180016088     libucrt:lcidtoname_downlevel.obj
 0002:00004098       ??_C@_1M@FLIDJFHL@?$AAh?$AAr?$AA?9?$AAB?$AAA@ 0000000180016098     libucrt:lcidtoname_downlevel.obj
 0002:000040a8       ??_C@_1O@FMCELNAJ@?$AAs?$AAm?$AAj?$AA?9?$AAN?$AAO@ 00000001800160a8     libucrt:lcidtoname_downlevel.obj
 0002:000040b8       ??_C@_1M@JHGLJMGJ@?$AAa?$AAr?$AA?9?$AAD?$AAZ@ 00000001800160b8     libucrt:lcidtoname_downlevel.obj
 0002:000040c8       ??_C@_1M@JKKFDCNP@?$AAz?$AAh?$AA?9?$AAM?$AAO@ 00000001800160c8     libucrt:lcidtoname_downlevel.obj
 0002:000040d8       ??_C@_1M@GEEFALPE@?$AAd?$AAe?$AA?9?$AAL?$AAI@ 00000001800160d8     libucrt:lcidtoname_downlevel.obj
 0002:000040e8       ??_C@_1M@IGEOFBG@?$AAe?$AAn?$AA?9?$AAN?$AAZ@ 00000001800160e8     libucrt:lcidtoname_downlevel.obj
 0002:000040f8       ??_C@_1M@KDBONEHP@?$AAe?$AAs?$AA?9?$AAC?$AAR@ 00000001800160f8     libucrt:lcidtoname_downlevel.obj
 0002:00004108       ??_C@_1M@FHMDOHNN@?$AAf?$AAr?$AA?9?$AAL?$AAU@ 0000000180016108     libucrt:lcidtoname_downlevel.obj
 0002:00004118       ??_C@_1BG@NFKKMAFG@?$AAb?$AAs?$AA?9?$AAB?$AAA?$AA?9?$AAL?$AAa?$AAt?$AAn@ 0000000180016118     libucrt:lcidtoname_downlevel.obj
 0002:00004130       ??_C@_1O@IMNBEMCI@?$AAs?$AAm?$AAj?$AA?9?$AAS?$AAE@ 0000000180016130     libucrt:lcidtoname_downlevel.obj
 0002:00004140       ??_C@_1M@DHHMBNDP@?$AAa?$AAr?$AA?9?$AAM?$AAA@ 0000000180016140     libucrt:lcidtoname_downlevel.obj
 0002:00004150       ??_C@_1M@BNBLJCGH@?$AAe?$AAn?$AA?9?$AAI?$AAE@ 0000000180016150     libucrt:lcidtoname_downlevel.obj
 0002:00004160       ??_C@_1M@GEPAFMDL@?$AAe?$AAs?$AA?9?$AAP?$AAA@ 0000000180016160     libucrt:lcidtoname_downlevel.obj
 0002:00004170       ??_C@_1M@OJONDMDL@?$AAf?$AAr?$AA?9?$AAM?$AAC@ 0000000180016170     libucrt:lcidtoname_downlevel.obj
 0002:00004180       ??_C@_1BG@OBCNFJB@?$AAs?$AAr?$AA?9?$AAB?$AAA?$AA?9?$AAL?$AAa?$AAt?$AAn@ 0000000180016180     libucrt:lcidtoname_downlevel.obj
 0002:00004198       ??_C@_1O@KEMEEGPO@?$AAs?$AAm?$AAa?$AA?9?$AAN?$AAO@ 0000000180016198     libucrt:lcidtoname_downlevel.obj
 0002:000041a8       ??_C@_1M@ELMGFODK@?$AAa?$AAr?$AA?9?$AAT?$AAN@ 00000001800161a8     libucrt:lcidtoname_downlevel.obj
 0002:000041b8       ??_C@_1M@BHDLHFAF@?$AAe?$AAn?$AA?9?$AAZ?$AAA@ 00000001800161b8     libucrt:lcidtoname_downlevel.obj
 0002:000041c8       ??_C@_1M@BMGIGLIF@?$AAe?$AAs?$AA?9?$AAD?$AAO@ 00000001800161c8     libucrt:lcidtoname_downlevel.obj
 0002:000041d8       ??_C@_1BG@CMBHIPBE@?$AAs?$AAr?$AA?9?$AAB?$AAA?$AA?9?$AAC?$AAy?$AAr?$AAl@ 00000001800161d8     libucrt:lcidtoname_downlevel.obj
 0002:000041f0       ??_C@_1O@HEDBLHNP@?$AAs?$AAm?$AAa?$AA?9?$AAS?$AAE@ 00000001800161f0     libucrt:lcidtoname_downlevel.obj
 0002:00004200       ??_C@_1M@DAGCADIM@?$AAa?$AAr?$AA?9?$AAO?$AAM@ 0000000180016200     libucrt:lcidtoname_downlevel.obj
 0002:00004210       ??_C@_1M@FODLMICG@?$AAe?$AAn?$AA?9?$AAJ?$AAM@ 0000000180016210     libucrt:lcidtoname_downlevel.obj
 0002:00004220       ??_C@_1M@DNMLCIHB@?$AAe?$AAs?$AA?9?$AAV?$AAE@ 0000000180016220     libucrt:lcidtoname_downlevel.obj
 0002:00004230       ??_C@_1O@EOKHMKJK@?$AAs?$AAm?$AAs?$AA?9?$AAF?$AAI@ 0000000180016230     libucrt:lcidtoname_downlevel.obj
 0002:00004240       ??_C@_1M@CAFJMKOF@?$AAa?$AAr?$AA?9?$AAY?$AAE@ 0000000180016240     libucrt:lcidtoname_downlevel.obj
 0002:00004250       ??_C@_1M@CBFHIJLI@?$AAe?$AAn?$AA?9?$AAC?$AAB@ 0000000180016250     libucrt:lcidtoname_downlevel.obj
 0002:00004260       ??_C@_1M@BGNFLDN@?$AAe?$AAs?$AA?9?$AAC?$AAO@ 0000000180016260     libucrt:lcidtoname_downlevel.obj
 0002:00004270       ??_C@_1O@JMPHMAMC@?$AAs?$AAm?$AAn?$AA?9?$AAF?$AAI@ 0000000180016270     libucrt:lcidtoname_downlevel.obj
 0002:00004280       ??_C@_1M@JLANABKE@?$AAa?$AAr?$AA?9?$AAS?$AAY@ 0000000180016280     libucrt:lcidtoname_downlevel.obj
 0002:00004290       ??_C@_1M@HPKGCFGN@?$AAe?$AAn?$AA?9?$AAB?$AAZ@ 0000000180016290     libucrt:lcidtoname_downlevel.obj
 0002:000042a0       ??_C@_1M@OLJCMLGM@?$AAe?$AAs?$AA?9?$AAP?$AAE@ 00000001800162a0     libucrt:lcidtoname_downlevel.obj
 0002:000042b0       ??_C@_1M@MKKGFKLE@?$AAa?$AAr?$AA?9?$AAJ?$AAO@ 00000001800162b0     libucrt:lcidtoname_downlevel.obj
 0002:000042c0       ??_C@_1M@EKPGLDNI@?$AAe?$AAn?$AA?9?$AAT?$AAT@ 00000001800162c0     libucrt:lcidtoname_downlevel.obj
 0002:000042d0       ??_C@_1M@OONGHFHE@?$AAe?$AAs?$AA?9?$AAA?$AAR@ 00000001800162d0     libucrt:lcidtoname_downlevel.obj
 0002:000042e0       ??_C@_1M@OOJFGBHE@?$AAa?$AAr?$AA?9?$AAL?$AAB@ 00000001800162e0     libucrt:lcidtoname_downlevel.obj
 0002:000042f0       ??_C@_1M@GCEJHNEG@?$AAe?$AAn?$AA?9?$AAZ?$AAW@ 00000001800162f0     libucrt:lcidtoname_downlevel.obj
 0002:00004300       ??_C@_1M@JNOCAHJI@?$AAe?$AAs?$AA?9?$AAE?$AAC@ 0000000180016300     libucrt:lcidtoname_downlevel.obj
 0002:00004310       ??_C@_1M@JEFHPGGB@?$AAa?$AAr?$AA?9?$AAK?$AAW@ 0000000180016310     libucrt:lcidtoname_downlevel.obj
 0002:00004320       ??_C@_1M@MLKIBJOJ@?$AAe?$AAn?$AA?9?$AAP?$AAH@ 0000000180016320     libucrt:lcidtoname_downlevel.obj
 0002:00004330       ??_C@_1M@BDNIPEND@?$AAe?$AAs?$AA?9?$AAC?$AAL@ 0000000180016330     libucrt:lcidtoname_downlevel.obj
 0002:00004340       ??_C@_1M@MPNMEKBD@?$AAa?$AAr?$AA?9?$AAA?$AAE@ 0000000180016340     libucrt:lcidtoname_downlevel.obj
 0002:00004350       ??_C@_1M@KBJALCPI@?$AAe?$AAs?$AA?9?$AAU?$AAY@ 0000000180016350     libucrt:lcidtoname_downlevel.obj
 0002:00004360       ??_C@_1M@LLCCOAGA@?$AAa?$AAr?$AA?9?$AAB?$AAH@ 0000000180016360     libucrt:lcidtoname_downlevel.obj
 0002:00004370       ??_C@_1M@PBFNCDEL@?$AAe?$AAs?$AA?9?$AAP?$AAY@ 0000000180016370     libucrt:lcidtoname_downlevel.obj
 0002:00004380       ??_C@_1M@EDGINPNP@?$AAa?$AAr?$AA?9?$AAQ?$AAA@ 0000000180016380     libucrt:lcidtoname_downlevel.obj
 0002:00004390       ??_C@_1M@MKDBIIJI@?$AAe?$AAs?$AA?9?$AAB?$AAO@ 0000000180016390     libucrt:lcidtoname_downlevel.obj
 0002:000043a0       ??_C@_1M@CPKKEBLD@?$AAe?$AAs?$AA?9?$AAS?$AAV@ 00000001800163a0     libucrt:lcidtoname_downlevel.obj
 0002:000043b0       ??_C@_1M@NDBGMMJL@?$AAe?$AAs?$AA?9?$AAH?$AAN@ 00000001800163b0     libucrt:lcidtoname_downlevel.obj
 0002:000043c0       ??_C@_1M@JIJIBHDP@?$AAe?$AAs?$AA?9?$AAN?$AAI@ 00000001800163c0     libucrt:lcidtoname_downlevel.obj
 0002:000043d0       ??_C@_1M@CGFMKEEK@?$AAe?$AAs?$AA?9?$AAP?$AAR@ 00000001800163d0     libucrt:lcidtoname_downlevel.obj
 0002:000043e0       ??_C@_1O@ICJHKIIK@?$AAz?$AAh?$AA?9?$AAC?$AAH?$AAT@ 00000001800163e0     libucrt:lcidtoname_downlevel.obj
 0002:000043f0       ??_C@_15CLNEJCE@?$AAs?$AAr@ 00000001800163f0     libucrt:lcidtoname_downlevel.obj
 0002:00005240       ??_C@_1M@KAHEKEIG@?$AAa?$AAf?$AA?9?$AAz?$AAa@ 0000000180017240     libucrt:lcidtoname_downlevel.obj
 0002:00005250       ??_C@_1M@GIECOABL@?$AAa?$AAr?$AA?9?$AAa?$AAe@ 0000000180017250     libucrt:lcidtoname_downlevel.obj
 0002:00005260       ??_C@_1M@BMLMEKGI@?$AAa?$AAr?$AA?9?$AAb?$AAh@ 0000000180017260     libucrt:lcidtoname_downlevel.obj
 0002:00005270       ??_C@_1M@DAPFDGGB@?$AAa?$AAr?$AA?9?$AAd?$AAz@ 0000000180017270     libucrt:lcidtoname_downlevel.obj
 0002:00005280       ??_C@_1M@FJNKGKIG@?$AAa?$AAr?$AA?9?$AAe?$AAg@ 0000000180017280     libucrt:lcidtoname_downlevel.obj
 0002:00005290       ??_C@_1M@FLGKKCLO@?$AAa?$AAr?$AA?9?$AAi?$AAq@ 0000000180017290     libucrt:lcidtoname_downlevel.obj
 0002:000052a0       ??_C@_1M@GNDIPALM@?$AAa?$AAr?$AA?9?$AAj?$AAo@ 00000001800172a0     libucrt:lcidtoname_downlevel.obj
 0002:000052b0       ??_C@_1M@DDMJFMGJ@?$AAa?$AAr?$AA?9?$AAk?$AAw@ 00000001800172b0     libucrt:lcidtoname_downlevel.obj
 0002:000052c0       ??_C@_1M@EJALMLHM@?$AAa?$AAr?$AA?9?$AAl?$AAb@ 00000001800172c0     libucrt:lcidtoname_downlevel.obj
 0002:000052d0       ??_C@_1M@MOBDBLOC@?$AAa?$AAr?$AA?9?$AAl?$AAy@ 00000001800172d0     libucrt:lcidtoname_downlevel.obj
 0002:000052e0       ??_C@_1M@JAOCLHDH@?$AAa?$AAr?$AA?9?$AAm?$AAa@ 00000001800172e0     libucrt:lcidtoname_downlevel.obj
 0002:000052f0       ??_C@_1M@JHPMKJIE@?$AAa?$AAr?$AA?9?$AAo?$AAm@ 00000001800172f0     libucrt:lcidtoname_downlevel.obj
 0002:00005300       ??_C@_1M@OEPGHFNH@?$AAa?$AAr?$AA?9?$AAq?$AAa@ 0000000180017300     libucrt:lcidtoname_downlevel.obj
 0002:00005310       ??_C@_1M@KJDONENM@?$AAa?$AAr?$AA?9?$AAs?$AAa@ 0000000180017310     libucrt:lcidtoname_downlevel.obj
 0002:00005320       ??_C@_1M@DMJDKLKM@?$AAa?$AAr?$AA?9?$AAs?$AAy@ 0000000180017320     libucrt:lcidtoname_downlevel.obj
 0002:00005330       ??_C@_1M@OMFIPEDC@?$AAa?$AAr?$AA?9?$AAt?$AAn@ 0000000180017330     libucrt:lcidtoname_downlevel.obj
 0002:00005340       ??_C@_1M@IHMHGAON@?$AAa?$AAr?$AA?9?$AAy?$AAe@ 0000000180017340     libucrt:lcidtoname_downlevel.obj
 0002:00005350       ??_C@_1BG@KDCPGJGB@?$AAa?$AAz?$AA?9?$AAa?$AAz?$AA?9?$AAc?$AAy?$AAr?$AAl@ 0000000180017350     libucrt:lcidtoname_downlevel.obj
 0002:00005368       ??_C@_1BG@IBCKDDOE@?$AAa?$AAz?$AA?9?$AAa?$AAz?$AA?9?$AAl?$AAa?$AAt?$AAn@ 0000000180017368     libucrt:lcidtoname_downlevel.obj
 0002:00005380       ??_C@_1M@EGPFDCPD@?$AAb?$AAe?$AA?9?$AAb?$AAy@ 0000000180017380     libucrt:lcidtoname_downlevel.obj
 0002:00005390       ??_C@_1M@PCMGMCGC@?$AAb?$AAg?$AA?9?$AAb?$AAg@ 0000000180017390     libucrt:lcidtoname_downlevel.obj
 0002:000053a0       ??_C@_1M@BJBMFGOB@?$AAb?$AAn?$AA?9?$AAi?$AAn@ 00000001800173a0     libucrt:lcidtoname_downlevel.obj
 0002:000053b0       ??_C@_1BG@EAKMMACD@?$AAb?$AAs?$AA?9?$AAb?$AAa?$AA?9?$AAl?$AAa?$AAt?$AAn@ 00000001800173b0     libucrt:lcidtoname_downlevel.obj
 0002:000053c8       ??_C@_1M@KGADAODK@?$AAc?$AAa?$AA?9?$AAe?$AAs@ 00000001800173c8     libucrt:lcidtoname_downlevel.obj
 0002:000053d8       ??_C@_1M@COAJPDHI@?$AAc?$AAs?$AA?9?$AAc?$AAz@ 00000001800173d8     libucrt:lcidtoname_downlevel.obj
 0002:000053e8       ??_C@_1M@DHBHFONH@?$AAc?$AAy?$AA?9?$AAg?$AAb@ 00000001800173e8     libucrt:lcidtoname_downlevel.obj
 0002:000053f8       ??_C@_1M@IMGKELGA@?$AAd?$AAa?$AA?9?$AAd?$AAk@ 00000001800173f8     libucrt:lcidtoname_downlevel.obj
 0002:00005408       ??_C@_1M@NNDGDNGA@?$AAd?$AAe?$AA?9?$AAa?$AAt@ 0000000180017408     libucrt:lcidtoname_downlevel.obj
 0002:00005418       ??_C@_1M@IKDBHEEM@?$AAd?$AAe?$AA?9?$AAc?$AAh@ 0000000180017418     libucrt:lcidtoname_downlevel.obj
 0002:00005428       ??_C@_1M@GFFOJMCJ@?$AAd?$AAe?$AA?9?$AAd?$AAe@ 0000000180017428     libucrt:lcidtoname_downlevel.obj
 0002:00005438       ??_C@_1M@MDNLKBPM@?$AAd?$AAe?$AA?9?$AAl?$AAi@ 0000000180017438     libucrt:lcidtoname_downlevel.obj
 0002:00005448       ??_C@_1M@NJBEEJNL@?$AAd?$AAe?$AA?9?$AAl?$AAu@ 0000000180017448     libucrt:lcidtoname_downlevel.obj
 0002:00005458       ??_C@_1O@GNNELBAP@?$AAd?$AAi?$AAv?$AA?9?$AAm?$AAv@ 0000000180017458     libucrt:lcidtoname_downlevel.obj
 0002:00005468       ??_C@_1M@EJLEOGAE@?$AAe?$AAl?$AA?9?$AAg?$AAr@ 0000000180017468     libucrt:lcidtoname_downlevel.obj
 0002:00005478       ??_C@_1M@GMPONJN@?$AAe?$AAn?$AA?9?$AAa?$AAu@ 0000000180017478     libucrt:lcidtoname_downlevel.obj
 0002:00005488       ??_C@_1M@NIDIIPGF@?$AAe?$AAn?$AA?9?$AAb?$AAz@ 0000000180017488     libucrt:lcidtoname_downlevel.obj
 0002:00005498       ??_C@_1M@JEHMIMFO@?$AAe?$AAn?$AA?9?$AAc?$AAa@ 0000000180017498     libucrt:lcidtoname_downlevel.obj
 0002:000054a8       ??_C@_1M@IGMJCDLA@?$AAe?$AAn?$AA?9?$AAc?$AAb@ 00000001800174a8     libucrt:lcidtoname_downlevel.obj
 0002:000054b8       ??_C@_1M@BNFIGBKG@?$AAe?$AAn?$AA?9?$AAg?$AAb@ 00000001800174b8     libucrt:lcidtoname_downlevel.obj
 0002:000054c8       ??_C@_1M@LKIFDIGP@?$AAe?$AAn?$AA?9?$AAi?$AAe@ 00000001800174c8     libucrt:lcidtoname_downlevel.obj
 0002:000054d8       ??_C@_1M@PJKFGCCO@?$AAe?$AAn?$AA?9?$AAj?$AAm@ 00000001800174d8     libucrt:lcidtoname_downlevel.obj
 0002:000054e8       ??_C@_1M@KPPKEPBO@?$AAe?$AAn?$AA?9?$AAn?$AAz@ 00000001800174e8     libucrt:lcidtoname_downlevel.obj
 0002:000054f8       ??_C@_1M@GMDGLDOB@?$AAe?$AAn?$AA?9?$AAp?$AAh@ 00000001800174f8     libucrt:lcidtoname_downlevel.obj
 0002:00005508       ??_C@_1M@ONGIBJNA@?$AAe?$AAn?$AA?9?$AAt?$AAt@ 0000000180017508     libucrt:lcidtoname_downlevel.obj
 0002:00005518       ??_C@_1M@LLODPCMM@?$AAe?$AAn?$AA?9?$AAu?$AAs@ 0000000180017518     libucrt:lcidtoname_downlevel.obj
 0002:00005528       ??_C@_1M@LAKFNPAN@?$AAe?$AAn?$AA?9?$AAz?$AAa@ 0000000180017528     libucrt:lcidtoname_downlevel.obj
 0002:00005538       ??_C@_1M@MFNHNHEO@?$AAe?$AAn?$AA?9?$AAz?$AAw@ 0000000180017538     libucrt:lcidtoname_downlevel.obj
 0002:00005548       ??_C@_1M@EJEINPHM@?$AAe?$AAs?$AA?9?$AAa?$AAr@ 0000000180017548     libucrt:lcidtoname_downlevel.obj
 0002:00005558       ??_C@_1M@GNKPCCJA@?$AAe?$AAs?$AA?9?$AAb?$AAo@ 0000000180017558     libucrt:lcidtoname_downlevel.obj
 0002:00005568       ??_C@_1M@LEEGFONL@?$AAe?$AAs?$AA?9?$AAc?$AAl@ 0000000180017568     libucrt:lcidtoname_downlevel.obj
 0002:00005578       ??_C@_1M@KGPDPBDF@?$AAe?$AAs?$AA?9?$AAc?$AAo@ 0000000180017578     libucrt:lcidtoname_downlevel.obj
 0002:00005588       ??_C@_1M@EIAHOHH@?$AAe?$AAs?$AA?9?$AAc?$AAr@ 0000000180017588     libucrt:lcidtoname_downlevel.obj
 0002:00005598       ??_C@_1M@LLPGMBIN@?$AAe?$AAs?$AA?9?$AAd?$AAo@ 0000000180017598     libucrt:lcidtoname_downlevel.obj
 0002:000055a8       ??_C@_1M@DKHMKNJA@?$AAe?$AAs?$AA?9?$AAe?$AAc@ 00000001800175a8     libucrt:lcidtoname_downlevel.obj
 0002:000055b8       ??_C@_1M@GKGFPKAP@?$AAe?$AAs?$AA?9?$AAe?$AAs@ 00000001800175b8     libucrt:lcidtoname_downlevel.obj
 0002:000055c8       ??_C@_1M@LKHKGDLN@?$AAe?$AAs?$AA?9?$AAg?$AAt@ 00000001800175c8     libucrt:lcidtoname_downlevel.obj
 0002:000055d8       ??_C@_1M@HEIIGGJD@?$AAe?$AAs?$AA?9?$AAh?$AAn@ 00000001800175d8     libucrt:lcidtoname_downlevel.obj
 0002:000055e8       ??_C@_1M@FBDHPPGD@?$AAe?$AAs?$AA?9?$AAm?$AAx@ 00000001800175e8     libucrt:lcidtoname_downlevel.obj
 0002:000055f8       ??_C@_1M@DPAGLNDH@?$AAe?$AAs?$AA?9?$AAn?$AAi@ 00000001800175f8     libucrt:lcidtoname_downlevel.obj
 0002:00005608       ??_C@_1M@MDGOPGDD@?$AAe?$AAs?$AA?9?$AAp?$AAa@ 0000000180017608     libucrt:lcidtoname_downlevel.obj
 0002:00005618       ??_C@_1M@EMAMGBGE@?$AAe?$AAs?$AA?9?$AAp?$AAe@ 0000000180017618     libucrt:lcidtoname_downlevel.obj
 0002:00005628       ??_C@_1M@IBMCAOEC@?$AAe?$AAs?$AA?9?$AAp?$AAr@ 0000000180017628     libucrt:lcidtoname_downlevel.obj
 0002:00005638       ??_C@_1M@FGMDIJED@?$AAe?$AAs?$AA?9?$AAp?$AAy@ 0000000180017638     libucrt:lcidtoname_downlevel.obj
 0002:00005648       ??_C@_1M@IIDEOLLL@?$AAe?$AAs?$AA?9?$AAs?$AAv@ 0000000180017648     libucrt:lcidtoname_downlevel.obj
 0002:00005658       ??_C@_1M@GAOBIPA@?$AAe?$AAs?$AA?9?$AAu?$AAy@ 0000000180017658     libucrt:lcidtoname_downlevel.obj
 0002:00005668       ??_C@_1M@JKFFICHJ@?$AAe?$AAs?$AA?9?$AAv?$AAe@ 0000000180017668     libucrt:lcidtoname_downlevel.obj
 0002:00005678       ??_C@_1M@PNMLOJDF@?$AAe?$AAt?$AA?9?$AAe?$AAe@ 0000000180017678     libucrt:lcidtoname_downlevel.obj
 0002:00005688       ??_C@_1M@GHHLIKEI@?$AAe?$AAu?$AA?9?$AAe?$AAs@ 0000000180017688     libucrt:lcidtoname_downlevel.obj
 0002:00005698       ??_C@_1M@PBNONODE@?$AAf?$AAa?$AA?9?$AAi?$AAr@ 0000000180017698     libucrt:lcidtoname_downlevel.obj
 0002:000056a8       ??_C@_1M@JEEHPMIL@?$AAf?$AAi?$AA?9?$AAf?$AAi@ 00000001800176a8     libucrt:lcidtoname_downlevel.obj
 0002:000056b8       ??_C@_1M@LMDCNDBA@?$AAf?$AAo?$AA?9?$AAf?$AAo@ 00000001800176b8     libucrt:lcidtoname_downlevel.obj
 0002:000056c8       ??_C@_1M@JKEOHLDK@?$AAf?$AAr?$AA?9?$AAb?$AAe@ 00000001800176c8     libucrt:lcidtoname_downlevel.obj
 0002:000056d8       ??_C@_1M@NOHADPMI@?$AAf?$AAr?$AA?9?$AAc?$AAa@ 00000001800176d8     libucrt:lcidtoname_downlevel.obj
 0002:000056e8       ??_C@_1M@KDHIHAEC@?$AAf?$AAr?$AA?9?$AAc?$AAh@ 00000001800176e8     libucrt:lcidtoname_downlevel.obj
 0002:000056f8       ??_C@_1M@MMBBFGAK@?$AAf?$AAr?$AA?9?$AAf?$AAr@ 00000001800176f8     libucrt:lcidtoname_downlevel.obj
 0002:00005708       ??_C@_1M@PAFNENNF@?$AAf?$AAr?$AA?9?$AAl?$AAu@ 0000000180017708     libucrt:lcidtoname_downlevel.obj
 0002:00005718       ??_C@_1M@EOHDJGDD@?$AAf?$AAr?$AA?9?$AAm?$AAc@ 0000000180017718     libucrt:lcidtoname_downlevel.obj
 0002:00005728       ??_C@_1M@FAPLLOPF@?$AAg?$AAl?$AA?9?$AAe?$AAs@ 0000000180017728     libucrt:lcidtoname_downlevel.obj
 0002:00005738       ??_C@_1M@FOPBFLOO@?$AAg?$AAu?$AA?9?$AAi?$AAn@ 0000000180017738     libucrt:lcidtoname_downlevel.obj
 0002:00005748       ??_C@_1M@KBMCINPM@?$AAh?$AAe?$AA?9?$AAi?$AAl@ 0000000180017748     libucrt:lcidtoname_downlevel.obj
 0002:00005758       ??_C@_1M@BBPHKFPJ@?$AAh?$AAi?$AA?9?$AAi?$AAn@ 0000000180017758     libucrt:lcidtoname_downlevel.obj
 0002:00005768       ??_C@_1M@PMBNDPHD@?$AAh?$AAr?$AA?9?$AAb?$AAa@ 0000000180017768     libucrt:lcidtoname_downlevel.obj
 0002:00005778       ??_C@_1M@BPCKOEGE@?$AAh?$AAr?$AA?9?$AAh?$AAr@ 0000000180017778     libucrt:lcidtoname_downlevel.obj
 0002:00005788       ??_C@_1M@GACBMHKE@?$AAh?$AAu?$AA?9?$AAh?$AAu@ 0000000180017788     libucrt:lcidtoname_downlevel.obj
 0002:00005798       ??_C@_1M@MILPAJJC@?$AAh?$AAy?$AA?9?$AAa?$AAm@ 0000000180017798     libucrt:lcidtoname_downlevel.obj
 0002:000057a8       ??_C@_1M@BABBICEC@?$AAi?$AAd?$AA?9?$AAi?$AAd@ 00000001800177a8     libucrt:lcidtoname_downlevel.obj
 0002:000057b8       ??_C@_1M@BIKNHHPF@?$AAi?$AAs?$AA?9?$AAi?$AAs@ 00000001800177b8     libucrt:lcidtoname_downlevel.obj
 0002:000057c8       ??_C@_1M@NMPCJPHE@?$AAi?$AAt?$AA?9?$AAc?$AAh@ 00000001800177c8     libucrt:lcidtoname_downlevel.obj
 0002:000057d8       ??_C@_1M@GHKGFEDF@?$AAi?$AAt?$AA?9?$AAi?$AAt@ 00000001800177d8     libucrt:lcidtoname_downlevel.obj
 0002:000057e8       ??_C@_1M@NIEJCJJA@?$AAj?$AAa?$AA?9?$AAj?$AAp@ 00000001800177e8     libucrt:lcidtoname_downlevel.obj
 0002:000057f8       ??_C@_1M@JILFNBIM@?$AAk?$AAa?$AA?9?$AAg?$AAe@ 00000001800177f8     libucrt:lcidtoname_downlevel.obj
 0002:00005808       ??_C@_1M@PACPMGPH@?$AAk?$AAk?$AA?9?$AAk?$AAz@ 0000000180017808     libucrt:lcidtoname_downlevel.obj
 0002:00005818       ??_C@_1M@IELFGMHA@?$AAk?$AAn?$AA?9?$AAi?$AAn@ 0000000180017818     libucrt:lcidtoname_downlevel.obj
 0002:00005828       ??_C@_1O@IBBJHCH@?$AAk?$AAo?$AAk?$AA?9?$AAi?$AAn@ 0000000180017828     libucrt:lcidtoname_downlevel.obj
 0002:00005838       ??_C@_1M@DMHAEOGC@?$AAk?$AAo?$AA?9?$AAk?$AAr@ 0000000180017838     libucrt:lcidtoname_downlevel.obj
 0002:00005848       ??_C@_1M@HBAHBIGA@?$AAk?$AAy?$AA?9?$AAk?$AAg@ 0000000180017848     libucrt:lcidtoname_downlevel.obj
 0002:00005858       ??_C@_1M@KPMILCJG@?$AAl?$AAt?$AA?9?$AAl?$AAt@ 0000000180017858     libucrt:lcidtoname_downlevel.obj
 0002:00005868       ??_C@_1M@BDEKKCA@?$AAl?$AAv?$AA?9?$AAl?$AAv@ 0000000180017868     libucrt:lcidtoname_downlevel.obj
 0002:00005878       ??_C@_1M@ELCKCCJJ@?$AAm?$AAi?$AA?9?$AAn?$AAz@ 0000000180017878     libucrt:lcidtoname_downlevel.obj
 0002:00005888       ??_C@_1M@CBOOLAPA@?$AAm?$AAk?$AA?9?$AAm?$AAk@ 0000000180017888     libucrt:lcidtoname_downlevel.obj
 0002:00005898       ??_C@_1M@GPHNBJKN@?$AAm?$AAl?$AA?9?$AAi?$AAn@ 0000000180017898     libucrt:lcidtoname_downlevel.obj
 0002:000058a8       ??_C@_1M@PABJILIG@?$AAm?$AAn?$AA?9?$AAm?$AAn@ 00000001800178a8     libucrt:lcidtoname_downlevel.obj
 0002:000058b8       ??_C@_1M@FGBKKIPG@?$AAm?$AAr?$AA?9?$AAi?$AAn@ 00000001800178b8     libucrt:lcidtoname_downlevel.obj
 0002:000058c8       ??_C@_1M@NDBPDDAL@?$AAm?$AAs?$AA?9?$AAb?$AAn@ 00000001800178c8     libucrt:lcidtoname_downlevel.obj
 0002:000058d8       ??_C@_1M@OPIHOOPI@?$AAm?$AAs?$AA?9?$AAm?$AAy@ 00000001800178d8     libucrt:lcidtoname_downlevel.obj
 0002:000058e8       ??_C@_1M@PPDBCNFM@?$AAm?$AAt?$AA?9?$AAm?$AAt@ 00000001800178e8     libucrt:lcidtoname_downlevel.obj
 0002:000058f8       ??_C@_1M@KDJDKMDD@?$AAn?$AAb?$AA?9?$AAn?$AAo@ 00000001800178f8     libucrt:lcidtoname_downlevel.obj
 0002:00005908       ??_C@_1M@KFCFLMJP@?$AAn?$AAl?$AA?9?$AAb?$AAe@ 0000000180017908     libucrt:lcidtoname_downlevel.obj
 0002:00005918       ??_C@_1M@KPOPDDGO@?$AAn?$AAl?$AA?9?$AAn?$AAl@ 0000000180017918     libucrt:lcidtoname_downlevel.obj
 0002:00005928       ??_C@_1M@LJKPEMLN@?$AAn?$AAn?$AA?9?$AAn?$AAo@ 0000000180017928     libucrt:lcidtoname_downlevel.obj
 0002:00005938       ??_C@_1M@BDGHHBFL@?$AAn?$AAs?$AA?9?$AAz?$AAa@ 0000000180017938     libucrt:lcidtoname_downlevel.obj
 0002:00005948       ??_C@_1M@IDEHOAP@?$AAp?$AAa?$AA?9?$AAi?$AAn@ 0000000180017948     libucrt:lcidtoname_downlevel.obj
 0002:00005958       ??_C@_1M@HDBKGOGH@?$AAp?$AAl?$AA?9?$AAp?$AAl@ 0000000180017958     libucrt:lcidtoname_downlevel.obj
 0002:00005968       ??_C@_1M@LJLLCMEH@?$AAp?$AAt?$AA?9?$AAb?$AAr@ 0000000180017968     libucrt:lcidtoname_downlevel.obj
 0002:00005978       ??_C@_1M@NCMONAAL@?$AAp?$AAt?$AA?9?$AAp?$AAt@ 0000000180017978     libucrt:lcidtoname_downlevel.obj
 0002:00005988       ??_C@_1O@EAKMAJDN@?$AAq?$AAu?$AAz?$AA?9?$AAb?$AAo@ 0000000180017988     libucrt:lcidtoname_downlevel.obj
 0002:00005998       ??_C@_1O@BHHPIGDN@?$AAq?$AAu?$AAz?$AA?9?$AAe?$AAc@ 0000000180017998     libucrt:lcidtoname_downlevel.obj
 0002:000059a8       ??_C@_1O@GBAPEKMJ@?$AAq?$AAu?$AAz?$AA?9?$AAp?$AAe@ 00000001800179a8     libucrt:lcidtoname_downlevel.obj
 0002:000059b8       ??_C@_1M@CLGLEFBO@?$AAr?$AAo?$AA?9?$AAr?$AAo@ 00000001800179b8     libucrt:lcidtoname_downlevel.obj
 0002:000059c8       ??_C@_1M@CEEDODME@?$AAr?$AAu?$AA?9?$AAr?$AAu@ 00000001800179c8     libucrt:lcidtoname_downlevel.obj
 0002:000059d8       ??_C@_1M@HPKKKMPP@?$AAs?$AAa?$AA?9?$AAi?$AAn@ 00000001800179d8     libucrt:lcidtoname_downlevel.obj
 0002:000059e8       ??_C@_1M@BKMAIGOJ@?$AAs?$AAe?$AA?9?$AAf?$AAi@ 00000001800179e8     libucrt:lcidtoname_downlevel.obj
 0002:000059f8       ??_C@_1M@NDPIFLFI@?$AAs?$AAe?$AA?9?$AAn?$AAo@ 00000001800179f8     libucrt:lcidtoname_downlevel.obj
 0002:00005a08       ??_C@_1M@DANKKHJ@?$AAs?$AAe?$AA?9?$AAs?$AAe@ 0000000180017a08     libucrt:lcidtoname_downlevel.obj
 0002:00005a18       ??_C@_1M@PNBLONPJ@?$AAs?$AAk?$AA?9?$AAs?$AAk@ 0000000180017a18     libucrt:lcidtoname_downlevel.obj
 0002:00005a28       ??_C@_1M@LFMODOAL@?$AAs?$AAl?$AA?9?$AAs?$AAi@ 0000000180017a28     libucrt:lcidtoname_downlevel.obj
 0002:00005a38       ??_C@_1O@DFKOMPG@?$AAs?$AAm?$AAa?$AA?9?$AAn?$AAo@ 0000000180017a38     libucrt:lcidtoname_downlevel.obj
 0002:00005a48       ??_C@_1O@NDKPBNNH@?$AAs?$AAm?$AAa?$AA?9?$AAs?$AAe@ 0000000180017a48     libucrt:lcidtoname_downlevel.obj
 0002:00005a58       ??_C@_1O@PLLKBHAB@?$AAs?$AAm?$AAj?$AA?9?$AAn?$AAo@ 0000000180017a58     libucrt:lcidtoname_downlevel.obj
 0002:00005a68       ??_C@_1O@CLEPOGCA@?$AAs?$AAm?$AAj?$AA?9?$AAs?$AAe@ 0000000180017a68     libucrt:lcidtoname_downlevel.obj
 0002:00005a78       ??_C@_1O@DLGJGKMK@?$AAs?$AAm?$AAn?$AA?9?$AAf?$AAi@ 0000000180017a78     libucrt:lcidtoname_downlevel.obj
 0002:00005a88       ??_C@_1O@OJDJGAJC@?$AAs?$AAm?$AAs?$AA?9?$AAf?$AAi@ 0000000180017a88     libucrt:lcidtoname_downlevel.obj
 0002:00005a98       ??_C@_1M@BOFOGHPB@?$AAs?$AAq?$AA?9?$AAa?$AAl@ 0000000180017a98     libucrt:lcidtoname_downlevel.obj
 0002:00005aa8       ??_C@_1BG@LJBBIPGB@?$AAs?$AAr?$AA?9?$AAb?$AAa?$AA?9?$AAc?$AAy?$AAr?$AAl@ 0000000180017aa8     libucrt:lcidtoname_downlevel.obj
 0002:00005ac0       ??_C@_1BG@JLBENFOE@?$AAs?$AAr?$AA?9?$AAb?$AAa?$AA?9?$AAl?$AAa?$AAt?$AAn@ 0000000180017ac0     libucrt:lcidtoname_downlevel.obj
 0002:00005ad8       ??_C@_1BG@KODPNHE@?$AAs?$AAr?$AA?9?$AAs?$AAp?$AA?9?$AAc?$AAy?$AAr?$AAl@ 0000000180017ad8     libucrt:lcidtoname_downlevel.obj
 0002:00005af0       ??_C@_1BG@CIOGKHPB@?$AAs?$AAr?$AA?9?$AAs?$AAp?$AA?9?$AAl?$AAa?$AAt?$AAn@ 0000000180017af0     libucrt:lcidtoname_downlevel.obj
 0002:00005b08       ??_C@_1M@NGFJLMAC@?$AAs?$AAv?$AA?9?$AAf?$AAi@ 0000000180017b08     libucrt:lcidtoname_downlevel.obj
 0002:00005b18       ??_C@_1M@MPJEJAJC@?$AAs?$AAv?$AA?9?$AAs?$AAe@ 0000000180017b18     libucrt:lcidtoname_downlevel.obj
 0002:00005b28       ??_C@_1M@MPNDHLFK@?$AAs?$AAw?$AA?9?$AAk?$AAe@ 0000000180017b28     libucrt:lcidtoname_downlevel.obj
 0002:00005b38       ??_C@_1O@KOHBJJI@?$AAs?$AAy?$AAr?$AA?9?$AAs?$AAy@ 0000000180017b38     libucrt:lcidtoname_downlevel.obj
 0002:00005b48       ??_C@_1M@LDCEFHA@?$AAt?$AAa?$AA?9?$AAi?$AAn@ 0000000180017b48     libucrt:lcidtoname_downlevel.obj
 0002:00005b58       ??_C@_1M@CNJOFAK@?$AAt?$AAe?$AA?9?$AAi?$AAn@ 0000000180017b58     libucrt:lcidtoname_downlevel.obj
 0002:00005b68       ??_C@_1M@GNAECACD@?$AAt?$AAh?$AA?9?$AAt?$AAh@ 0000000180017b68     libucrt:lcidtoname_downlevel.obj
 0002:00005b78       ??_C@_1M@CHBIHOJO@?$AAt?$AAn?$AA?9?$AAz?$AAa@ 0000000180017b78     libucrt:lcidtoname_downlevel.obj
 0002:00005b88       ??_C@_1M@GCCMIGPJ@?$AAt?$AAr?$AA?9?$AAt?$AAr@ 0000000180017b88     libucrt:lcidtoname_downlevel.obj
 0002:00005b98       ??_C@_1M@CELMCNBK@?$AAt?$AAt?$AA?9?$AAr?$AAu@ 0000000180017b98     libucrt:lcidtoname_downlevel.obj
 0002:00005ba8       ??_C@_1M@KLMCELGA@?$AAu?$AAk?$AA?9?$AAu?$AAa@ 0000000180017ba8     libucrt:lcidtoname_downlevel.obj
 0002:00005bb8       ??_C@_1M@EPAJJAJF@?$AAu?$AAr?$AA?9?$AAp?$AAk@ 0000000180017bb8     libucrt:lcidtoname_downlevel.obj
 0002:00005bc8       ??_C@_1BG@GEGPMCDJ@?$AAu?$AAz?$AA?9?$AAu?$AAz?$AA?9?$AAc?$AAy?$AAr?$AAl@ 0000000180017bc8     libucrt:lcidtoname_downlevel.obj
 0002:00005be0       ??_C@_1BG@EGGKJILM@?$AAu?$AAz?$AA?9?$AAu?$AAz?$AA?9?$AAl?$AAa?$AAt?$AAn@ 0000000180017be0     libucrt:lcidtoname_downlevel.obj
 0002:00005bf8       ??_C@_1M@GFOCLFF@?$AAv?$AAi?$AA?9?$AAv?$AAn@ 0000000180017bf8     libucrt:lcidtoname_downlevel.obj
 0002:00005c08       ??_C@_1M@CPAMEDFI@?$AAx?$AAh?$AA?9?$AAz?$AAa@ 0000000180017c08     libucrt:lcidtoname_downlevel.obj
 0002:00005c18       ??_C@_1O@EBKIFIGN@?$AAz?$AAh?$AA?9?$AAc?$AAh?$AAs@ 0000000180017c18     libucrt:lcidtoname_downlevel.obj
 0002:00005c28       ??_C@_1O@NMHPGANE@?$AAz?$AAh?$AA?9?$AAc?$AAh?$AAt@ 0000000180017c28     libucrt:lcidtoname_downlevel.obj
 0002:00005c38       ??_C@_1M@LPINJOMC@?$AAz?$AAh?$AA?9?$AAc?$AAn@ 0000000180017c38     libucrt:lcidtoname_downlevel.obj
 0002:00005c48       ??_C@_1M@OCJEJODD@?$AAz?$AAh?$AA?9?$AAh?$AAk@ 0000000180017c48     libucrt:lcidtoname_downlevel.obj
 0002:00005c58       ??_C@_1M@DNDLJINH@?$AAz?$AAh?$AA?9?$AAm?$AAo@ 0000000180017c58     libucrt:lcidtoname_downlevel.obj
 0002:00005c68       ??_C@_1M@MBFDNDND@?$AAz?$AAh?$AA?9?$AAs?$AAg@ 0000000180017c68     libucrt:lcidtoname_downlevel.obj
 0002:00005c78       ??_C@_1M@IMEPLEPE@?$AAz?$AAh?$AA?9?$AAt?$AAw@ 0000000180017c78     libucrt:lcidtoname_downlevel.obj
 0002:00005c88       ??_C@_1M@BBGHNHJP@?$AAz?$AAu?$AA?9?$AAz?$AAa@ 0000000180017c88     libucrt:lcidtoname_downlevel.obj
 0002:00005ef0       ??_C@_1BA@BALFACEM@?$AAC?$AAO?$AAN?$AAO?$AAU?$AAT?$AA$@ 0000000180017ef0     libucrt:initcon.obj
 0002:00005f00       __log10_256_lead           0000000180017f00     libucrt:log10_256_lead_tail_table.obj
 0002:00006710       __log10_256_tail           0000000180018710     libucrt:log10_256_lead_tail_table.obj
 0002:00006f20       __log_F_inv_qword          0000000180018f20     libucrt:log_f_inv_qword_table.obj
 0002:00007730       ??_C@_05HGHHAHAP@log10@    0000000180019730     libucrt:log_special.obj
 0002:00007750       ??_C@_1BC@DGHEBOMK@?$AAF?$AAi?$AAl?$AAe?$AAC?$AAa?$AAs?$AAe@ 0000000180019750     FileCase.obj
 0002:00007770       ??_C@_1FG@IEAGHMHI@?$AAF?$AAi?$AAl?$AAe?$AA?5?$AAn?$AAa?$AAm?$AAe?$AAs?$AA?5?$AAc?$AAa?$AAs?$AAe@ 0000000180019770     FileCase.obj
 0002:000077c8       ??_C@_1DE@BGKMIKPD@?$AAE?$AAu?$AAg?$AAe?$AAn?$AAe?$AA?5?$AAR?$AAo?$AAs?$AAh?$AAa?$AAl?$AA?5?$AA?$CG@ 00000001800197c8     FileCase.obj
 0002:00007800       ??_C@_1BI@NPBILFDJ@?$AAC?$AAo?$AAn?$AAv?$AAe?$AAr?$AAt?$AAM?$AAo?$AAd?$AAe@ 0000000180019800     FileCase.obj
 0002:00007818       ??_C@_1BO@IKHLKIJC@?$AAC?$AAo?$AAn?$AAv?$AAe?$AAr?$AAt?$AAM?$AAo?$AAd?$AAe?$AAE?$AAx?$AAt@ 0000000180019818     FileCase.obj
 0002:00007838       ??_C@_1BM@HMLICANP@?$AAS?$AAk?$AAi?$AAp?$AAM?$AAi?$AAx?$AAe?$AAd?$AAC?$AAa?$AAs?$AAe@ 0000000180019838     FileCase.obj
 0002:00007858       ??_C@_1BM@BNELJCPP@?$AAP?$AAr?$AAo?$AAc?$AAe?$AAs?$AAs?$AAS?$AAu?$AAb?$AAD?$AAi?$AAr@ 0000000180019858     FileCase.obj
 0002:00007878       ??_C@_1BG@DFJACJCJ@?$AAP?$AAr?$AAo?$AAc?$AAe?$AAs?$AAs?$AAD?$AAi?$AAr@ 0000000180019878     FileCase.obj
 0002:00007890       ??_C@_15NKPPEEJO@?$AA?5?$AA_@ 0000000180019890     FileCase.obj
 0002:00007898       ??_C@_1BA@CAKIGJMA@?$AAW?$AAo?$AAr?$AAd?$AAD?$AAi?$AAv@ 0000000180019898     FileCase.obj
 0002:000078a8       MenuGuid                   00000001800198a8     FileCase.obj
 0002:000078b8       MainGuid                   00000001800198b8     FileCase.obj
 0002:000078c8       DialogGuid                 00000001800198c8     FileCase.obj
 0002:000078d8       ??_C@_0BC@EOODALEL@Unknown?5exception@ 00000001800198d8     filecvt.obj
 0002:000078f0       ??_C@_0BF@KINCDENJ@bad?5array?5new?5length@ 00000001800198f0     filecvt.obj
 0002:00007908       ??_C@_0BA@JFNIOLAK@string?5too?5long@ 0000000180019908     filecvt.obj
 0002:00007918       ??_C@_11LOCGONAA@@         0000000180019918     filecvt.obj
 0002:00007920       ??_C@_1BC@ENICKDH@?$AAC?$AAo?$AAn?$AAt?$AAe?$AAn?$AAt?$AAs@ 0000000180019920     filecvt.obj
 0002:00007938       ??_C@_1CC@CKMDHNMO@?$AAF?$AAi?$AAl?$AAe?$AAC?$AAa?$AAs?$AAe?$AA_?$AAW?$AAo?$AAr?$AAd?$AAD?$AAi@ 0000000180019938     filecvt.obj
 0002:00007968       ??_7PluginCheckBoxBinding@@6B@ 0000000180019968     filecvt.obj
 0002:00007980       ??_7PluginEditFieldBinding@@6B@ 0000000180019980     filecvt.obj
 0002:00007998       ??_7PluginRadioButtonBinding@@6B@ 0000000180019998     filecvt.obj
 0002:000079a8       ??_C@_13JOFGPIOO@?$AA?4@   00000001800199a8     ProcessName.obj
 0002:000079b0       __xmm@00000009000000080000000700000006 00000001800199b0     filecvt.obj
 0002:000079c0       __xmm@0000000e0000000d0000000c0000000b 00000001800199c0     filecvt.obj
 0002:00007a30       _load_config_used          0000000180019a30     LIBCMT:loadcfg.obj
 0002:00007b80       ??_R4type_info@@6B@        0000000180019b80     LIBCMT:std_type_info_static.obj
 0002:00007ba8       ??_R3type_info@@8          0000000180019ba8     LIBCMT:std_type_info_static.obj
 0002:00007bc0       ??_R2type_info@@8          0000000180019bc0     LIBCMT:std_type_info_static.obj
 0002:00007bd0       ??_R1A@?0A@EA@type_info@@8 0000000180019bd0     LIBCMT:std_type_info_static.obj
 0002:00007bf8       ??_R4logic_error@std@@6B@  0000000180019bf8     libcpmt:xthrow.obj
 0002:00007c20       ??_R3logic_error@std@@8    0000000180019c20     libcpmt:xthrow.obj
 0002:00007c38       ??_R2logic_error@std@@8    0000000180019c38     libcpmt:xthrow.obj
 0002:00007c50       ??_R1A@?0A@EA@logic_error@std@@8 0000000180019c50     libcpmt:xthrow.obj
 0002:00007c78       ??_R4length_error@std@@6B@ 0000000180019c78     libcpmt:xthrow.obj
 0002:00007ca0       ??_R3length_error@std@@8   0000000180019ca0     libcpmt:xthrow.obj
 0002:00007cb8       ??_R2length_error@std@@8   0000000180019cb8     libcpmt:xthrow.obj
 0002:00007cd8       ??_R1A@?0A@EA@length_error@std@@8 0000000180019cd8     libcpmt:xthrow.obj
 0002:00007d00       ??_R4bad_exception@std@@6B@ 0000000180019d00     libvcruntime:frame.obj
 0002:00007d28       ??_R3bad_exception@std@@8  0000000180019d28     libvcruntime:frame.obj
 0002:00007d40       ??_R2bad_exception@std@@8  0000000180019d40     libvcruntime:frame.obj
 0002:00007d58       ??_R1A@?0A@EA@bad_exception@std@@8 0000000180019d58     libvcruntime:frame.obj
 0002:00007d80       ??_R4exception@std@@6B@    0000000180019d80     filecvt.obj
 0002:00007da8       ??_R2bad_array_new_length@std@@8 0000000180019da8     filecvt.obj
 0002:00007dc8       ??_R2PluginEditFieldBinding@@8 0000000180019dc8     filecvt.obj
 0002:00007de0       ??_R3DialogAPIBinding@@8   0000000180019de0     filecvt.obj
 0002:00007df8       ??_R1A@?0A@EA@PluginCheckBoxBinding@@8 0000000180019df8     filecvt.obj
 0002:00007e20       ??_R2bad_alloc@std@@8      0000000180019e20     filecvt.obj
 0002:00007e38       ??_R1A@?0A@EA@exception@std@@8 0000000180019e38     filecvt.obj
 0002:00007e60       ??_R2PluginRadioButtonBinding@@8 0000000180019e60     filecvt.obj
 0002:00007e78       ??_R1A@?0A@EA@bad_alloc@std@@8 0000000180019e78     filecvt.obj
 0002:00007ea0       ??_R3PluginRadioButtonBinding@@8 0000000180019ea0     filecvt.obj
 0002:00007eb8       ??_R2exception@std@@8      0000000180019eb8     filecvt.obj
 0002:00007ec8       ??_R4PluginRadioButtonBinding@@6B@ 0000000180019ec8     filecvt.obj
 0002:00007ef0       ??_R3PluginCheckBoxBinding@@8 0000000180019ef0     filecvt.obj
 0002:00007f08       ??_R2DialogAPIBinding@@8   0000000180019f08     filecvt.obj
 0002:00007f18       ??_R3exception@std@@8      0000000180019f18     filecvt.obj
 0002:00007f30       ??_R4PluginEditFieldBinding@@6B@ 0000000180019f30     filecvt.obj
 0002:00007f58       ??_R4bad_alloc@std@@6B@    0000000180019f58     filecvt.obj
 0002:00007f80       ??_R4PluginCheckBoxBinding@@6B@ 0000000180019f80     filecvt.obj
 0002:00007fa8       ??_R1A@?0A@EA@PluginRadioButtonBinding@@8 0000000180019fa8     filecvt.obj
 0002:00007fd0       ??_R3bad_array_new_length@std@@8 0000000180019fd0     filecvt.obj
 0002:00007fe8       ??_R3bad_alloc@std@@8      0000000180019fe8     filecvt.obj
 0002:00008000       ??_R4bad_array_new_length@std@@6B@ 000000018001a000     filecvt.obj
 0002:00008028       ??_R3PluginEditFieldBinding@@8 000000018001a028     filecvt.obj
 0002:00008040       ??_R1A@?0A@EA@bad_array_new_length@std@@8 000000018001a040     filecvt.obj
 0002:00008068       ??_R1A@?0A@EA@PluginEditFieldBinding@@8 000000018001a068     filecvt.obj
 0002:00008090       ??_R2PluginCheckBoxBinding@@8 000000018001a090     filecvt.obj
 0002:000080a8       ??_R1A@?0A@EA@DialogAPIBinding@@8 000000018001a0a8     filecvt.obj
 0002:000080cc       __volatile_metadata        000000018001a0cc     <linker-defined>
 0002:00008448       __rtc_iaa                  000000018001a448     LIBCMT:initsect.obj
 0002:00008450       __rtc_izz                  000000018001a450     LIBCMT:initsect.obj
 0002:00008458       __rtc_taa                  000000018001a458     LIBCMT:initsect.obj
 0002:00008460       __rtc_tzz                  000000018001a460     LIBCMT:initsect.obj
 0002:00009460       _TI2?AVbad_alloc@std@@     000000018001b460     LIBCMT:throw_bad_alloc.obj
 0002:00009480       _CTA2?AVbad_alloc@std@@    000000018001b480     LIBCMT:throw_bad_alloc.obj
 0002:00009498       _CT??_R0?AVlogic_error@std@@@8??0logic_error@std@@QEAA@AEBV01@@Z24 000000018001b498     libcpmt:xthrow.obj
 0002:000094c0       _TI3?AVlength_error@std@@  000000018001b4c0     libcpmt:xthrow.obj
 0002:000094e0       _CTA3?AVlength_error@std@@ 000000018001b4e0     libcpmt:xthrow.obj
 0002:00009500       _CT??_R0?AVlength_error@std@@@8??0length_error@std@@QEAA@AEBV01@@Z24 000000018001b500     libcpmt:xthrow.obj
 0002:00009528       _TI2?AVbad_exception@std@@ 000000018001b528     libvcruntime:frame.obj
 0002:00009548       _CTA2?AVbad_exception@std@@ 000000018001b548     libvcruntime:frame.obj
 0002:00009560       _CT??_R0?AVbad_exception@std@@@8??0bad_exception@std@@QEAA@AEBV01@@Z24 000000018001b560     libvcruntime:frame.obj
 0002:00009588       _CTA3?AVbad_array_new_length@std@@ 000000018001b588     filecvt.obj
 0002:000095a8       _CT??_R0?AVbad_array_new_length@std@@@8??0bad_array_new_length@std@@QEAA@AEBV01@@Z24 000000018001b5a8     filecvt.obj
 0002:000095d0       _CT??_R0?AVbad_alloc@std@@@8??0bad_alloc@std@@QEAA@AEBV01@@Z24 000000018001b5d0     filecvt.obj
 0002:000095f8       _CT??_R0?AVexception@std@@@8??0exception@std@@QEAA@AEBV01@@Z24 000000018001b5f8     filecvt.obj
 0002:00009620       _TI3?AVbad_array_new_length@std@@ 000000018001b620     filecvt.obj
 0002:000096d4       __IMPORT_DESCRIPTOR_KERNEL32 000000018001b6d4     kernel32:KERNEL32.dll
 0002:000096e8       __NULL_IMPORT_DESCRIPTOR   000000018001b6e8     kernel32:KERNEL32.dll
 0003:00000000       __security_cookie_complement 000000018001c000     LIBCMT:gs_cookie.obj
 0003:00000008       __security_cookie          000000018001c008     LIBCMT:gs_cookie.obj
 0003:00000010       __scrt_native_dllmain_reason 000000018001c010     LIBCMT:utility.obj
 0003:00000018       __isa_available            000000018001c018     LIBCMT:cpu_disp.obj
 0003:0000001c       __isa_enabled              000000018001c01c     LIBCMT:cpu_disp.obj
 0003:00000020       __memcpy_nt_iters          000000018001c020     LIBCMT:cpu_disp.obj
 0003:00000028       __memset_nt_iters          000000018001c028     LIBCMT:cpu_disp.obj
 0003:00000040       __abort_behavior           000000018001c040     libucrt:abort.obj
 0003:00000060       __acrt_initial_multibyte_data 000000018001c060     libucrt:mbctype.obj
 0003:000005a0       __acrt_initial_locale_data 000000018001c5a0     libucrt:nlsdata.obj
 0003:000006f8       __acrt_initial_locale_pointers 000000018001c6f8     libucrt:nlsdata.obj
 0003:00000708       __acrt_wide_c_locale_string 000000018001c708     libucrt:nlsdata.obj
 0003:00000710       _iob                       000000018001c710     libucrt:_file.obj
 0003:00000818       __globallocalestatus       000000018001c818     libucrt:glstatus.obj
 0003:00000820       __acrt_lconv_c             000000018001c820     libucrt:localeconv.obj
 0003:000008b8       __acrt_lconv_static_decimal 000000018001c8b8     libucrt:localeconv.obj
 0003:000008bc       __acrt_lconv_static_W_decimal 000000018001c8bc     libucrt:localeconv.obj
 0003:000008c0       _lookuptrailbytes          000000018001c8c0     libucrt:read.obj
 0003:000009d4       _fltused                   000000018001c9d4     LIBCMT:fltused.obj
 0003:000009e0       ??_R0?AVlogic_error@std@@@8 000000018001c9e0     libcpmt:xthrow.obj
 0003:00000a08       ??_R0?AVlength_error@std@@@8 000000018001ca08     libcpmt:xthrow.obj
 0003:00000a30       ??_R0?AVbad_exception@std@@@8 000000018001ca30     libvcruntime:frame.obj
 0003:00000a58       ??_R0?AVbad_alloc@std@@@8  000000018001ca58     filecvt.obj
 0003:00000a80       ??_R0?AVexception@std@@@8  000000018001ca80     filecvt.obj
 0003:00000aa8       ??_R0?AVbad_array_new_length@std@@@8 000000018001caa8     filecvt.obj
 0003:00000ad8       ??_R0?AVtype_info@@@8      000000018001cad8     LIBCMT:std_type_info_static.obj
 0003:00000af8       ??_R0?AVPluginEditFieldBinding@@@8 000000018001caf8     filecvt.obj
 0003:00000b28       ??_R0?AVPluginRadioButtonBinding@@@8 000000018001cb28     filecvt.obj
 0003:00000b58       ??_R0?AVDialogAPIBinding@@@8 000000018001cb58     filecvt.obj
 0003:00000b80       ??_R0?AVPluginCheckBoxBinding@@@8 000000018001cb80     filecvt.obj
 0003:00001130       ?__type_info_root_node@@3U__type_info_node@@A 000000018001d130     LIBCMT:tncleanup.obj
 0003:00001140       ?_OptionsStorage@?1??__local_stdio_printf_options@@9@4_KA 000000018001d140     LIBCMT:default_local_stdio_options.obj
 0003:00001148       ?_OptionsStorage@?1??__local_stdio_scanf_options@@9@4_KA 000000018001d148     LIBCMT:default_local_stdio_options.obj
 0003:00001150       __scrt_current_native_startup_state 000000018001d150     LIBCMT:utility.obj
 0003:00001158       __scrt_native_startup_lock 000000018001d158     LIBCMT:utility.obj
 0003:00001198       __scrt_debugger_hook_flag  000000018001d198     LIBCMT:utility_desktop.obj
 0003:000011a0       __castguard_check_failure_os_handled_fptr 000000018001d1a0     LIBCMT:guard_support.obj
 0003:000011a8       __favor                    000000018001d1a8     LIBCMT:cpu_disp.obj
 0003:000011b0       ?__WinRTOutOfMemoryExceptionCallback@@3P6APEAXXZEA 000000018001d1b0     libvcruntime:ehhelpers.obj
 0003:00001240       __pPurecall                000000018001d240     libvcruntime:purevirt_data.obj
 0003:00001248       ?pArgList@UnDecorator@@0PEAVReplicator@@EA 000000018001d248     libvcruntime:undname.obj
 0003:00001250       ?pZNameList@UnDecorator@@0PEAVReplicator@@EA 000000018001d250     libvcruntime:undname.obj
 0003:00001258       ?pTemplateArgList@UnDecorator@@0PEAVReplicator@@EA 000000018001d258     libvcruntime:undname.obj
 0003:00001260       ?gName@UnDecorator@@0PEBDEB 000000018001d260     libvcruntime:undname.obj
 0003:00001268       ?name@UnDecorator@@0PEBDEB 000000018001d268     libvcruntime:undname.obj
 0003:00001270       ?disableFlags@UnDecorator@@0KA 000000018001d270     libvcruntime:undname.obj
 0003:00001274       ?fExplicitTemplateParams@UnDecorator@@0_NA 000000018001d274     libvcruntime:undname.obj
 0003:00001275       ?fGetTemplateArgumentList@UnDecorator@@0_NA 000000018001d275     libvcruntime:undname.obj
 0003:00001278       ?m_pGetParameter@UnDecorator@@0P6APEADJ@ZEA 000000018001d278     libvcruntime:undname.obj
 0003:00001280       ?m_CHPENameOffset@UnDecorator@@0KA 000000018001d280     libvcruntime:undname.obj
 0003:00001284       ?m_recursionLevel@UnDecorator@@0KA 000000018001d284     libvcruntime:undname.obj
 0003:00001340       ?c_exit_complete@?1???R<lambda_6e4b09c48022b2350581041d5f6b0c4c>@@QEBA@XZ@4_NA 000000018001d340     libucrt:exit.obj
 0003:00001458       _environ_table             000000018001d458     libucrt:environment_initialization.obj
 0003:00001460       _wenviron_table            000000018001d460     libucrt:environment_initialization.obj
 0003:00001468       __dcrt_initial_wide_environment 000000018001d468     libucrt:environment_initialization.obj
 0003:00001470       __dcrt_initial_narrow_environment 000000018001d470     libucrt:environment_initialization.obj
 0003:00001478       __acrt_atexit_table        000000018001d478     libucrt:onexit.obj
 0003:00001490       __acrt_at_quick_exit_table 000000018001d490     libucrt:onexit.obj
 0003:000016e8       _mbctype                   000000018001d6e8     libucrt:mbctype.obj
 0003:000016f0       _mbcasemap                 000000018001d6f0     libucrt:mbctype.obj
 0003:000016f8       __acrt_current_multibyte_data 000000018001d6f8     libucrt:mbctype.obj
 0003:00001708       _pgmptr                    000000018001d708     libucrt:argv_data.obj
 0003:00001710       __argc                     000000018001d710     libucrt:argv_data.obj
 0003:00001718       __argv                     000000018001d718     libucrt:argv_data.obj
 0003:00001720       __wargv                    000000018001d720     libucrt:argv_data.obj
 0003:00001728       _acmdln                    000000018001d728     libucrt:argv_data.obj
 0003:00001730       _wcmdln                    000000018001d730     libucrt:argv_data.obj
 0003:000018f0       __acrt_heap                000000018001d8f0     libucrt:heap_handle.obj
 0003:00001900       __pioinfo                  000000018001d900     libucrt:ioinit.obj
 0003:00001d00       _nhandle                   000000018001dd00     libucrt:ioinit.obj
 0003:00001d30       __acrt_current_locale_data 000000018001dd30     libucrt:nlsdata.obj
 0003:00001d38       _nstream                   000000018001dd38     libucrt:_file.obj
 0003:00001d40       __piob                     000000018001dd40     libucrt:_file.obj
 0003:00001d48       __acrt_stdout_buffer       000000018001dd48     libucrt:_sftbuf.obj
 0003:00001d50       __acrt_stderr_buffer       000000018001dd50     libucrt:_sftbuf.obj
 0003:00001d60       __acrt_locale_changed_data 000000018001dd60     libucrt:wsetlocale.obj
 0003:00001d68       __acrt_lconv_static_null   000000018001dd68     libucrt:localeconv.obj
 0003:00001d6c       __acrt_lconv_static_W_null 000000018001dd6c     libucrt:localeconv.obj
 0003:00001d80       __fma3_is_available        000000018001dd80     libucrt:fma3_available.obj
 0003:00001d84       __use_fma3_lib             000000018001dd84     libucrt:fma3_available.obj
 0003:00001d90       ?Opt@@3UOptions@@A         000000018001dd90     FileCase.obj
 0003:000021b0       ?PsInfo@@3UPluginStartupInfo@@A 000000018001e1b0     FileCase.obj
 0003:000022d0       ?FSF@@3UFarStandardFunctions@@A 000000018001e2d0     FileCase.obj
 0003:00002470       __scrt_ucrt_dll_is_in_use  000000018001e470     <common>
 0003:00002478       __dyn_tls_init_callback    000000018001e478     <common>

 entry point at        0001:00003030

 Static symbols

 0000:fffdc000       .debug$S                   0000000180000000     FileCase.exp
 0000:fffdc000       .debug$S                   0000000180000000     kernel32:KERNEL32.dll
 0000:fffdc000       .debug$S                   0000000180000000     kernel32:KERNEL32.dll
 0000:fffdc000       .debug$S                   0000000180000000     kernel32:KERNEL32.dll
 0000:fffdc000       .debug$S                   0000000180000000     kernel32:KERNEL32.dll
 0000:fffdc000       .debug$S                   0000000180000000     kernel32:KERNEL32.dll
 0000:fffdc000       .debug$S                   0000000180000000     kernel32:KERNEL32.dll
 0000:fffdc000       .debug$S                   0000000180000000     kernel32:KERNEL32.dll
 0000:fffdc000       .debug$S                   0000000180000000     kernel32:KERNEL32.dll
 0000:fffdc000       .debug$S                   0000000180000000     kernel32:KERNEL32.dll
 0000:fffdc000       .debug$S                   0000000180000000     kernel32:KERNEL32.dll
 0000:fffdc000       .debug$S                   0000000180000000     kernel32:KERNEL32.dll
 0000:fffdc000       .debug$S                   0000000180000000     kernel32:KERNEL32.dll
 0000:fffdc000       .debug$S                   0000000180000000     kernel32:KERNEL32.dll
 0000:fffdc000       .debug$S                   0000000180000000     kernel32:KERNEL32.dll
 0000:fffdc000       .debug$S                   0000000180000000     kernel32:KERNEL32.dll
 0000:fffdc000       .debug$S                   0000000180000000     kernel32:KERNEL32.dll
 0000:fffdc000       .debug$S                   0000000180000000     kernel32:KERNEL32.dll
 0000:fffdc000       .debug$S                   0000000180000000     kernel32:KERNEL32.dll
 0000:fffdc000       .debug$S                   0000000180000000     kernel32:KERNEL32.dll
 0000:fffdc000       .debug$S                   0000000180000000     kernel32:KERNEL32.dll
 0000:fffdc000       .debug$S                   0000000180000000     kernel32:KERNEL32.dll
 0000:fffdc000       .debug$S                   0000000180000000     kernel32:KERNEL32.dll
 0000:fffdc000       .debug$S                   0000000180000000     kernel32:KERNEL32.dll
 0000:fffdc000       .debug$S                   0000000180000000     kernel32:KERNEL32.dll
 0000:fffdc000       .debug$S                   0000000180000000     kernel32:KERNEL32.dll
 0000:fffdc000       .debug$S                   0000000180000000     kernel32:KERNEL32.dll
 0000:fffdc000       .debug$S                   0000000180000000     kernel32:KERNEL32.dll
 0000:fffdc000       .debug$S                   0000000180000000     kernel32:KERNEL32.dll
 0000:fffdc000       .debug$S                   0000000180000000     kernel32:KERNEL32.dll
 0000:fffdc000       .debug$S                   0000000180000000     kernel32:KERNEL32.dll
 0000:fffdc000       .debug$S                   0000000180000000     kernel32:KERNEL32.dll
 0000:fffdc000       .debug$S                   0000000180000000     kernel32:KERNEL32.dll
 0000:fffdc000       .debug$S                   0000000180000000     kernel32:KERNEL32.dll
 0000:fffdc000       .debug$S                   0000000180000000     kernel32:KERNEL32.dll
 0000:fffdc000       .debug$S                   0000000180000000     kernel32:KERNEL32.dll
 0000:fffdc000       .debug$S                   0000000180000000     kernel32:KERNEL32.dll
 0000:fffdc000       .debug$S                   0000000180000000     kernel32:KERNEL32.dll
 0000:fffdc000       .debug$S                   0000000180000000     kernel32:KERNEL32.dll
 0000:fffdc000       .debug$S                   0000000180000000     kernel32:KERNEL32.dll
 0000:fffdc000       .debug$S                   0000000180000000     kernel32:KERNEL32.dll
 0000:fffdc000       .debug$S                   0000000180000000     kernel32:KERNEL32.dll
 0000:fffdc000       .debug$S                   0000000180000000     kernel32:KERNEL32.dll
 0000:fffdc000       .debug$S                   0000000180000000     kernel32:KERNEL32.dll
 0000:fffdc000       .debug$S                   0000000180000000     kernel32:KERNEL32.dll
 0000:fffdc000       .debug$S                   0000000180000000     kernel32:KERNEL32.dll
 0000:fffdc000       .debug$S                   0000000180000000     kernel32:KERNEL32.dll
 0000:fffdc000       .debug$S                   0000000180000000     kernel32:KERNEL32.dll
 0000:fffdc000       .debug$S                   0000000180000000     kernel32:KERNEL32.dll
 0000:fffdc000       .debug$S                   0000000180000000     kernel32:KERNEL32.dll
 0000:fffdc000       .debug$S                   0000000180000000     kernel32:KERNEL32.dll
 0000:fffdc000       .debug$S                   0000000180000000     kernel32:KERNEL32.dll
 0000:fffdc000       .debug$S                   0000000180000000     kernel32:KERNEL32.dll
 0000:fffdc000       .debug$S                   0000000180000000     kernel32:KERNEL32.dll
 0000:fffdc000       .debug$S                   0000000180000000     kernel32:KERNEL32.dll
 0000:fffdc000       .debug$S                   0000000180000000     kernel32:KERNEL32.dll
 0000:fffdc000       .debug$S                   0000000180000000     kernel32:KERNEL32.dll
 0000:fffdc000       .debug$S                   0000000180000000     kernel32:KERNEL32.dll
 0000:fffdc000       .debug$S                   0000000180000000     kernel32:KERNEL32.dll
 0000:fffdc000       .debug$S                   0000000180000000     kernel32:KERNEL32.dll
 0000:fffdc000       .debug$S                   0000000180000000     kernel32:KERNEL32.dll
 0000:fffdc000       .debug$S                   0000000180000000     kernel32:KERNEL32.dll
 0000:fffdc000       .debug$S                   0000000180000000     kernel32:KERNEL32.dll
 0000:fffdc000       .debug$S                   0000000180000000     kernel32:KERNEL32.dll
 0000:fffdc000       .debug$S                   0000000180000000     kernel32:KERNEL32.dll
 0000:fffdc000       .debug$S                   0000000180000000     kernel32:KERNEL32.dll
 0000:fffdc000       .debug$S                   0000000180000000     kernel32:KERNEL32.dll
 0000:fffdc000       .debug$S                   0000000180000000     kernel32:KERNEL32.dll
 0000:fffdc000       .debug$S                   0000000180000000     kernel32:KERNEL32.dll
 0000:fffdc000       .debug$S                   0000000180000000     kernel32:KERNEL32.dll
 0000:fffdc000       .debug$S                   0000000180000000     kernel32:KERNEL32.dll
 0000:fffdc000       .debug$S                   0000000180000000     kernel32:KERNEL32.dll
 0000:fffdc000       .debug$S                   0000000180000000     kernel32:KERNEL32.dll
 0000:fffdc000       .debug$S                   0000000180000000     kernel32:KERNEL32.dll
 0000:fffdc000       .debug$S                   0000000180000000     kernel32:KERNEL32.dll
 0000:fffdc000       .debug$S                   0000000180000000     kernel32:KERNEL32.dll
 0000:fffdc000       .debug$S                   0000000180000000     kernel32:KERNEL32.dll
 0000:fffdc000       .debug$S                   0000000180000000     kernel32:KERNEL32.dll
 0000:fffdc000       .debug$S                   0000000180000000     kernel32:KERNEL32.dll
 0000:fffdc000       .debug$S                   0000000180000000     kernel32:KERNEL32.dll
 0000:fffdc000       .debug$S                   0000000180000000     kernel32:KERNEL32.dll
 0000:fffdc000       .debug$S                   0000000180000000     kernel32:KERNEL32.dll
 0000:fffdc000       .debug$S                   0000000180000000     kernel32:KERNEL32.dll
 0000:fffdc000       .debug$S                   0000000180000000     kernel32:KERNEL32.dll
 0000:fffdc000       .debug$S                   0000000180000000     kernel32:KERNEL32.dll
 0000:fffdc000       .debug$S                   0000000180000000     kernel32:KERNEL32.dll
 0000:fffdc000       .debug$S                   0000000180000000     kernel32:KERNEL32.dll
 0000:fffdc000       .debug$S                   0000000180000000     kernel32:KERNEL32.dll
 0000:fffdc000       .debug$S                   0000000180000000     kernel32:KERNEL32.dll
 0000:fffdc000       .debug$S                   0000000180000000     kernel32:KERNEL32.dll
 0001:00000d68       $LN61                      0000000180001d68     filecvt.obj
 0001:00001070       $LN50                      0000000180002070     filecvt.obj
 0001:000013c0       $LN75                      00000001800023c0     filecvt.obj
 0001:000015fc       $LN19                      00000001800025fc     filecvt.obj
 0001:00001630       ?DlgProc@@YA_JPEAX_J10@Z   0000000180002630 f   filecvt.obj
 0001:00002608       $LN283                     0000000180003608     filecvt.obj
 0001:00002c60       $$000000                   0000000180003c60     LIBCMT:amdsecgs.obj
 0001:00002d10       ?dllmain_crt_dispatch@@YAHQEAUHINSTANCE__@@KQEAX@Z 0000000180003d10 f   LIBCMT:dll_dllmain.obj
 0001:00002d60       ?dllmain_crt_process_attach@@YAHQEAUHINSTANCE__@@QEAX@Z 0000000180003d60 f   LIBCMT:dll_dllmain.obj
 0001:00002e78       ?dllmain_crt_process_detach@@YAH_N@Z 0000000180003e78 f   LIBCMT:dll_dllmain.obj
 0001:00002efc       ?dllmain_dispatch@@YAHQEAUHINSTANCE__@@KQEAX@Z 0000000180003efc f   LIBCMT:dll_dllmain.obj
 0001:00003228       capture_current_context    0000000180004228 f   LIBCMT:gs_report.obj
 0001:00003298       capture_previous_context   0000000180004298 f   LIBCMT:gs_report.obj
 0001:000049d0       $$000000                   00000001800059d0     libvcruntime:memset.obj
 0001:00004e38       ??$BuildCatchObjectHelperInternal@V__FrameHandler4@@@@YAHPEAUEHExceptionRecord@@PEAXPEAUHandlerType4@FH4@@PEBU_s_CatchableType@@@Z 0000000180005e38 f   libvcruntime:frame.obj
 0001:0000503c       ??$BuildCatchObjectInternal@V__FrameHandler4@@@@YAXPEAUEHExceptionRecord@@PEAXPEAUHandlerType4@FH4@@PEBU_s_CatchableType@@@Z 000000018000603c f   libvcruntime:frame.obj
 0001:00005100       ??$CatchIt@V__FrameHandler4@@@@YAXPEAUEHExceptionRecord@@PEA_KPEAU_CONTEXT@@PEAU_xDISPATCHER_CONTEXT@@PEAUFuncInfo4@FH4@@PEAUHandlerType4@4@PEBU_s_CatchableType@@PEAUTryBlockMapEntry4@4@H1EE@Z 0000000180006100 f   libvcruntime:frame.obj
 0001:000051d4       ??$FindHandler@V__FrameHandler4@@@@YAXPEAUEHExceptionRecord@@PEA_KPEAU_CONTEXT@@PEAU_xDISPATCHER_CONTEXT@@PEAUFuncInfo4@FH4@@EH1@Z 00000001800061d4 f   libvcruntime:frame.obj
 0001:000056d0       ??$FindHandlerForForeignException@V__FrameHandler4@@@@YAXPEAUEHExceptionRecord@@PEA_KPEAU_CONTEXT@@PEAU_xDISPATCHER_CONTEXT@@PEAUFuncInfo4@FH4@@HH1@Z 00000001800066d0 f   libvcruntime:frame.obj
 0001:00006460       ?ExFilterRethrow@@YAHPEAU_EXCEPTION_POINTERS@@PEAUEHExceptionRecord@@PEAH@Z 0000000180007460 f   libvcruntime:frame.obj
 0001:000064e8       ?ExFilterRethrowFH4@@YAHPEAU_EXCEPTION_POINTERS@@PEAUEHExceptionRecord@@HPEAH@Z 00000001800074e8 f   libvcruntime:frame.obj
 0001:00006800       ?IsInExceptionSpec@@YAEPEAUEHExceptionRecord@@PEBU_s_ESTypeList@@@Z 0000000180007800 f   libvcruntime:frame.obj
 0001:000068f0       ?Is_bad_exception_allowed@@YAEPEBU_s_ESTypeList@@@Z 00000001800078f0 f   libvcruntime:frame.obj
 0001:00006bd0       $$000000                   0000000180007bd0     libvcruntime:notify.obj
 0001:00006cb8       ?try_get_function@@YAPEAXW4function_id@?A0x3064ecbf@@QEBDQEBW4module_id@2@2@Z 0000000180007cb8 f   libvcruntime:winapi_downlevel.obj
 0001:00006fa0       $$000000                   0000000180007fa0     libvcruntime:handlers.obj
 0001:000070b0       $$000000                   00000001800080b0     libvcruntime:memcpy.obj
 0001:00007cc8       ??$?RV<lambda_d80eeec6fff315bfe5c115232f3240e3>@@AEAV<lambda_6e4b09c48022b2350581041d5f6b0c4c>@@V<lambda_2358e3775559c9db80273638284d5e45>@@@?$__crt_seh_guarded_call@X@@QEAAX$$QEAV<lambda_d80eeec6fff315bfe5c115232f3240e3>@@AEAV<lambda_6e4b09c48022b2350581041d5f6b0c4c>@@$$QEAV<lambda_2358e3775559c9db80273638284d5e45>@@@Z 0000000180008cc8 f   libucrt:exit.obj
 0001:00007d00       ??R<lambda_6e4b09c48022b2350581041d5f6b0c4c>@@QEBA@XZ 0000000180008d00 f   libucrt:exit.obj
 0001:00007dc4       ?atexit_exception_filter@@YAHK@Z 0000000180008dc4 f   libucrt:exit.obj
 0001:00007dd0       ?common_exit@@YAXHW4_crt_exit_cleanup_mode@@W4_crt_exit_return_mode@@@Z 0000000180008dd0 f   libucrt:exit.obj
 0001:00007e8c       ?exit_or_terminate_process@@YAXI@Z 0000000180008e8c f   libucrt:exit.obj
 0001:00007ed8       ?try_cor_exit_process@@YAXI@Z 0000000180008ed8 f   libucrt:exit.obj
 0001:00007f60       ??$parse_command_line@D@@YAXPEADPEAPEAD0PEA_K2@Z 0000000180008f60 f   libucrt:argv_parsing.obj
 0001:0000830c       ??$common_initialize_environment_nolock@D@@YAHXZ 000000018000930c f   libucrt:environment_initialization.obj
 0001:00008378       ??$create_environment@D@@YAQEAPEADQEAD@Z 0000000180009378 f   libucrt:environment_initialization.obj
 0001:00008480       ??$free_environment@D@@YAXQEAPEAD@Z 0000000180009480 f   libucrt:environment_initialization.obj
 0001:00008480       ??$free_environment@_W@@YAXQEAPEA_W@Z 0000000180009480 f   libucrt:environment_initialization.obj
 0001:000084c4       ??$uninitialize_environment_internal@D@@YAXAEAPEAPEAD@Z 00000001800094c4 f   libucrt:environment_initialization.obj
 0001:000084e0       ??$uninitialize_environment_internal@_W@@YAXAEAPEAPEA_W@Z 00000001800094e0 f   libucrt:environment_initialization.obj
 0001:0000853c       ??$?RV<lambda_7777bce6b2f8c936911f934f8298dc43>@@AEAV<lambda_f03950bc5685219e0bcd2087efbe011e>@@V<lambda_3883c3dff614d5e0c5f61bb1ac94921c>@@@?$__crt_seh_guarded_call@H@@QEAAH$$QEAV<lambda_7777bce6b2f8c936911f934f8298dc43>@@AEAV<lambda_f03950bc5685219e0bcd2087efbe011e>@@$$QEAV<lambda_3883c3dff614d5e0c5f61bb1ac94921c>@@@Z 000000018000953c f   libucrt:onexit.obj
 0001:00008578       ??R<lambda_f03950bc5685219e0bcd2087efbe011e>@@QEBAHXZ 0000000180009578 f   libucrt:onexit.obj
 0001:000086f4       initialize_global_variables 00000001800096f4 f   libucrt:initialization.obj
 0001:00008708       initialize_c               0000000180009708 f   libucrt:initialization.obj
 0001:0000872c       initialize_environment     000000018000972c f   libucrt:initialization.obj
 0001:0000872c       initialize_global_state_isolation 000000018000972c f   libucrt:initialization.obj
 0001:0000872c       report_memory_leaks        000000018000972c f   libucrt:initialization.obj
 0001:0000872c       uninitialize_c             000000018000972c f   libucrt:initialization.obj
 0001:0000872c       uninitialize_global_state_isolation 000000018000972c f   libucrt:initialization.obj
 0001:00008730       uninitialize_environment   0000000180009730 f   libucrt:initialization.obj
 0001:00008740       initialize_pointers        0000000180009740 f   libucrt:initialization.obj
 0001:00008780       uninitialize_vcruntime     0000000180009780 f   libucrt:initialization.obj
 0001:00008788       uninitialize_allocated_memory 0000000180009788 f   libucrt:initialization.obj
 0001:000087c8       uninitialize_allocated_io_buffers 00000001800097c8 f   libucrt:initialization.obj
 0001:00008a20       $$000000                   0000000180009a20     libucrt:strncmp.obj
 0001:00008b1c       ??$?RV<lambda_0ae27a3a962d80f24befdcbee591983d>@@AEAV<lambda_8d0ee55de4b1038c4002e0adecdf1839>@@V<lambda_dc504788e8f1664fe9b84e20bfb512f2>@@@?$__crt_seh_guarded_call@X@@QEAAX$$QEAV<lambda_0ae27a3a962d80f24befdcbee591983d>@@AEAV<lambda_8d0ee55de4b1038c4002e0adecdf1839>@@$$QEAV<lambda_dc504788e8f1664fe9b84e20bfb512f2>@@@Z 0000000180009b1c f   libucrt:per_thread_data.obj
 0001:00008b5c       ??$?RV<lambda_2d41944a1d46af3157314b8a01080d33>@@AEAV<lambda_8f455de75cd7d7f24b4096f044d8b9e6>@@V<lambda_aa500f224e6afead328df44964fe2772>@@@?$__crt_seh_guarded_call@X@@QEAAX$$QEAV<lambda_2d41944a1d46af3157314b8a01080d33>@@AEAV<lambda_8f455de75cd7d7f24b4096f044d8b9e6>@@$$QEAV<lambda_aa500f224e6afead328df44964fe2772>@@@Z 0000000180009b5c f   libucrt:per_thread_data.obj
 0001:00008b9c       ??$?RV<lambda_aa87e3671a710a21b5dc78c0bdf72e11>@@AEAV<lambda_92619d2358a28f41a33ba319515a20b9>@@V<lambda_6992ecaafeb10aed2b74cb1fae11a551>@@@?$__crt_seh_guarded_call@X@@QEAAX$$QEAV<lambda_aa87e3671a710a21b5dc78c0bdf72e11>@@AEAV<lambda_92619d2358a28f41a33ba319515a20b9>@@$$QEAV<lambda_6992ecaafeb10aed2b74cb1fae11a551>@@@Z 0000000180009b9c f   libucrt:per_thread_data.obj
 0001:00008be4       ??$?RV<lambda_f2e299630e499de9f9a165e60fcd3db5>@@AEAV<lambda_2ae9d31cdba2644fcbeaf08da7c24588>@@V<lambda_40d01ff24d0e7b3814fdbdcee8eab3c7>@@@?$__crt_seh_guarded_call@X@@QEAAX$$QEAV<lambda_f2e299630e499de9f9a165e60fcd3db5>@@AEAV<lambda_2ae9d31cdba2644fcbeaf08da7c24588>@@$$QEAV<lambda_40d01ff24d0e7b3814fdbdcee8eab3c7>@@@Z 0000000180009be4 f   libucrt:per_thread_data.obj
 0001:00008c44       ?construct_ptd_array@@YAXQEAU__acrt_ptd@@@Z 0000000180009c44 f   libucrt:per_thread_data.obj
 0001:00008d14       ?destroy_fls@@YAXPEAX@Z    0000000180009d14 f   libucrt:per_thread_data.obj
 0001:00008d34       ?destroy_ptd_array@@YAXQEAU__acrt_ptd@@@Z 0000000180009d34 f   libucrt:per_thread_data.obj
 0001:00008e2c       ?replace_current_thread_locale_nolock@@YAXQEAU__acrt_ptd@@QEAU__crt_locale_data@@@Z 0000000180009e2c f   libucrt:per_thread_data.obj
 0001:00009424       ?<lambda_invoker_cdecl>@<lambda_a1ce4c8ae42411fd470c77163914f50e>@@CAHPEBX0@Z 000000018000a424 f   libucrt:argv_wildcards.obj
 0001:0000973c       ??$common_expand_argv_wildcards@D@@YAHQEAPEADQEAPEAPEAD@Z 000000018000a73c f   libucrt:argv_wildcards.obj
 0001:00009948       ??$copy_and_add_argument_to_buffer@D@@YAHQEBD0_KAEAV?$argument_list@D@?A0x5f5c8891@@@Z 000000018000a948 f   libucrt:argv_wildcards.obj
 0001:00009ad0       ??$expand_argument_wildcards@D@@YAHQEAD0AEAV?$argument_list@D@?A0x5f5c8891@@@Z 000000018000aad0 f   libucrt:argv_wildcards.obj
 0001:0000a01c       ??$?RV<lambda_efdfa57d1f175319df784efa44bb7b81>@@AEAV<lambda_5f0a4c1567f8adc6734073e5d1e1b35c>@@V<lambda_2e8a7d3640ea6ccb4c2413664c2db6fd>@@@?$__crt_seh_guarded_call@X@@QEAAX$$QEAV<lambda_efdfa57d1f175319df784efa44bb7b81>@@AEAV<lambda_5f0a4c1567f8adc6734073e5d1e1b35c>@@$$QEAV<lambda_2e8a7d3640ea6ccb4c2413664c2db6fd>@@@Z 000000018000b01c f   libucrt:mbctype.obj
 0001:0000a1d8       ?getSystemCP@@YAHH@Z       000000018000b1d8 f   libucrt:mbctype.obj
 0001:0000a258       ?setSBCS@@YAXPEAU__crt_multibyte_data@@@Z 000000018000b258 f   libucrt:mbctype.obj
 0001:0000a2e8       ?setSBUpLow@@YAXPEAU__crt_multibyte_data@@@Z 000000018000b2e8 f   libucrt:mbctype.obj
 0001:0000a4cc       ?setmbcp_internal@@YAHH_NQEAU__acrt_ptd@@QEAPEAU__crt_multibyte_data@@@Z 000000018000b4cc f   libucrt:mbctype.obj
 0001:0000a690       ?update_thread_multibyte_data_internal@@YAPEAU__crt_multibyte_data@@QEAU__acrt_ptd@@QEAPEAU1@@Z 000000018000b690 f   libucrt:mbctype.obj
 0001:0000aa80       ?x_ismbbtype_l@@YAHPEAU__crt_locale_pointers@@IHH@Z 000000018000ba80 f   libucrt:ismbbyte.obj
 0001:0000adc4       ?try_get_function@@YAPEAXW4function_id@?A0x391cf84c@@QEBDQEBW4module_id@2@2@Z 000000018000bdc4 f   libucrt:winapi_thunks.obj
 0001:0000b384       ?initialize_inherited_file_handles_nolock@@YAXXZ 000000018000c384 f   libucrt:ioinit.obj
 0001:0000b474       ?initialize_stdio_handles_nolock@@YAXXZ 000000018000c474 f   libucrt:ioinit.obj
 0001:0000b6b8       ??$?RV<lambda_450d765d439847d4c735a33c368b5fc0>@@AEAV<lambda_44731a7d0e6d81c3e6aa82d741081786>@@V<lambda_601a2a7da3b7a96e9554ac7215c4b07c>@@@?$__crt_seh_guarded_call@P6AXH@Z@@QEAAP6AXH@Z$$QEAV<lambda_450d765d439847d4c735a33c368b5fc0>@@AEAV<lambda_44731a7d0e6d81c3e6aa82d741081786>@@$$QEAV<lambda_601a2a7da3b7a96e9554ac7215c4b07c>@@@Z 000000018000c6b8 f   libucrt:signal.obj
 0001:0000ba14       ??$?RV<lambda_842d9ff0dc9ef11c61343bbaebe7f885>@@AEAV<lambda_c5860995281e5c4ce005b3de8f5874ee>@@V<lambda_d90129c13df834fdcbf8d2b88dafcf2d>@@@?$__crt_seh_guarded_call@X@@QEAAX$$QEAV<lambda_842d9ff0dc9ef11c61343bbaebe7f885>@@AEAV<lambda_c5860995281e5c4ce005b3de8f5874ee>@@$$QEAV<lambda_d90129c13df834fdcbf8d2b88dafcf2d>@@@Z 000000018000ca14 f   libucrt:fflush.obj
 0001:0000bab0       ??$?RV<lambda_886d6c58226a84441f68b9f2b8217b83>@@AEAV<lambda_ab61a845afdef5b7c387490eaf3616ee>@@V<lambda_f7f22ab5edc0698d5f6905b0d3f44752>@@@?$__crt_seh_guarded_call@X@@QEAAX$$QEAV<lambda_886d6c58226a84441f68b9f2b8217b83>@@AEAV<lambda_ab61a845afdef5b7c387490eaf3616ee>@@$$QEAV<lambda_f7f22ab5edc0698d5f6905b0d3f44752>@@@Z 000000018000cab0 f   libucrt:fflush.obj
 0001:0000bb90       ?common_flush_all@@YAH_N@Z 000000018000cb90 f   libucrt:fflush.obj
 0001:0000c06c       ??$?RV<lambda_410d79af7f07d98d83a3f525b3859a53>@@AEAV<lambda_3e16ef9562a7dcce91392c22ab16ea36>@@V<lambda_38119f0e861e05405d8a144b9b982f0a>@@@?$__crt_seh_guarded_call@X@@QEAAX$$QEAV<lambda_410d79af7f07d98d83a3f525b3859a53>@@AEAV<lambda_3e16ef9562a7dcce91392c22ab16ea36>@@$$QEAV<lambda_38119f0e861e05405d8a144b9b982f0a>@@@Z 000000018000d06c f   libucrt:wsetlocale.obj
 0001:0000c9e4       fallbackMethod             000000018000d9e4 f   libucrt:strpbrk.obj
 0001:0000cdb4       $LN78                      000000018000ddb4     libucrt:strpbrk.obj
 0001:0000cdf0       $LN77                      000000018000ddf0     libucrt:strpbrk.obj
 0001:0000ce30       $LN76                      000000018000de30     libucrt:strpbrk.obj
 0001:0000d09c       ?__acrt_LCMapStringA_stat@@YAHPEAU__crt_locale_pointers@@PEB_WKPEBDHPEADHHH@Z 000000018000e09c f   libucrt:lcmapstringa.obj
 0001:0000d44c       ?initialize_multibyte@@YAHXZ 000000018000e44c f   libucrt:multibyte_initializer.obj
 0001:0000d8f0       ??$?RV<lambda_a37b2b86f63e897a80ea819b0eb08c01>@@AEAV<lambda_38ce7e780aa69e748d6df282ebc68efe>@@V<lambda_99fb1378e971ab6e7edea83e3a7a83a2>@@@?$__crt_seh_guarded_call@H@@QEAAH$$QEAV<lambda_a37b2b86f63e897a80ea819b0eb08c01>@@AEAV<lambda_38ce7e780aa69e748d6df282ebc68efe>@@$$QEAV<lambda_99fb1378e971ab6e7edea83e3a7a83a2>@@@Z 000000018000e8f0 f   libucrt:commit.obj
 0001:0000da10       ?write_double_translated_ansi_nolock@@YA?AUwrite_result@?A0x17268360@@HQEBDI@Z 000000018000ea10 f   libucrt:write.obj
 0001:0000dee0       ?write_text_ansi_nolock@@YA?AUwrite_result@?A0x17268360@@HQEBDI@Z 000000018000eee0 f   libucrt:write.obj
 0001:0000dfe4       ?write_text_utf16le_nolock@@YA?AUwrite_result@?A0x17268360@@HQEBDI@Z 000000018000efe4 f   libucrt:write.obj
 0001:0000e100       ?write_text_utf8_nolock@@YA?AUwrite_result@?A0x17268360@@HQEBDI@Z 000000018000f100 f   libucrt:write.obj
 0001:0000eb04       ?free_crt_array_internal@@YAXQEAPEBX_K@Z 000000018000fb04 f   libucrt:inittime.obj
 0001:0000ecd0       ??$common_lseek_nolock@_J@@YA_JH_JH@Z 000000018000fcd0 f   libucrt:lseek.obj
 0001:0000f080       $$000000                   0000000180010080     libucrt:log10.obj
 0001:0000f75c       ??$?RV<lambda_751a882b2c74d4b022dec766aa51a29a>@@AEAV<lambda_628dfdc04ba53c8bfc02c9951375f3f5>@@V<lambda_f6c7be5f7998530c34de24c7437d6b54>@@@?$__crt_seh_guarded_call@H@@QEAAH$$QEAV<lambda_751a882b2c74d4b022dec766aa51a29a>@@AEAV<lambda_628dfdc04ba53c8bfc02c9951375f3f5>@@$$QEAV<lambda_f6c7be5f7998530c34de24c7437d6b54>@@@Z 000000018001075c f   libucrt:close.obj
 0001:0000f950       _call_matherr              0000000180010950 f   libucrt:libm_error.obj
 0001:0000f9b8       _exception_enabled         00000001800109b8 f   libucrt:libm_error.obj
 0001:0000fc30       _log_special_common        0000000180010c30 f   libucrt:log_special.obj
 0001:0000fcd0       $$000000                   0000000180010cd0     libucrt:fpsr.obj
 0001:00010350       $$000000                   0000000180011350     LIBCMT:chkstk.obj
 0001:000103b0       $$000000                   00000001800113b0     libvcruntime:memcmp.obj
 0001:00010510       $$000000                   0000000180011510     LIBCMT:guard_dispatch.obj
 0001:00010530       $$000000                   0000000180011530     LIBCMT:guard_xfg_dispatch.obj
 0001:00010550       ?dtor$0@?0??CaseConvertion@@YAXXZ@4HA 0000000180011550 f   filecvt.obj
 0001:00010560       ?dtor$1@?0??CaseConvertion@@YAXXZ@4HA 0000000180011560 f   filecvt.obj
 0001:0001056c       ?fin$0@?0??dllmain_crt_process_attach@@YAHQEAUHINSTANCE__@@QEAX@Z@4HA 000000018001156c f   LIBCMT:dll_dllmain.obj
 0001:00010583       ?fin$0@?0??dllmain_crt_process_detach@@YAH_N@Z@4HA 0000000180011583 f   LIBCMT:dll_dllmain.obj
 0001:0001059c       ?fin$1@?0??dllmain_crt_process_detach@@YAH_N@Z@4HA 000000018001159c f   LIBCMT:dll_dllmain.obj
 0001:000105b0       ?filt$0@?0??dllmain_dispatch@@YAHQEAUHINSTANCE__@@KQEAX@Z@4HA 00000001800115b0 f   LIBCMT:dll_dllmain.obj
 0001:000105e6       __scrt_is_nonwritable_in_current_image$filt$0 00000001800115e6 f   LIBCMT:utility.obj
 0001:000105fe       ?filt$0@?0???$_CallSETranslator@V__FrameHandler4@@@@YAHPEAUEHExceptionRecord@@PEA_KPEAU_CONTEXT@@PEAU_xDISPATCHER_CONTEXT@@PEAUFuncInfo4@FH4@@K1H@Z@4HA 00000001800115fe f   libvcruntime:risctrnsctrl.obj
 0001:0001069d       __DestructExceptionObject$filt$0 000000018001169d f   libvcruntime:ehhelpers.obj
 0001:00010733       ?filt$0@?0??CxxCallCatchBlock@__FrameHandler4@@SAPEAXPEAU_EXCEPTION_RECORD@@@Z@4HA 0000000180011733 f   libvcruntime:frame.obj
 0001:00010762       ?fin$1@?0??CxxCallCatchBlock@__FrameHandler4@@SAPEAXPEAU_EXCEPTION_RECORD@@@Z@4HA 0000000180011762 f   libvcruntime:frame.obj
 0001:000107e5       ?filt$0@?0??FrameUnwindToState@__FrameHandler4@@SAXPEA_KPEAU_xDISPATCHER_CONTEXT@@PEAUFuncInfo4@FH4@@H@Z@4HA 00000001800117e5 f   libvcruntime:frame.obj
 0001:000107fb       ?fin$1@?0??FrameUnwindToState@__FrameHandler4@@SAXPEA_KPEAU_xDISPATCHER_CONTEXT@@PEAUFuncInfo4@FH4@@H@Z@4HA 00000001800117fb f   libvcruntime:frame.obj
 0001:0001081e       _query_new_handler$fin$0   000000018001181e f   libucrt:new_handler.obj
 0001:00010834       ?fin$0@?0???$?RV<lambda_0ae27a3a962d80f24befdcbee591983d>@@AEAV<lambda_8d0ee55de4b1038c4002e0adecdf1839>@@V<lambda_dc504788e8f1664fe9b84e20bfb512f2>@@@?$__crt_seh_guarded_call@X@@QEAAX$$QEAV<lambda_0ae27a3a962d80f24befdcbee591983d>@@AEAV<lambda_8d0ee55de4b1038c4002e0adecdf1839>@@$$QEAV<lambda_dc504788e8f1664fe9b84e20bfb512f2>@@@Z@4HA 0000000180011834 f   libucrt:per_thread_data.obj
 0001:00010834       ?fin$0@?0???$?RV<lambda_2d41944a1d46af3157314b8a01080d33>@@AEAV<lambda_8f455de75cd7d7f24b4096f044d8b9e6>@@V<lambda_aa500f224e6afead328df44964fe2772>@@@?$__crt_seh_guarded_call@X@@QEAAX$$QEAV<lambda_2d41944a1d46af3157314b8a01080d33>@@AEAV<lambda_8f455de75cd7d7f24b4096f044d8b9e6>@@$$QEAV<lambda_aa500f224e6afead328df44964fe2772>@@@Z@4HA 0000000180011834 f   libucrt:per_thread_data.obj
 0001:00010834       ?fin$0@?0???$?RV<lambda_aa87e3671a710a21b5dc78c0bdf72e11>@@AEAV<lambda_92619d2358a28f41a33ba319515a20b9>@@V<lambda_6992ecaafeb10aed2b74cb1fae11a551>@@@?$__crt_seh_guarded_call@X@@QEAAX$$QEAV<lambda_aa87e3671a710a21b5dc78c0bdf72e11>@@AEAV<lambda_92619d2358a28f41a33ba319515a20b9>@@$$QEAV<lambda_6992ecaafeb10aed2b74cb1fae11a551>@@@Z@4HA 0000000180011834 f   libucrt:per_thread_data.obj
 0001:00010834       ?fin$0@?0???$?RV<lambda_f2e299630e499de9f9a165e60fcd3db5>@@AEAV<lambda_2ae9d31cdba2644fcbeaf08da7c24588>@@V<lambda_40d01ff24d0e7b3814fdbdcee8eab3c7>@@@?$__crt_seh_guarded_call@X@@QEAAX$$QEAV<lambda_f2e299630e499de9f9a165e60fcd3db5>@@AEAV<lambda_2ae9d31cdba2644fcbeaf08da7c24588>@@$$QEAV<lambda_40d01ff24d0e7b3814fdbdcee8eab3c7>@@@Z@4HA 0000000180011834 f   libucrt:per_thread_data.obj
 0001:00010834       ?fin$0@?0???$?RV<lambda_efdfa57d1f175319df784efa44bb7b81>@@AEAV<lambda_5f0a4c1567f8adc6734073e5d1e1b35c>@@V<lambda_2e8a7d3640ea6ccb4c2413664c2db6fd>@@@?$__crt_seh_guarded_call@X@@QEAAX$$QEAV<lambda_efdfa57d1f175319df784efa44bb7b81>@@AEAV<lambda_5f0a4c1567f8adc6734073e5d1e1b35c>@@$$QEAV<lambda_2e8a7d3640ea6ccb4c2413664c2db6fd>@@@Z@4HA 0000000180011834 f   libucrt:mbctype.obj
 0001:00010834       ?fin$0@?0???$?RV<lambda_450d765d439847d4c735a33c368b5fc0>@@AEAV<lambda_44731a7d0e6d81c3e6aa82d741081786>@@V<lambda_601a2a7da3b7a96e9554ac7215c4b07c>@@@?$__crt_seh_guarded_call@P6AXH@Z@@QEAAP6AXH@Z$$QEAV<lambda_450d765d439847d4c735a33c368b5fc0>@@AEAV<lambda_44731a7d0e6d81c3e6aa82d741081786>@@$$QEAV<lambda_601a2a7da3b7a96e9554ac7215c4b07c>@@@Z@4HA 0000000180011834 f   libucrt:signal.obj
 0001:00010834       ?fin$0@?0???$?RV<lambda_d80eeec6fff315bfe5c115232f3240e3>@@AEAV<lambda_6e4b09c48022b2350581041d5f6b0c4c>@@V<lambda_2358e3775559c9db80273638284d5e45>@@@?$__crt_seh_guarded_call@X@@QEAAX$$QEAV<lambda_d80eeec6fff315bfe5c115232f3240e3>@@AEAV<lambda_6e4b09c48022b2350581041d5f6b0c4c>@@$$QEAV<lambda_2358e3775559c9db80273638284d5e45>@@@Z@4HA 0000000180011834 f   libucrt:exit.obj
 0001:00010834       ?fin$0@?0???$?RV<lambda_7777bce6b2f8c936911f934f8298dc43>@@AEAV<lambda_f03950bc5685219e0bcd2087efbe011e>@@V<lambda_3883c3dff614d5e0c5f61bb1ac94921c>@@@?$__crt_seh_guarded_call@H@@QEAAH$$QEAV<lambda_7777bce6b2f8c936911f934f8298dc43>@@AEAV<lambda_f03950bc5685219e0bcd2087efbe011e>@@$$QEAV<lambda_3883c3dff614d5e0c5f61bb1ac94921c>@@@Z@4HA 0000000180011834 f   libucrt:onexit.obj
 0001:0001084e       ?filt$0@?0???R<lambda_6e4b09c48022b2350581041d5f6b0c4c>@@QEBA@XZ@4HA 000000018001184e f   libucrt:exit.obj
 0001:00010869       ?fin$0@?0??update_thread_multibyte_data_internal@@YAPEAU__crt_multibyte_data@@QEAU__acrt_ptd@@QEAPEAU1@@Z@4HA 0000000180011869 f   libucrt:mbctype.obj
 0001:00010882       __acrt_initialize_lowio$fin$0 0000000180011882 f   libucrt:ioinit.obj
 0001:00010882       __acrt_lowio_ensure_fh_exists$fin$0 0000000180011882 f   libucrt:osfinfo.obj
 0001:0001089b       raise$fin$0                000000018001189b f   libucrt:signal.obj
 0001:000108bc       ?fin$0@?0???$?RV<lambda_842d9ff0dc9ef11c61343bbaebe7f885>@@AEAV<lambda_c5860995281e5c4ce005b3de8f5874ee>@@V<lambda_d90129c13df834fdcbf8d2b88dafcf2d>@@@?$__crt_seh_guarded_call@X@@QEAAX$$QEAV<lambda_842d9ff0dc9ef11c61343bbaebe7f885>@@AEAV<lambda_c5860995281e5c4ce005b3de8f5874ee>@@$$QEAV<lambda_d90129c13df834fdcbf8d2b88dafcf2d>@@@Z@4HA 00000001800118bc f   libucrt:fflush.obj
 0001:000108d7       ?fin$0@?0???$?RV<lambda_886d6c58226a84441f68b9f2b8217b83>@@AEAV<lambda_ab61a845afdef5b7c387490eaf3616ee>@@V<lambda_f7f22ab5edc0698d5f6905b0d3f44752>@@@?$__crt_seh_guarded_call@X@@QEAAX$$QEAV<lambda_886d6c58226a84441f68b9f2b8217b83>@@AEAV<lambda_ab61a845afdef5b7c387490eaf3616ee>@@$$QEAV<lambda_f7f22ab5edc0698d5f6905b0d3f44752>@@@Z@4HA 00000001800118d7 f   libucrt:fflush.obj
 0001:000108f4       ?fin$0@?0???$?RV<lambda_410d79af7f07d98d83a3f525b3859a53>@@AEAV<lambda_3e16ef9562a7dcce91392c22ab16ea36>@@V<lambda_38119f0e861e05405d8a144b9b982f0a>@@@?$__crt_seh_guarded_call@X@@QEAAX$$QEAV<lambda_410d79af7f07d98d83a3f525b3859a53>@@AEAV<lambda_3e16ef9562a7dcce91392c22ab16ea36>@@$$QEAV<lambda_38119f0e861e05405d8a144b9b982f0a>@@@Z@4HA 00000001800118f4 f   libucrt:wsetlocale.obj
 0001:0001090e       __acrt_update_thread_locale_data$fin$0 000000018001190e f   libucrt:locale_refcounting.obj
 0001:00010927       ?fin$0@?0???$?RV<lambda_751a882b2c74d4b022dec766aa51a29a>@@AEAV<lambda_628dfdc04ba53c8bfc02c9951375f3f5>@@V<lambda_f6c7be5f7998530c34de24c7437d6b54>@@@?$__crt_seh_guarded_call@H@@QEAAH$$QEAV<lambda_751a882b2c74d4b022dec766aa51a29a>@@AEAV<lambda_628dfdc04ba53c8bfc02c9951375f3f5>@@$$QEAV<lambda_f6c7be5f7998530c34de24c7437d6b54>@@@Z@4HA 0000000180011927 f   libucrt:close.obj
 0001:00010927       ?fin$0@?0???$?RV<lambda_a37b2b86f63e897a80ea819b0eb08c01>@@AEAV<lambda_38ce7e780aa69e748d6df282ebc68efe>@@V<lambda_99fb1378e971ab6e7edea83e3a7a83a2>@@@?$__crt_seh_guarded_call@H@@QEAAH$$QEAV<lambda_a37b2b86f63e897a80ea819b0eb08c01>@@AEAV<lambda_38ce7e780aa69e748d6df282ebc68efe>@@$$QEAV<lambda_99fb1378e971ab6e7edea83e3a7a83a2>@@@Z@4HA 0000000180011927 f   libucrt:commit.obj
 0001:00010941       _write$fin$0               0000000180011941 f   libucrt:write.obj
 0001:00010958       _fcloseall$fin$0           0000000180011958 f   libucrt:closeall.obj
 0001:00010971       fclose$fin$0               0000000180011971 f   libucrt:fclose.obj
 0001:00010989       _ctrlfp$filt$0             0000000180011989 f   libucrt:fpctrl.obj
 0001:000109c0       _IsNonwritableInCurrentImage$filt$0 00000001800119c0 f   LIBCMT:pesect.obj
 0002:00000308       GS_ExceptionPointers       0000000180012308     LIBCMT:gs_report.obj
 0002:000003d0       ?ExceptionTemplate@?1??UnwindNestedFrames@__FrameHandler4@@SAXPEA_KPEAUEHExceptionRecord@@PEAU_CONTEXT@@0PEAXPEAUFuncInfo4@FH4@@HHPEAUHandlerType4@6@PEAU_xDISPATCHER_CONTEXT@@E@Z@4U_EXCEPTION_RECORD@@B 00000001800123d0     libvcruntime:risctrnsctrl.obj
 0002:000004a0       ?tokenTable@@3QBUStringLiteral@@B 00000001800124a0     libvcruntime:undname.obj
 0002:000005a0       ?nameTable@@3QBUStringLiteral@@B 00000001800125a0     libvcruntime:undname.obj
 0002:00000ad0       ?rttiTable@@3QBUStringLiteral@@B 0000000180012ad0     libvcruntime:undname.obj
 0002:00000b20       ?IndirectionName@@3QBUStringLiteral@@B 0000000180012b20     libvcruntime:undname.obj
 0002:00000b80       ?PrefixName@@3QBUStringLiteral@@B 0000000180012b80     libvcruntime:undname.obj
 0002:00001258       ?module_names@?A0x3064ecbf@@3QBQEB_WB 0000000180013258     libvcruntime:winapi_downlevel.obj
 0002:00001318       ?candidate_modules@?1??try_get_FlsAlloc@@YAP6AKP6AXPEAX@Z@ZXZ@4QBW4module_id@?A0x3064ecbf@@B 0000000180013318     libvcruntime:winapi_downlevel.obj
 0002:00001330       ?candidate_modules@?1??try_get_FlsFree@@YAP6AHK@ZXZ@4QBW4module_id@?A0x3064ecbf@@B 0000000180013330     libvcruntime:winapi_downlevel.obj
 0002:00001340       ?candidate_modules@?1??try_get_FlsGetValue@@YAP6APEAXK@ZXZ@4QBW4module_id@?A0x3064ecbf@@B 0000000180013340     libvcruntime:winapi_downlevel.obj
 0002:00001358       ?candidate_modules@?1??try_get_FlsSetValue@@YAP6AHKPEAX@ZXZ@4QBW4module_id@?A0x3064ecbf@@B 0000000180013358     libvcruntime:winapi_downlevel.obj
 0002:00001370       ?candidate_modules@?1??try_get_InitializeCriticalSectionEx@@YAP6AHPEAU_RTL_CRITICAL_SECTION@@KK@ZXZ@4QBW4module_id@?A0x3064ecbf@@B 0000000180013370     libvcruntime:winapi_downlevel.obj
 0002:000014a0       __acrt_initializers        00000001800134a0     libucrt:initialization.obj
 0002:000015a0       ?errtable@@3QBUerrentry@?A0x31fdb9ec@@B 00000001800135a0     libucrt:errno.obj
 0002:00001708       ?_mb_locale_names@@3QBQEB_WB 0000000180013708     libucrt:mbctype.obj
 0002:00001770       ?module_names@?A0x391cf84c@@3QBQEB_WB 0000000180013770     libucrt:winapi_thunks.obj
 0002:00001c78       ?candidate_modules@?1??try_get_AreFileApisANSI@@YAP6AHXZXZ@4QBW4module_id@?A0x391cf84c@@B 0000000180013c78     libucrt:winapi_thunks.obj
 0002:00001c90       ?candidate_modules@?1??try_get_FlsAlloc@@YAP6AKP6AXPEAX@Z@ZXZ@4QBW4module_id@?A0x391cf84c@@B 0000000180013c90     libucrt:winapi_thunks.obj
 0002:00001c98       ?candidate_modules@?1??try_get_FlsFree@@YAP6AHK@ZXZ@4QBW4module_id@?A0x391cf84c@@B 0000000180013c98     libucrt:winapi_thunks.obj
 0002:00001ca0       ?candidate_modules@?1??try_get_FlsGetValue@@YAP6APEAXK@ZXZ@4QBW4module_id@?A0x391cf84c@@B 0000000180013ca0     libucrt:winapi_thunks.obj
 0002:00001ca8       ?candidate_modules@?1??try_get_FlsSetValue@@YAP6AHKPEAX@ZXZ@4QBW4module_id@?A0x391cf84c@@B 0000000180013ca8     libucrt:winapi_thunks.obj
 0002:00001cb0       ?candidate_modules@?1??try_get_InitializeCriticalSectionEx@@YAP6AHPEAU_RTL_CRITICAL_SECTION@@KK@ZXZ@4QBW4module_id@?A0x391cf84c@@B 0000000180013cb0     libucrt:winapi_thunks.obj
 0002:00001cb8       ?candidate_modules@?1??try_get_LCMapStringEx@@YAP6AHPEB_WK0HPEA_WHPEAU_nlsversioninfo@@PEAX_J@ZXZ@4QBW4module_id@?A0x391cf84c@@B 0000000180013cb8     libucrt:winapi_thunks.obj
 0002:00001cd0       ?candidate_modules@?1??try_get_LocaleNameToLCID@@YAP6AKPEB_WK@ZXZ@4QBW4module_id@?A0x391cf84c@@B 0000000180013cd0     libucrt:winapi_thunks.obj
 0002:00001cec       ?candidate_modules@?1??try_get_AppPolicyGetProcessTerminationMethod@@YAP6AJPEAXPEAW4AppPolicyProcessTerminationMethod@@@ZXZ@4QBW4module_id@?A0x391cf84c@@B 0000000180013cec     libucrt:winapi_thunks.obj
 0002:000029a0       ?LcidToLocaleNameTable@?A0x881e4c05@@3QBULcidToLocaleName@1@B 00000001800149a0     libucrt:lcidtoname_downlevel.obj
 0002:00004400       ?LocaleNameToIndexTable@?A0x881e4c05@@3QBULocaleNameIndex@1@B 0000000180016400     libucrt:lcidtoname_downlevel.obj
 0002:00005ca0       __real_ninf                0000000180017ca0     libucrt:log10.obj
 0002:00005cb0       __real_inf                 0000000180017cb0     libucrt:log10.obj
 0002:00005cc0       __real_neg_qnan            0000000180017cc0     libucrt:log10.obj
 0002:00005cd0       __real_qnanbit             0000000180017cd0     libucrt:log10.obj
 0002:00005ce0       __int_1023                 0000000180017ce0     libucrt:log10.obj
 0002:00005cf0       __mask_001                 0000000180017cf0     libucrt:log10.obj
 0002:00005d00       __mask_mant                0000000180017d00     libucrt:log10.obj
 0002:00005d10       __mask_mant_top8           0000000180017d10     libucrt:log10.obj
 0002:00005d20       __mask_mant9               0000000180017d20     libucrt:log10.obj
 0002:00005d30       __real_log10_e             0000000180017d30     libucrt:log10.obj
 0002:00005d40       __real_log10_e_lead        0000000180017d40     libucrt:log10.obj
 0002:00005d50       __real_log10_e_tail        0000000180017d50     libucrt:log10.obj
 0002:00005d60       __real_log10_2_lead        0000000180017d60     libucrt:log10.obj
 0002:00005d70       __real_log10_2_tail        0000000180017d70     libucrt:log10.obj
 0002:00005d80       __real_two                 0000000180017d80     libucrt:log10.obj
 0002:00005d90       __real_one                 0000000180017d90     libucrt:log10.obj
 0002:00005da0       __real_half                0000000180017da0     libucrt:log10.obj
 0002:00005db0       __mask_100                 0000000180017db0     libucrt:log10.obj
 0002:00005dc0       __real_1_over_512          0000000180017dc0     libucrt:log10.obj
 0002:00005dd0       __real_1_over_2            0000000180017dd0     libucrt:log10.obj
 0002:00005de0       __real_1_over_3            0000000180017de0     libucrt:log10.obj
 0002:00005df0       __real_1_over_4            0000000180017df0     libucrt:log10.obj
 0002:00005e00       __real_1_over_5            0000000180017e00     libucrt:log10.obj
 0002:00005e10       __real_1_over_6            0000000180017e10     libucrt:log10.obj
 0002:00005e20       __real_neg_1023            0000000180017e20     libucrt:log10.obj
 0002:00005e30       __mask_2045                0000000180017e30     libucrt:log10.obj
 0002:00005e40       __real_threshold           0000000180017e40     libucrt:log10.obj
 0002:00005e50       __real_near_one_lt         0000000180017e50     libucrt:log10.obj
 0002:00005e60       __real_near_one_gt         0000000180017e60     libucrt:log10.obj
 0002:00005e70       __real_min_norm            0000000180017e70     libucrt:log10.obj
 0002:00005e80       __real_notsign             0000000180017e80     libucrt:log10.obj
 0002:00005e90       __real_ca1                 0000000180017e90     libucrt:log10.obj
 0002:00005ea0       __real_ca2                 0000000180017ea0     libucrt:log10.obj
 0002:00005eb0       __real_ca3                 0000000180017eb0     libucrt:log10.obj
 0002:00005ec0       __real_ca4                 0000000180017ec0     libucrt:log10.obj
 0002:00005ed0       __mask_lower               0000000180017ed0     libucrt:log10.obj
 0002:00005ee0       __flag_x_zero              0000000180017ee0     libucrt:log10.obj
 0002:00005ee4       __flag_x_neg               0000000180017ee4     libucrt:log10.obj
 0002:00005ee8       __flag_x_nan               0000000180017ee8     libucrt:log10.obj
 0002:00007740       __real@433fffffffffffff    0000000180019740     libucrt:fpsr.obj
 0002:00007748       __real@c33fffffffffffff    0000000180019748     libucrt:fpsr.obj
 0002:00008468       $unwind$??1PluginSettings@@QEAA@XZ 000000018001a468     FileCase.obj
 0002:00008478       $cppxdata$??1PluginSettings@@QEAA@XZ 000000018001a478     FileCase.obj
 0002:0000847d       $ip2state$??1PluginSettings@@QEAA@XZ 000000018001a47d     FileCase.obj
 0002:00008480       $unwind$GetGlobalInfoW     000000018001a480     FileCase.obj
 0002:00008480       $unwind$OpenW              000000018001a480     FileCase.obj
 0002:00008480       $unwind$?DlgProc@@YA_JPEAX_J10@Z 000000018001a480     filecvt.obj
 0002:00008480       $unwind$?ItemWidth@PluginDialogBuilder@@CA_JAEBUFarDialogItem@@@Z 000000018001a480     filecvt.obj
 0002:00008480       $unwind$?_Xlen_string@std@@YAXXZ 000000018001a480     filecvt.obj
 0002:00008480       $unwind$__scrt_initialize_default_local_stdio_options 000000018001a480     LIBCMT:default_local_stdio_options.obj
 0002:00008480       $unwind$?dllmain_crt_dispatch@@YAHQEAUHINSTANCE__@@KQEAX@Z 000000018001a480     LIBCMT:dll_dllmain.obj
 0002:00008480       $unwind$__report_rangecheckfailure 000000018001a480     LIBCMT:gs_report.obj
 0002:00008480       $unwind$__GSHandlerCheck   000000018001a480     LIBCMT:gshandler.obj
 0002:00008480       $unwind$__scrt_acquire_startup_lock 000000018001a480     LIBCMT:utility.obj
 0002:00008480       $unwind$__scrt_dllmain_after_initialize_c 000000018001a480     LIBCMT:utility.obj
 0002:00008480       $unwind$__scrt_dllmain_before_initialize_c 000000018001a480     LIBCMT:utility.obj
 0002:00008480       $unwind$__scrt_dllmain_crt_thread_attach 000000018001a480     LIBCMT:utility.obj
 0002:00008480       $unwind$__scrt_dllmain_crt_thread_detach 000000018001a480     LIBCMT:utility.obj
 0002:00008480       $unwind$__scrt_dllmain_uninitialize_c 000000018001a480     LIBCMT:utility.obj
 0002:00008480       $unwind$__scrt_dllmain_uninitialize_critical 000000018001a480     LIBCMT:utility.obj
 0002:00008480       $unwind$__std_terminate    000000018001a480     libvcruntime:ehhelpers.obj
 0002:00008480       $unwind$__vcrt_initialize  000000018001a480     libvcruntime:initialization.obj
 0002:00008480       $unwind$__vcrt_thread_attach 000000018001a480     libvcruntime:initialization.obj
 0002:00008480       $unwind$__vcrt_thread_detach 000000018001a480     libvcruntime:initialization.obj
 0002:00008480       $unwind$__vcrt_uninitialize 000000018001a480     libvcruntime:initialization.obj
 0002:00008480       $unwind$__vcrt_uninitialize_critical 000000018001a480     libvcruntime:initialization.obj
 0002:00008480       $unwind$__vcrt_initialize_locks 000000018001a480     libvcruntime:locks.obj
 0002:00008480       $unwind$__vcrt_freefls     000000018001a480     libvcruntime:per_thread_data.obj
 0002:00008480       $unwind$__vcrt_getptd      000000018001a480     libvcruntime:per_thread_data.obj
 0002:00008480       $unwind$__vcrt_initialize_ptd 000000018001a480     libvcruntime:per_thread_data.obj
 0002:00008480       $unwind$__vcrt_uninitialize_ptd 000000018001a480     libvcruntime:per_thread_data.obj
 0002:00008480       $unwind$?FrameUnwindToEmptyState@__FrameHandler4@@SAXPEA_KPEAU_xDISPATCHER_CONTEXT@@PEAUFuncInfo4@FH4@@@Z 000000018001a480     libvcruntime:risctrnsctrl.obj
 0002:00008480       $unwind$_GetImageBase      000000018001a480     libvcruntime:risctrnsctrl.obj
 0002:00008480       $unwind$_GetThrowImageBase 000000018001a480     libvcruntime:risctrnsctrl.obj
 0002:00008480       $unwind$__dcrt_terminate_console_output 000000018001a480     libucrt:initcon.obj
 0002:00008480       $unwind$??$uninitialize_environment_internal@D@@YAXAEAPEAPEAD@Z 000000018001a480     libucrt:environment_initialization.obj
 0002:00008480       $unwind$??$uninitialize_environment_internal@_W@@YAXAEAPEAPEA_W@Z 000000018001a480     libucrt:environment_initialization.obj
 0002:00008480       $unwind$__dcrt_uninitialize_environments_nolock 000000018001a480     libucrt:environment_initialization.obj
 0002:00008480       $unwind$__acrt_initialize_heap 000000018001a480     libucrt:heap_handle.obj
 0002:00008480       $unwind$_msize_base        000000018001a480     libucrt:msize.obj
 0002:00008480       $unwind$?initialize_multibyte@@YAHXZ 000000018001a480     libucrt:multibyte_initializer.obj
 0002:00008480       $unwind$__acrt_thread_attach 000000018001a480     libucrt:initialization.obj
 0002:00008480       $unwind$__acrt_thread_detach 000000018001a480     libucrt:initialization.obj
 0002:00008480       $unwind$__acrt_uninitialize 000000018001a480     libucrt:initialization.obj
 0002:00008480       $unwind$__acrt_uninitialize_critical 000000018001a480     libucrt:initialization.obj
 0002:00008480       $unwind$initialize_c       000000018001a480     libucrt:initialization.obj
 0002:00008480       $unwind$uninitialize_allocated_io_buffers 000000018001a480     libucrt:initialization.obj
 0002:00008480       $unwind$uninitialize_environment 000000018001a480     libucrt:initialization.obj
 0002:00008480       $unwind$__acrt_initialize_ptd 000000018001a480     libucrt:per_thread_data.obj
 0002:00008480       $unwind$__acrt_uninitialize_ptd 000000018001a480     libucrt:per_thread_data.obj
 0002:00008480       $unwind$__acrt_AreFileApisANSI 000000018001a480     libucrt:winapi_thunks.obj
 0002:00008480       $unwind$__pctype_func      000000018001a480     libucrt:ctype.obj
 0002:00008480       $unwind$__acrt_release_locale_ref 000000018001a480     libucrt:locale_refcounting.obj
 0002:00008480       $unwind$_isatty            000000018001a480     libucrt:isatty.obj
 0002:00008480       $unwind$_get_osfhandle     000000018001a480     libucrt:osfinfo.obj
 0002:00008480       $unwind$__acrt_initialize_multibyte 000000018001a480     libucrt:mbctype.obj
 0002:00008480       $unwind$__acrt_update_thread_multibyte_data 000000018001a480     libucrt:mbctype.obj
 0002:00008480       $unwind$__doserrno         000000018001a480     libucrt:errno.obj
 0002:00008480       $unwind$_errno             000000018001a480     libucrt:errno.obj
 0002:00008480       $unwind$_invoke_watson     000000018001a480     libucrt:invalid_parameter.obj
 0002:00008480       $unwind$abort              000000018001a480     libucrt:abort.obj
 0002:00008480       $unwind$__acrt_initialize_command_line 000000018001a480     libucrt:argv_data.obj
 0002:00008480       $unwind$_fileno            000000018001a480     libucrt:fileno.obj
 0002:00008480       $unwind$_statfp            000000018001a480     libucrt:fpctrl.obj
 0002:00008480       $unwind$_set_errno_from_matherr 000000018001a480     libucrt:fpexcept.obj
 0002:00008488       $unwind$SetStartupInfoW    000000018001a488     FileCase.obj
 0002:000084a8       $cppxdata$SetStartupInfoW  000000018001a4a8     FileCase.obj
 0002:000084b1       $stateUnwindMap$SetStartupInfoW 000000018001a4b1     FileCase.obj
 0002:000084b7       $ip2state$SetStartupInfoW  000000018001a4b7     FileCase.obj
 0002:000084c0       $unwind$GetPluginInfoW     000000018001a4c0     FileCase.obj
 0002:000084c0       $unwind$??0bad_alloc@std@@QEAA@AEBV01@@Z 000000018001a4c0     filecvt.obj
 0002:000084c0       $unwind$??0bad_array_new_length@std@@QEAA@AEBV01@@Z 000000018001a4c0     filecvt.obj
 0002:000084c0       $unwind$??0exception@std@@QEAA@AEBV01@@Z 000000018001a4c0     filecvt.obj
 0002:000084c0       $unwind$??_GPluginCheckBoxBinding@@UEAAPEAXI@Z 000000018001a4c0     filecvt.obj
 0002:000084c0       $unwind$??_GPluginEditFieldBinding@@UEAAPEAXI@Z 000000018001a4c0     filecvt.obj
 0002:000084c0       $unwind$??_GPluginRadioButtonBinding@@UEAAPEAXI@Z 000000018001a4c0     filecvt.obj
 0002:000084c0       $unwind$?SaveValue@PluginCheckBoxBinding@@UEAAXPEBUFarDialogItem@@H@Z 000000018001a4c0     filecvt.obj
 0002:000084c0       $unwind$?SaveValue@PluginEditFieldBinding@@UEAAXPEBUFarDialogItem@@H@Z 000000018001a4c0     filecvt.obj
 0002:000084c0       $unwind$__raise_securityfailure 000000018001a4c0     LIBCMT:gs_report.obj
 0002:000084c0       $unwind$??2@YAPEAX_K@Z     000000018001a4c0     LIBCMT:new_scalar.obj
 0002:000084c0       $unwind$??_Gtype_info@@UEAAPEAXI@Z 000000018001a4c0     LIBCMT:std_type_info_static.obj
 0002:000084c0       $unwind$__scrt_initialize_crt 000000018001a4c0     LIBCMT:utility.obj
 0002:000084c0       $unwind$__scrt_initialize_onexit_tables 000000018001a4c0     LIBCMT:utility.obj
 0002:000084c0       $unwind$__scrt_release_startup_lock 000000018001a4c0     LIBCMT:utility.obj
 0002:000084c0       $unwind$__scrt_uninitialize_crt 000000018001a4c0     LIBCMT:utility.obj
 0002:000084c0       $unwind$??0length_error@std@@QEAA@AEBV01@@Z 000000018001a4c0     libcpmt:xthrow.obj
 0002:000084c0       $unwind$??0logic_error@std@@QEAA@AEBV01@@Z 000000018001a4c0     libcpmt:xthrow.obj
 0002:000084c0       $unwind$_IsExceptionObjectToBeDestroyed 000000018001a4c0     libvcruntime:ehhelpers.obj
 0002:000084c0       $unwind$??0HandlerMap4@FH4@@QEAA@PEBUTryBlockMapEntry4@1@_KH@Z 000000018001a4c0     libvcruntime:frame.obj
 0002:000084c0       $unwind$??0bad_exception@std@@QEAA@AEBV01@@Z 000000018001a4c0     libvcruntime:frame.obj
 0002:000084c0       $unwind$?ExFilterRethrow@@YAHPEAU_EXCEPTION_POINTERS@@PEAUEHExceptionRecord@@PEAH@Z 000000018001a4c0     libvcruntime:frame.obj
 0002:000084c0       $unwind$__vcrt_uninitialize_locks 000000018001a4c0     libvcruntime:locks.obj
 0002:000084c0       $unwind$__vcrt_freeptd     000000018001a4c0     libvcruntime:per_thread_data.obj
 0002:000084c0       $unwind$_CreateFrameInfo   000000018001a4c0     libvcruntime:risctrnsctrl.obj
 0002:000084c0       $unwind$_SetImageBase      000000018001a4c0     libvcruntime:risctrnsctrl.obj
 0002:000084c0       $unwind$_SetThrowImageBase 000000018001a4c0     libvcruntime:risctrnsctrl.obj
 0002:000084c0       $unwind$__std_exception_destroy 000000018001a4c0     libvcruntime:std_exception.obj
 0002:000084c0       $unwind$__std_type_info_destroy_list 000000018001a4c0     libvcruntime:std_type_info.obj
 0002:000084c0       $unwind$__vcrt_FlsAlloc    000000018001a4c0     libvcruntime:winapi_downlevel.obj
 0002:000084c0       $unwind$__vcrt_FlsFree     000000018001a4c0     libvcruntime:winapi_downlevel.obj
 0002:000084c0       $unwind$__vcrt_FlsGetValue 000000018001a4c0     libvcruntime:winapi_downlevel.obj
 0002:000084c0       $unwind$_calloc_base       000000018001a4c0     libucrt:calloc_base.obj
 0002:000084c0       $unwind$_malloc_base       000000018001a4c0     libucrt:malloc_base.obj
 0002:000084c0       $unwind$_callnewh          000000018001a4c0     libucrt:new_handler.obj
 0002:000084c0       $unwind$initialize_pointers 000000018001a4c0     libucrt:initialization.obj
 0002:000084c0       $unwind$uninitialize_allocated_memory 000000018001a4c0     libucrt:initialization.obj
 0002:000084c0       $unwind$__acrt_initialize_locks 000000018001a4c0     libucrt:locks.obj
 0002:000084c0       $unwind$__acrt_uninitialize_locks 000000018001a4c0     libucrt:locks.obj
 0002:000084c0       $unwind$__acrt_freeptd     000000018001a4c0     libucrt:per_thread_data.obj
 0002:000084c0       $unwind$__acrt_getptd_head 000000018001a4c0     libucrt:per_thread_data.obj
 0002:000084c0       $unwind$__acrt_get_process_end_policy 000000018001a4c0     libucrt:win_policies.obj
 0002:000084c0       $unwind$__acrt_AppPolicyGetProcessTerminationMethodInternal 000000018001a4c0     libucrt:winapi_thunks.obj
 0002:000084c0       $unwind$__acrt_FlsAlloc    000000018001a4c0     libucrt:winapi_thunks.obj
 0002:000084c0       $unwind$__acrt_FlsFree     000000018001a4c0     libucrt:winapi_thunks.obj
 0002:000084c0       $unwind$__acrt_FlsGetValue 000000018001a4c0     libucrt:winapi_thunks.obj
 0002:000084c0       $unwind$__acrt_uninitialize_winapi_thunks 000000018001a4c0     libucrt:winapi_thunks.obj
 0002:000084c0       $unwind$__acrt_update_locale_info 000000018001a4c0     libucrt:locale_update.obj
 0002:000084c0       $unwind$__acrt_update_multibyte_info 000000018001a4c0     libucrt:locale_update.obj
 0002:000084c0       $unwind$__acrt_allocate_buffer_for_argv 000000018001a4c0     libucrt:argv_parsing.obj
 0002:000084c0       $unwind$?exit_or_terminate_process@@YAXI@Z 000000018001a4c0     libucrt:exit.obj
 0002:000084c0       $unwind$?try_cor_exit_process@@YAXI@Z 000000018001a4c0     libucrt:exit.obj
 0002:000084c0       $unwind$__acrt_uninitialize_stdio 000000018001a4c0     libucrt:_file.obj
 0002:000084c0       $unwind$__acrt_stdio_free_buffer_nolock 000000018001a4c0     libucrt:_freebuf.obj
 0002:000084c0       $unwind$_fflush_nolock     000000018001a4c0     libucrt:fflush.obj
 0002:000084c0       $unwind$strcpy_s           000000018001a4c0     libucrt:strcpy_s.obj
 0002:000084c0       $unwind$_clrfp             000000018001a4c0     libucrt:fpctrl.obj
 0002:000084c0       $unwind$_set_statfp        000000018001a4c0     libucrt:fpctrl.obj
 0002:000084c8       $unwind$?IsCaseMixed@@YAHPEB_W@Z 000000018001a4c8     FileMix.obj
 0002:000084c8       $unwind$??_Gbad_alloc@std@@UEAAPEAXI@Z 000000018001a4c8     filecvt.obj
 0002:000084c8       $unwind$??_Gbad_array_new_length@std@@UEAAPEAXI@Z 000000018001a4c8     filecvt.obj
 0002:000084c8       $unwind$??_Gexception@std@@UEAAPEAXI@Z 000000018001a4c8     filecvt.obj
 0002:000084c8       $unwind$?SaveValue@PluginRadioButtonBinding@@UEAAXPEBUFarDialogItem@@H@Z 000000018001a4c8     filecvt.obj
 0002:000084c8       $unwind$_RTC_Initialize    000000018001a4c8     LIBCMT:initsect.obj
 0002:000084c8       $unwind$_RTC_Terminate     000000018001a4c8     LIBCMT:initsect.obj
 0002:000084c8       $unwind$??_Glength_error@std@@UEAAPEAXI@Z 000000018001a4c8     libcpmt:xthrow.obj
 0002:000084c8       $unwind$??_Glogic_error@std@@UEAAPEAXI@Z 000000018001a4c8     libcpmt:xthrow.obj
 0002:000084c8       $unwind$__FrameUnwindFilter 000000018001a4c8     libvcruntime:ehhelpers.obj
 0002:000084c8       $unwind$??_Gbad_exception@std@@UEAAPEAXI@Z 000000018001a4c8     libvcruntime:frame.obj
 0002:000084c8       $unwind$?ExFilterRethrowFH4@@YAHPEAU_EXCEPTION_POINTERS@@PEAUEHExceptionRecord@@HPEAH@Z 000000018001a4c8     libvcruntime:frame.obj
 0002:000084c8       $unwind$_FindAndUnlinkFrame 000000018001a4c8     libvcruntime:risctrnsctrl.obj
 0002:000084c8       $unwind$__vcrt_FlsSetValue 000000018001a4c8     libvcruntime:winapi_downlevel.obj
 0002:000084c8       $unwind$??$common_initialize_environment_nolock@D@@YAHXZ 000000018001a4c8     libucrt:environment_initialization.obj
 0002:000084c8       $unwind$_realloc_base      000000018001a4c8     libucrt:realloc_base.obj
 0002:000084c8       $unwind$?replace_current_thread_locale_nolock@@YAXQEAU__acrt_ptd@@QEAU__crt_locale_data@@@Z 000000018001a4c8     libucrt:per_thread_data.obj
 0002:000084c8       $unwind$__acrt_execute_uninitializers 000000018001a4c8     libucrt:shared_initialization.obj
 0002:000084c8       $unwind$__acrt_FlsSetValue 000000018001a4c8     libucrt:winapi_thunks.obj
 0002:000084c8       $unwind$__acrt_LocaleNameToLCID 000000018001a4c8     libucrt:winapi_thunks.obj
 0002:000084c8       $unwind$_updatetlocinfoEx_nolock 000000018001a4c8     libucrt:locale_refcounting.obj
 0002:000084c8       $unwind$_close_nolock      000000018001a4c8     libucrt:close.obj
 0002:000084c8       $unwind$__acrt_uninitialize_lowio 000000018001a4c8     libucrt:ioinit.obj
 0002:000084c8       $unwind$__acrt_errno_map_os_error 000000018001a4c8     libucrt:errno.obj
 0002:000084c8       $unwind$_initterm_e        000000018001a4c8     libucrt:initterm.obj
 0002:000084c8       $unwind$_fclose_nolock     000000018001a4c8     libucrt:fclose.obj
 0002:000084c8       $unwind$strncpy_s          000000018001a4c8     libucrt:strncpy_s.obj
 0002:000084d4       $unwind$?_Throw_bad_array_new_length@std@@YAXXZ 000000018001a4d4     filecvt.obj
 0002:000084d4       $unwind$?__scrt_throw_std_bad_alloc@@YAXXZ 000000018001a4d4     LIBCMT:throw_bad_alloc.obj
 0002:000084d4       $unwind$?__scrt_throw_std_bad_array_new_length@@YAXXZ 000000018001a4d4     LIBCMT:throw_bad_alloc.obj
 0002:000084d4       $unwind$?_Xlength_error@std@@YAXPEBD@Z 000000018001a4d4     libcpmt:xthrow.obj
 0002:000084d4       $unwind$_raise_exc         000000018001a4d4     libucrt:fpexcept.obj
 0002:000084dc       $unwind$??0PluginDialogBuilder@@QEAA@AEBUPluginStartupInfo@@AEBU_GUID@@1HPEB_WP6A_JPEAX_J43@Z3_K@Z 000000018001a4dc     filecvt.obj
 0002:000084f0       $chain$0$??0PluginDialogBuilder@@QEAA@AEBUPluginStartupInfo@@AEBU_GUID@@1HPEB_WP6A_JPEAX_J43@Z3_K@Z 000000018001a4f0     filecvt.obj
 0002:00008504       $chain$1$??0PluginDialogBuilder@@QEAA@AEBUPluginStartupInfo@@AEBU_GUID@@1HPEB_WP6A_JPEAX_J43@Z3_K@Z 000000018001a504     filecvt.obj
 0002:00008514       $unwind$??1PluginDialogBuilder@@QEAA@XZ 000000018001a514     filecvt.obj
 0002:0000852c       $cppxdata$??1PluginDialogBuilder@@QEAA@XZ 000000018001a52c     filecvt.obj
 0002:00008531       $ip2state$??1PluginDialogBuilder@@QEAA@XZ 000000018001a531     filecvt.obj
 0002:00008534       $unwind$?AddRadioButtons@PluginDialogBuilder@@QEAAPEAUFarDialogItem@@PEAHHQEBH_N@Z 000000018001a534     filecvt.obj
 0002:00008550       $unwind$?AddButtons@PluginDialogBuilder@@QEAAXHPEBHHH@Z 000000018001a550     filecvt.obj
 0002:00008560       $chain$3$?AddButtons@PluginDialogBuilder@@QEAAXHPEBHHH@Z 000000018001a560     filecvt.obj
 0002:00008580       $chain$4$?AddButtons@PluginDialogBuilder@@QEAAXHPEBHHH@Z 000000018001a580     filecvt.obj
 0002:00008590       $unwind$?ShowDialogEx@PluginDialogBuilder@@QEAA_JXZ 000000018001a590     filecvt.obj
 0002:0000859c       $chain$4$?ShowDialogEx@PluginDialogBuilder@@QEAA_JXZ 000000018001a59c     filecvt.obj
 0002:000085c0       $chain$6$?ShowDialogEx@PluginDialogBuilder@@QEAA_JXZ 000000018001a5c0     filecvt.obj
 0002:000085d8       $chain$7$?ShowDialogEx@PluginDialogBuilder@@QEAA_JXZ 000000018001a5d8     filecvt.obj
 0002:000085ec       $chain$8$?ShowDialogEx@PluginDialogBuilder@@QEAA_JXZ 000000018001a5ec     filecvt.obj
 0002:000085fc       $unwind$?AddDialogItem@PluginDialogBuilder@@AEAAPEAUFarDialogItem@@W4FARDIALOGITEMTYPES@@PEB_W@Z 000000018001a5fc     filecvt.obj
 0002:0000860c       $chain$0$?AddDialogItem@PluginDialogBuilder@@AEAAPEAUFarDialogItem@@W4FARDIALOGITEMTYPES@@PEB_W@Z 000000018001a60c     filecvt.obj
 0002:00008620       $chain$1$?AddDialogItem@PluginDialogBuilder@@AEAAPEAUFarDialogItem@@W4FARDIALOGITEMTYPES@@PEB_W@Z 000000018001a620     filecvt.obj
 0002:00008634       $chain$2$?AddDialogItem@PluginDialogBuilder@@AEAAPEAUFarDialogItem@@W4FARDIALOGITEMTYPES@@PEB_W@Z 000000018001a634     filecvt.obj
 0002:00008644       $chain$3$?AddDialogItem@PluginDialogBuilder@@AEAAPEAUFarDialogItem@@W4FARDIALOGITEMTYPES@@PEB_W@Z 000000018001a644     filecvt.obj
 0002:00008654       $unwind$?CaseConvertion@@YAXXZ 000000018001a654     filecvt.obj
 0002:00008680       $cppxdata$?CaseConvertion@@YAXXZ 000000018001a680     filecvt.obj
 0002:00008689       $stateUnwindMap$?CaseConvertion@@YAXXZ 000000018001a689     filecvt.obj
 0002:000086a2       $ip2state$?CaseConvertion@@YAXXZ 000000018001a6a2     filecvt.obj
 0002:000086b8       $unwind$?assign@?$basic_string@_WU?$char_traits@_W@std@@V?$allocator@_W@2@@std@@QEAAAEAV12@QEB_W_K@Z 000000018001a6b8     filecvt.obj
 0002:000086d4       $unwind$?CaseWord@@YAXPEA_WH@Z 000000018001a6d4     FileMix.obj
 0002:000086dc       $chain$3$?CaseWord@@YAXPEA_WH@Z 000000018001a6dc     FileMix.obj
 0002:000086fc       $chain$4$?CaseWord@@YAXPEA_WH@Z 000000018001a6fc     FileMix.obj
 0002:0000870c       $unwind$?ProcessName@@YAXPEB_WK@Z 000000018001a70c     ProcessName.obj
 0002:00008720       $chain$0$?ProcessName@@YAXPEB_WK@Z 000000018001a720     ProcessName.obj
 0002:00008734       $chain$1$?ProcessName@@YAXPEB_WK@Z 000000018001a734     ProcessName.obj
 0002:00008748       $xdatasym                  000000018001a748     LIBCMT:amdsecgs.obj
 0002:0000874c       $unwind$?dllmain_crt_process_attach@@YAHQEAUHINSTANCE__@@QEAX@Z 000000018001a74c     LIBCMT:dll_dllmain.obj
 0002:00008788       $unwind$?fin$0@?0??dllmain_crt_process_attach@@YAHQEAUHINSTANCE__@@QEAX@Z@4HA 000000018001a788     LIBCMT:dll_dllmain.obj
 0002:00008788       $unwind$?fin$0@?0??dllmain_crt_process_detach@@YAH_N@Z@4HA 000000018001a788     LIBCMT:dll_dllmain.obj
 0002:00008788       $unwind$?fin$1@?0??dllmain_crt_process_detach@@YAH_N@Z@4HA 000000018001a788     LIBCMT:dll_dllmain.obj
 0002:00008788       $unwind$_IsNonwritableInCurrentImage$filt$0 000000018001a788     LIBCMT:pesect.obj
 0002:00008788       $unwind$?filt$0@?0??CxxCallCatchBlock@__FrameHandler4@@SAPEAXPEAU_EXCEPTION_RECORD@@@Z@4HA 000000018001a788     libvcruntime:frame.obj
 0002:00008788       $unwind$_query_new_handler$fin$0 000000018001a788     libucrt:new_handler.obj
 0002:00008788       $unwind$?fin$0@?0???$?RV<lambda_0ae27a3a962d80f24befdcbee591983d>@@AEAV<lambda_8d0ee55de4b1038c4002e0adecdf1839>@@V<lambda_dc504788e8f1664fe9b84e20bfb512f2>@@@?$__crt_seh_guarded_call@X@@QEAAX$$QEAV<lambda_0ae27a3a962d80f24befdcbee591983d>@@AEAV<lambda_8d0ee55de4b1038c4002e0adecdf1839>@@$$QEAV<lambda_dc504788e8f1664fe9b84e20bfb512f2>@@@Z@4HA 000000018001a788     libucrt:per_thread_data.obj
 0002:00008788       $unwind$?fin$0@?0???$?RV<lambda_2d41944a1d46af3157314b8a01080d33>@@AEAV<lambda_8f455de75cd7d7f24b4096f044d8b9e6>@@V<lambda_aa500f224e6afead328df44964fe2772>@@@?$__crt_seh_guarded_call@X@@QEAAX$$QEAV<lambda_2d41944a1d46af3157314b8a01080d33>@@AEAV<lambda_8f455de75cd7d7f24b4096f044d8b9e6>@@$$QEAV<lambda_aa500f224e6afead328df44964fe2772>@@@Z@4HA 000000018001a788     libucrt:per_thread_data.obj
 0002:00008788       $unwind$?fin$0@?0???$?RV<lambda_aa87e3671a710a21b5dc78c0bdf72e11>@@AEAV<lambda_92619d2358a28f41a33ba319515a20b9>@@V<lambda_6992ecaafeb10aed2b74cb1fae11a551>@@@?$__crt_seh_guarded_call@X@@QEAAX$$QEAV<lambda_aa87e3671a710a21b5dc78c0bdf72e11>@@AEAV<lambda_92619d2358a28f41a33ba319515a20b9>@@$$QEAV<lambda_6992ecaafeb10aed2b74cb1fae11a551>@@@Z@4HA 000000018001a788     libucrt:per_thread_data.obj
 0002:00008788       $unwind$?fin$0@?0???$?RV<lambda_f2e299630e499de9f9a165e60fcd3db5>@@AEAV<lambda_2ae9d31cdba2644fcbeaf08da7c24588>@@V<lambda_40d01ff24d0e7b3814fdbdcee8eab3c7>@@@?$__crt_seh_guarded_call@X@@QEAAX$$QEAV<lambda_f2e299630e499de9f9a165e60fcd3db5>@@AEAV<lambda_2ae9d31cdba2644fcbeaf08da7c24588>@@$$QEAV<lambda_40d01ff24d0e7b3814fdbdcee8eab3c7>@@@Z@4HA 000000018001a788     libucrt:per_thread_data.obj
 0002:00008788       $unwind$__acrt_update_thread_locale_data$fin$0 000000018001a788     libucrt:locale_refcounting.obj
 0002:00008788       $unwind$?fin$0@?0???$?RV<lambda_410d79af7f07d98d83a3f525b3859a53>@@AEAV<lambda_3e16ef9562a7dcce91392c22ab16ea36>@@V<lambda_38119f0e861e05405d8a144b9b982f0a>@@@?$__crt_seh_guarded_call@X@@QEAAX$$QEAV<lambda_410d79af7f07d98d83a3f525b3859a53>@@AEAV<lambda_3e16ef9562a7dcce91392c22ab16ea36>@@$$QEAV<lambda_38119f0e861e05405d8a144b9b982f0a>@@@Z@4HA 000000018001a788     libucrt:wsetlocale.obj
 0002:00008788       $unwind$?fin$0@?0???$?RV<lambda_751a882b2c74d4b022dec766aa51a29a>@@AEAV<lambda_628dfdc04ba53c8bfc02c9951375f3f5>@@V<lambda_f6c7be5f7998530c34de24c7437d6b54>@@@?$__crt_seh_guarded_call@H@@QEAAH$$QEAV<lambda_751a882b2c74d4b022dec766aa51a29a>@@AEAV<lambda_628dfdc04ba53c8bfc02c9951375f3f5>@@$$QEAV<lambda_f6c7be5f7998530c34de24c7437d6b54>@@@Z@4HA 000000018001a788     libucrt:close.obj
 0002:00008788       $unwind$?fin$0@?0???$?RV<lambda_a37b2b86f63e897a80ea819b0eb08c01>@@AEAV<lambda_38ce7e780aa69e748d6df282ebc68efe>@@V<lambda_99fb1378e971ab6e7edea83e3a7a83a2>@@@?$__crt_seh_guarded_call@H@@QEAAH$$QEAV<lambda_a37b2b86f63e897a80ea819b0eb08c01>@@AEAV<lambda_38ce7e780aa69e748d6df282ebc68efe>@@$$QEAV<lambda_99fb1378e971ab6e7edea83e3a7a83a2>@@@Z@4HA 000000018001a788     libucrt:commit.obj
 0002:00008788       $unwind$__acrt_initialize_lowio$fin$0 000000018001a788     libucrt:ioinit.obj
 0002:00008788       $unwind$__acrt_lowio_ensure_fh_exists$fin$0 000000018001a788     libucrt:osfinfo.obj
 0002:00008788       $unwind$_write$fin$0       000000018001a788     libucrt:write.obj
 0002:00008788       $unwind$?fin$0@?0???$?RV<lambda_efdfa57d1f175319df784efa44bb7b81>@@AEAV<lambda_5f0a4c1567f8adc6734073e5d1e1b35c>@@V<lambda_2e8a7d3640ea6ccb4c2413664c2db6fd>@@@?$__crt_seh_guarded_call@X@@QEAAX$$QEAV<lambda_efdfa57d1f175319df784efa44bb7b81>@@AEAV<lambda_5f0a4c1567f8adc6734073e5d1e1b35c>@@$$QEAV<lambda_2e8a7d3640ea6ccb4c2413664c2db6fd>@@@Z@4HA 000000018001a788     libucrt:mbctype.obj
 0002:00008788       $unwind$?fin$0@?0??update_thread_multibyte_data_internal@@YAPEAU__crt_multibyte_data@@QEAU__acrt_ptd@@QEAPEAU1@@Z@4HA 000000018001a788     libucrt:mbctype.obj
 0002:00008788       $unwind$?fin$0@?0???$?RV<lambda_450d765d439847d4c735a33c368b5fc0>@@AEAV<lambda_44731a7d0e6d81c3e6aa82d741081786>@@V<lambda_601a2a7da3b7a96e9554ac7215c4b07c>@@@?$__crt_seh_guarded_call@P6AXH@Z@@QEAAP6AXH@Z$$QEAV<lambda_450d765d439847d4c735a33c368b5fc0>@@AEAV<lambda_44731a7d0e6d81c3e6aa82d741081786>@@$$QEAV<lambda_601a2a7da3b7a96e9554ac7215c4b07c>@@@Z@4HA 000000018001a788     libucrt:signal.obj
 0002:00008788       $unwind$raise$fin$0        000000018001a788     libucrt:signal.obj
 0002:00008788       $unwind$?filt$0@?0???R<lambda_6e4b09c48022b2350581041d5f6b0c4c>@@QEBA@XZ@4HA 000000018001a788     libucrt:exit.obj
 0002:00008788       $unwind$?fin$0@?0???$?RV<lambda_d80eeec6fff315bfe5c115232f3240e3>@@AEAV<lambda_6e4b09c48022b2350581041d5f6b0c4c>@@V<lambda_2358e3775559c9db80273638284d5e45>@@@?$__crt_seh_guarded_call@X@@QEAAX$$QEAV<lambda_d80eeec6fff315bfe5c115232f3240e3>@@AEAV<lambda_6e4b09c48022b2350581041d5f6b0c4c>@@$$QEAV<lambda_2358e3775559c9db80273638284d5e45>@@@Z@4HA 000000018001a788     libucrt:exit.obj
 0002:00008788       $unwind$?fin$0@?0???$?RV<lambda_7777bce6b2f8c936911f934f8298dc43>@@AEAV<lambda_f03950bc5685219e0bcd2087efbe011e>@@V<lambda_3883c3dff614d5e0c5f61bb1ac94921c>@@@?$__crt_seh_guarded_call@H@@QEAAH$$QEAV<lambda_7777bce6b2f8c936911f934f8298dc43>@@AEAV<lambda_f03950bc5685219e0bcd2087efbe011e>@@$$QEAV<lambda_3883c3dff614d5e0c5f61bb1ac94921c>@@@Z@4HA 000000018001a788     libucrt:onexit.obj
 0002:00008788       $unwind$_fcloseall$fin$0   000000018001a788     libucrt:closeall.obj
 0002:00008788       $unwind$fclose$fin$0       000000018001a788     libucrt:fclose.obj
 0002:00008788       $unwind$?fin$0@?0???$?RV<lambda_842d9ff0dc9ef11c61343bbaebe7f885>@@AEAV<lambda_c5860995281e5c4ce005b3de8f5874ee>@@V<lambda_d90129c13df834fdcbf8d2b88dafcf2d>@@@?$__crt_seh_guarded_call@X@@QEAAX$$QEAV<lambda_842d9ff0dc9ef11c61343bbaebe7f885>@@AEAV<lambda_c5860995281e5c4ce005b3de8f5874ee>@@$$QEAV<lambda_d90129c13df834fdcbf8d2b88dafcf2d>@@@Z@4HA 000000018001a788     libucrt:fflush.obj
 0002:00008788       $unwind$?fin$0@?0???$?RV<lambda_886d6c58226a84441f68b9f2b8217b83>@@AEAV<lambda_ab61a845afdef5b7c387490eaf3616ee>@@V<lambda_f7f22ab5edc0698d5f6905b0d3f44752>@@@?$__crt_seh_guarded_call@X@@QEAAX$$QEAV<lambda_886d6c58226a84441f68b9f2b8217b83>@@AEAV<lambda_ab61a845afdef5b7c387490eaf3616ee>@@$$QEAV<lambda_f7f22ab5edc0698d5f6905b0d3f44752>@@@Z@4HA 000000018001a788     libucrt:fflush.obj
 0002:00008788       $unwind$_ctrlfp$filt$0     000000018001a788     libucrt:fpctrl.obj
 0002:00008790       $unwind$?dllmain_crt_process_detach@@YAH_N@Z 000000018001a790     LIBCMT:dll_dllmain.obj
 0002:000087e4       $unwind$?dllmain_dispatch@@YAHQEAUHINSTANCE__@@KQEAX@Z 000000018001a7e4     LIBCMT:dll_dllmain.obj
 0002:0000880c       $unwind$?filt$0@?0??dllmain_dispatch@@YAHQEAUHINSTANCE__@@KQEAX@Z@4HA 000000018001a80c     LIBCMT:dll_dllmain.obj
 0002:0000880c       $unwind$?filt$0@?0??FrameUnwindToState@__FrameHandler4@@SAXPEA_KPEAU_xDISPATCHER_CONTEXT@@PEAUFuncInfo4@FH4@@H@Z@4HA 000000018001a80c     libvcruntime:frame.obj
 0002:0000880c       $unwind$?fin$1@?0??FrameUnwindToState@__FrameHandler4@@SAXPEA_KPEAU_xDISPATCHER_CONTEXT@@PEAUFuncInfo4@FH4@@H@Z@4HA 000000018001a80c     libvcruntime:frame.obj
 0002:00008814       $unwind$_DllMainCRTStartup 000000018001a814     LIBCMT:dll_dllmain.obj
 0002:00008814       $unwind$__vcrt_getptd_noexit 000000018001a814     libvcruntime:per_thread_data.obj
 0002:00008814       $unwind$__vcrt_InitializeCriticalSectionEx 000000018001a814     libvcruntime:winapi_downlevel.obj
 0002:00008814       $unwind$__acrt_getptd      000000018001a814     libucrt:per_thread_data.obj
 0002:00008814       $unwind$__acrt_getptd_noexit 000000018001a814     libucrt:per_thread_data.obj
 0002:00008814       $unwind$__acrt_execute_initializers 000000018001a814     libucrt:shared_initialization.obj
 0002:00008814       $unwind$__acrt_InitializeCriticalSectionEx 000000018001a814     libucrt:winapi_thunks.obj
 0002:00008814       $unwind$?free_crt_array_internal@@YAXQEAPEBX_K@Z 000000018001a814     libucrt:inittime.obj
 0002:00008814       $unwind$??$common_lseek_nolock@_J@@YA_JH_JH@Z 000000018001a814     libucrt:lseek.obj
 0002:00008814       $unwind$__acrt_stdio_flush_nolock 000000018001a814     libucrt:fflush.obj
 0002:00008814       $unwind$??0_LocaleUpdate@@QEAA@QEAU__crt_locale_pointers@@@Z 000000018001a814     libucrt:output.obj
 0002:00008814       $unwind$_exception_enabled 000000018001a814     libucrt:libm_error.obj
 0002:00008824       $unwind$__report_securityfailure 000000018001a824     LIBCMT:gs_report.obj
 0002:0000882c       $unwind$__report_gsfailure 000000018001a82c     LIBCMT:gs_report.obj
 0002:00008834       $unwind$capture_current_context 000000018001a834     LIBCMT:gs_report.obj
 0002:00008840       $unwind$capture_previous_context 000000018001a840     LIBCMT:gs_report.obj
 0002:0000884c       $unwind$__security_init_cookie 000000018001a84c     LIBCMT:gs_support.obj
 0002:00008858       $unwind$__scrt_is_nonwritable_in_current_image 000000018001a858     LIBCMT:utility.obj
 0002:00008878       $unwind$__scrt_is_nonwritable_in_current_image$filt$0 000000018001a878     LIBCMT:utility.obj
 0002:00008880       $unwind$__scrt_dllmain_exception_filter 000000018001a880     LIBCMT:utility.obj
 0002:00008880       $unwind$?Is_bad_exception_allowed@@YAEPEBU_s_ESTypeList@@@Z 000000018001a880     libvcruntime:frame.obj
 0002:00008880       $unwind$_recalloc_base     000000018001a880     libucrt:recalloc.obj
 0002:00008880       $unwind$__acrt_free_locale 000000018001a880     libucrt:locale_refcounting.obj
 0002:00008880       $unwind$__acrt_lowio_create_handle_array 000000018001a880     libucrt:osfinfo.obj
 0002:00008880       $unwind$?setSBCS@@YAXPEAU__crt_multibyte_data@@@Z 000000018001a880     libucrt:mbctype.obj
 0002:00008880       $unwind$_seh_filter_exe    000000018001a880     libucrt:exception_filter.obj
 0002:00008880       $unwind$_initterm          000000018001a880     libucrt:initterm.obj
 0002:00008894       $unwind$__scrt_fastfail    000000018001a894     LIBCMT:utility_desktop.obj
 0002:000088a4       $unwind$__isa_available_init 000000018001a8a4     LIBCMT:cpu_disp.obj
 0002:000088b8       $xdatasym                  000000018001a8b8     LIBCMT:guard_dispatch.obj
 0002:000088c0       $xdatasym                  000000018001a8c0     LIBCMT:guard_xfg_dispatch.obj
 0002:000088c4       $unwind$??0length_error@std@@QEAA@PEBD@Z 000000018001a8c4     libcpmt:xthrow.obj
 0002:000088c4       $unwind$?__mbrtowc_utf8@__crt_mbstring@@YA_KPEA_WPEBD_KPEAU_Mbstatet@@@Z 000000018001a8c4     libucrt:mbrtowc.obj
 0002:000088cc       $unwind$?DecompFuncInfo@FH4@@YA_JPEAEAEAUFuncInfo4@1@_KH_N@Z 000000018001a8cc     libvcruntime:risctrnsctrl.obj
 0002:000088e4       $unwind$?UnwindNestedFrames@__FrameHandler4@@SAXPEA_KPEAUEHExceptionRecord@@PEAU_CONTEXT@@0PEAXPEAUFuncInfo4@FH4@@HHPEAUHandlerType4@5@PEAU_xDISPATCHER_CONTEXT@@E@Z 000000018001a8e4     libvcruntime:risctrnsctrl.obj
 0002:000088f8       $unwind$?GetRangeOfTrysToCheck@__FrameHandler4@@SA?AU?$pair@Viterator@TryBlockMap4@FH4@@V123@@std@@AEAVTryBlockMap4@FH4@@HPEAU_xDISPATCHER_CONTEXT@@PEAUFuncInfo4@5@H@Z 000000018001a8f8     libvcruntime:risctrnsctrl.obj
 0002:00008914       $unwind$__CxxFrameHandler4 000000018001a914     libvcruntime:risctrnsctrl.obj
 0002:00008928       $unwind$??$_CallSETranslator@V__FrameHandler4@@@@YAHPEAUEHExceptionRecord@@PEA_KPEAU_CONTEXT@@PEAU_xDISPATCHER_CONTEXT@@PEAUFuncInfo4@FH4@@K1H@Z 000000018001a928     libvcruntime:risctrnsctrl.obj
 0002:00008948       $unwind$?filt$0@?0???$_CallSETranslator@V__FrameHandler4@@@@YAHPEAUEHExceptionRecord@@PEA_KPEAU_CONTEXT@@PEAU_xDISPATCHER_CONTEXT@@PEAUFuncInfo4@FH4@@K1H@Z@4HA 000000018001a948     libvcruntime:risctrnsctrl.obj
 0002:00008954       $unwind$__DestructExceptionObject 000000018001a954     libvcruntime:ehhelpers.obj
 0002:00008974       $unwind$__DestructExceptionObject$filt$0 000000018001a974     libvcruntime:ehhelpers.obj
 0002:00008974       $unwind$?fin$1@?0??CxxCallCatchBlock@__FrameHandler4@@SAPEAXPEAU_EXCEPTION_RECORD@@@Z@4HA 000000018001a974     libvcruntime:frame.obj
 0002:00008980       $unwind$__std_exception_copy 000000018001a980     libvcruntime:std_exception.obj
 0002:00008980       $unwind$_free_osfhnd       000000018001a980     libucrt:osfinfo.obj
 0002:00008994       $unwind$__C_specific_handler 000000018001a994     libvcruntime:riscchandler.obj
 0002:000089b0       $unwind$_CxxThrowException 000000018001a9b0     libvcruntime:throw.obj
 0002:000089c0       $xdatasym                  000000018001a9c0     libvcruntime:memset.obj
 0002:000089d0       $unwind$?StateFromIp@__FrameHandler4@@SAHPEAUFuncInfo4@FH4@@PEAU_xDISPATCHER_CONTEXT@@_K@Z 000000018001a9d0     libvcruntime:ehstate.obj
 0002:000089e4       $unwind$?getStartStop@UWMap4@FH4@@QEAAXHHAEAViterator@12@0@Z 000000018001a9e4     libvcruntime:frame.obj
 0002:000089fc       $unwind$?getStateFromIterators@UWMap4@FH4@@SAHAEBViterator@12@H0H0@Z 000000018001a9fc     libvcruntime:frame.obj
 0002:000089fc       $unwind$strpbrk            000000018001a9fc     libucrt:strpbrk.obj
 0002:00008a0c       $unwind$?FrameUnwindToState@__FrameHandler4@@SAXPEA_KPEAU_xDISPATCHER_CONTEXT@@PEAUFuncInfo4@FH4@@H@Z 000000018001aa0c     libvcruntime:frame.obj
 0002:00008a54       $unwind$?CxxCallCatchBlock@__FrameHandler4@@SAPEAXPEAU_EXCEPTION_RECORD@@@Z 000000018001aa54     libvcruntime:frame.obj
 0002:00008ab0       $unwind$?IsInExceptionSpec@@YAEPEAUEHExceptionRecord@@PEBU_s_ESTypeList@@@Z 000000018001aab0     libvcruntime:frame.obj
 0002:00008acc       $unwind$??$__InternalCxxFrameHandler@V__FrameHandler4@@@@YA?AW4_EXCEPTION_DISPOSITION@@PEAUEHExceptionRecord@@PEA_KPEAU_CONTEXT@@PEAU_xDISPATCHER_CONTEXT@@PEAUFuncInfo4@FH4@@H1E@Z 000000018001aacc     libvcruntime:frame.obj
 0002:00008ae4       $unwind$__GSHandlerCheck_EH4 000000018001aae4     LIBCMT:gshandlereh4.obj
 0002:00008ae4       $unwind$__GSHandlerCheck_SEH 000000018001aae4     LIBCMT:gshandlerseh.obj
 0002:00008ae4       $unwind$??$TypeMatchHelper@V__FrameHandler3@@@@YAHPEBU_s_HandlerType@@PEBU_s_CatchableType@@PEBU_s_ThrowInfo@@@Z 000000018001aae4     libvcruntime:frame.obj
 0002:00008ae4       $unwind$??$TypeMatchHelper@V__FrameHandler4@@@@YAHPEAUHandlerType4@FH4@@PEBU_s_CatchableType@@PEBU_s_ThrowInfo@@@Z 000000018001aae4     libvcruntime:frame.obj
 0002:00008ae4       $unwind$?initialize_stdio_handles_nolock@@YAXXZ 000000018001aae4     libucrt:ioinit.obj
 0002:00008ae4       $unwind$__acrt_initialize_stdio 000000018001aae4     libucrt:_file.obj
 0002:00008afc       $unwind$??$BuildCatchObjectHelperInternal@V__FrameHandler4@@@@YAHPEAUEHExceptionRecord@@PEAXPEAUHandlerType4@FH4@@PEBU_s_CatchableType@@@Z 000000018001aafc     libvcruntime:frame.obj
 0002:00008b3c       $unwind$??$BuildCatchObjectInternal@V__FrameHandler4@@@@YAXPEAUEHExceptionRecord@@PEAXPEAUHandlerType4@FH4@@PEBU_s_CatchableType@@@Z 000000018001ab3c     libvcruntime:frame.obj
 0002:00008b68       $unwind$??$FindHandler@V__FrameHandler4@@@@YAXPEAUEHExceptionRecord@@PEA_KPEAU_CONTEXT@@PEAU_xDISPATCHER_CONTEXT@@PEAUFuncInfo4@FH4@@EH1@Z 000000018001ab68     libvcruntime:frame.obj
 0002:00008b88       $unwind$??$CatchIt@V__FrameHandler4@@@@YAXPEAUEHExceptionRecord@@PEA_KPEAU_CONTEXT@@PEAU_xDISPATCHER_CONTEXT@@PEAUFuncInfo4@FH4@@PEAUHandlerType4@4@PEBU_s_CatchableType@@PEAUTryBlockMapEntry4@4@H1EE@Z 000000018001ab88     libvcruntime:frame.obj
 0002:00008ba0       $unwind$??$FindHandlerForForeignException@V__FrameHandler4@@@@YAXPEAUEHExceptionRecord@@PEA_KPEAU_CONTEXT@@PEAU_xDISPATCHER_CONTEXT@@PEAUFuncInfo4@FH4@@HH1@Z 000000018001aba0     libvcruntime:frame.obj
 0002:00008bc0       $xdatasym                  000000018001abc0     libvcruntime:notify.obj
 0002:00008bcc       $unwind$?try_get_function@@YAPEAXW4function_id@?A0x3064ecbf@@QEBDQEBW4module_id@2@2@Z 000000018001abcc     libvcruntime:winapi_downlevel.obj
 0002:00008bcc       $unwind$?try_get_function@@YAPEAXW4function_id@?A0x391cf84c@@QEBDQEBW4module_id@2@2@Z 000000018001abcc     libucrt:winapi_thunks.obj
 0002:00008be8       $xdatasym                  000000018001abe8     libvcruntime:handlers.obj
 0002:00008c08       $xdatasym                  000000018001ac08     libvcruntime:memcpy.obj
 0002:00008c18       $unwind$_invalid_parameter_noinfo 000000018001ac18     libucrt:invalid_parameter.obj
 0002:00008c18       $unwind$_invalid_parameter_noinfo_noreturn 000000018001ac18     libucrt:invalid_parameter.obj
 0002:00008c18       $unwind$_log10_special     000000018001ac18     libucrt:log_special.obj
 0002:00008c20       $unwind$__acrt_call_reportfault 000000018001ac20     libucrt:invalid_parameter.obj
 0002:00008c40       $unwind$_invalid_parameter 000000018001ac40     libucrt:invalid_parameter.obj
 0002:00008c54       $unwind$_query_new_handler 000000018001ac54     libucrt:new_handler.obj
 0002:00008c74       $unwind$?common_exit@@YAXHW4_crt_exit_cleanup_mode@@W4_crt_exit_return_mode@@@Z 000000018001ac74     libucrt:exit.obj
 0002:00008c80       $unwind$??R<lambda_6e4b09c48022b2350581041d5f6b0c4c>@@QEBA@XZ 000000018001ac80     libucrt:exit.obj
 0002:00008ca0       $unwind$??$?RV<lambda_d80eeec6fff315bfe5c115232f3240e3>@@AEAV<lambda_6e4b09c48022b2350581041d5f6b0c4c>@@V<lambda_2358e3775559c9db80273638284d5e45>@@@?$__crt_seh_guarded_call@X@@QEAAX$$QEAV<lambda_d80eeec6fff315bfe5c115232f3240e3>@@AEAV<lambda_6e4b09c48022b2350581041d5f6b0c4c>@@$$QEAV<lambda_2358e3775559c9db80273638284d5e45>@@@Z 000000018001aca0     libucrt:exit.obj
 0002:00008cc4       $unwind$_configure_narrow_argv 000000018001acc4     libucrt:argv_parsing.obj
 0002:00008cd8       $unwind$??$parse_command_line@D@@YAXPEADPEAPEAD0PEA_K2@Z 000000018001acd8     libucrt:argv_parsing.obj
 0002:00008cf4       $unwind$??$free_environment@D@@YAXQEAPEAD@Z 000000018001acf4     libucrt:environment_initialization.obj
 0002:00008cf4       $unwind$??$free_environment@_W@@YAXQEAPEA_W@Z 000000018001acf4     libucrt:environment_initialization.obj
 0002:00008d00       $unwind$??$create_environment@D@@YAQEAPEADQEAD@Z 000000018001ad00     libucrt:environment_initialization.obj
 0002:00008d18       $unwind$_execute_onexit_table 000000018001ad18     libucrt:onexit.obj
 0002:00008d20       $unwind$__acrt_DownlevelLocaleNameToLCID 000000018001ad20     libucrt:lcidtoname_downlevel.obj
 0002:00008d20       $unwind$??R<lambda_f03950bc5685219e0bcd2087efbe011e>@@QEBAHXZ 000000018001ad20     libucrt:onexit.obj
 0002:00008d38       $unwind$??$?RV<lambda_7777bce6b2f8c936911f934f8298dc43>@@AEAV<lambda_f03950bc5685219e0bcd2087efbe011e>@@V<lambda_3883c3dff614d5e0c5f61bb1ac94921c>@@@?$__crt_seh_guarded_call@H@@QEAAH$$QEAV<lambda_7777bce6b2f8c936911f934f8298dc43>@@AEAV<lambda_f03950bc5685219e0bcd2087efbe011e>@@$$QEAV<lambda_3883c3dff614d5e0c5f61bb1ac94921c>@@@Z 000000018001ad38     libucrt:onexit.obj
 0002:00008d5c       $unwind$terminate          000000018001ad5c     libucrt:terminate.obj
 0002:00008d80       $xdatasym                  000000018001ad80     libucrt:strncmp.obj
 0002:00008d84       $unwind$_free_base         000000018001ad84     libucrt:free_base.obj
 0002:00008d84       $unwind$?destroy_fls@@YAXPEAX@Z 000000018001ad84     libucrt:per_thread_data.obj
 0002:00008d84       $unwind$__acrt_locale_free_numeric 000000018001ad84     libucrt:initnum.obj
 0002:00008d84       $unwind$__acrt_locale_free_lc_time_if_unreferenced 000000018001ad84     libucrt:locale_refcounting.obj
 0002:00008d8c       $unwind$?construct_ptd_array@@YAXQEAU__acrt_ptd@@@Z 000000018001ad8c     libucrt:per_thread_data.obj
 0002:00008d94       $unwind$?destroy_ptd_array@@YAXQEAU__acrt_ptd@@@Z 000000018001ad94     libucrt:per_thread_data.obj
 0002:00008d9c       $unwind$??$?RV<lambda_0ae27a3a962d80f24befdcbee591983d>@@AEAV<lambda_8d0ee55de4b1038c4002e0adecdf1839>@@V<lambda_dc504788e8f1664fe9b84e20bfb512f2>@@@?$__crt_seh_guarded_call@X@@QEAAX$$QEAV<lambda_0ae27a3a962d80f24befdcbee591983d>@@AEAV<lambda_8d0ee55de4b1038c4002e0adecdf1839>@@$$QEAV<lambda_dc504788e8f1664fe9b84e20bfb512f2>@@@Z 000000018001ad9c     libucrt:per_thread_data.obj
 0002:00008dc0       $unwind$??$?RV<lambda_aa87e3671a710a21b5dc78c0bdf72e11>@@AEAV<lambda_92619d2358a28f41a33ba319515a20b9>@@V<lambda_6992ecaafeb10aed2b74cb1fae11a551>@@@?$__crt_seh_guarded_call@X@@QEAAX$$QEAV<lambda_aa87e3671a710a21b5dc78c0bdf72e11>@@AEAV<lambda_92619d2358a28f41a33ba319515a20b9>@@$$QEAV<lambda_6992ecaafeb10aed2b74cb1fae11a551>@@@Z 000000018001adc0     libucrt:per_thread_data.obj
 0002:00008de4       $unwind$??$?RV<lambda_f2e299630e499de9f9a165e60fcd3db5>@@AEAV<lambda_2ae9d31cdba2644fcbeaf08da7c24588>@@V<lambda_40d01ff24d0e7b3814fdbdcee8eab3c7>@@@?$__crt_seh_guarded_call@X@@QEAAX$$QEAV<lambda_f2e299630e499de9f9a165e60fcd3db5>@@AEAV<lambda_2ae9d31cdba2644fcbeaf08da7c24588>@@$$QEAV<lambda_40d01ff24d0e7b3814fdbdcee8eab3c7>@@@Z 000000018001ade4     libucrt:per_thread_data.obj
 0002:00008e08       $unwind$??$?RV<lambda_2d41944a1d46af3157314b8a01080d33>@@AEAV<lambda_8f455de75cd7d7f24b4096f044d8b9e6>@@V<lambda_aa500f224e6afead328df44964fe2772>@@@?$__crt_seh_guarded_call@X@@QEAAX$$QEAV<lambda_2d41944a1d46af3157314b8a01080d33>@@AEAV<lambda_8f455de75cd7d7f24b4096f044d8b9e6>@@$$QEAV<lambda_aa500f224e6afead328df44964fe2772>@@@Z 000000018001ae08     libucrt:per_thread_data.obj
 0002:00008e2c       $unwind$??$__acrt_mbs_to_wcs_cp@U__crt_win32_buffer_internal_dynamic_resizing@@@@YAHQEBDAEAV?$__crt_win32_buffer@_WU__crt_win32_buffer_internal_dynamic_resizing@@@@I@Z 000000018001ae2c     libucrt:argv_wildcards.obj
 0002:00008e44       $unwind$__dcrt_get_narrow_environment_from_os 000000018001ae44     libucrt:get_environment_from_os.obj
 0002:00008e44       $unwind$??$__acrt_wcs_to_mbs_cp@U__crt_win32_buffer_internal_dynamic_resizing@@@@YAHQEB_WAEAV?$__crt_win32_buffer@DU__crt_win32_buffer_internal_dynamic_resizing@@@@I@Z 000000018001ae44     libucrt:argv_wildcards.obj
 0002:00008e5c       $unwind$??$common_expand_argv_wildcards@D@@YAHQEAPEADQEAPEAPEAD@Z 000000018001ae5c     libucrt:argv_wildcards.obj
 0002:00008e74       $unwind$??$copy_and_add_argument_to_buffer@D@@YAHQEBD0_KAEAV?$argument_list@D@?A0x5f5c8891@@@Z 000000018001ae74     libucrt:argv_wildcards.obj
 0002:00008e90       $unwind$??$expand_argument_wildcards@D@@YAHQEAD0AEAV?$argument_list@D@?A0x5f5c8891@@@Z 000000018001ae90     libucrt:argv_wildcards.obj
 0002:00008eb4       $unwind$__acrt_GetModuleFileNameA 000000018001aeb4     libucrt:getmodulefilenamea.obj
 0002:00008ed0       $unwind$__dcrt_write_console 000000018001aed0     libucrt:initcon.obj
 0002:00008ed0       $unwind$??$__acrt_wcs_to_mbs_cp@U__crt_win32_buffer_no_resizing@@@@YAHQEB_WAEAV?$__crt_win32_buffer@DU__crt_win32_buffer_no_resizing@@@@I@Z 000000018001aed0     libucrt:getmodulefilenamea.obj
 0002:00008ee4       $unwind$_setmbcp_nolock    000000018001aee4     libucrt:mbctype.obj
 0002:00008f04       $unwind$__dcrt_lowio_ensure_console_output_initialized 000000018001af04     libucrt:initcon.obj
 0002:00008f04       $unwind$_isleadbyte_l      000000018001af04     libucrt:_wctype.obj
 0002:00008f04       $unwind$?getSystemCP@@YAHH@Z 000000018001af04     libucrt:mbctype.obj
 0002:00008f0c       $unwind$?update_thread_multibyte_data_internal@@YAPEAU__crt_multibyte_data@@QEAU__acrt_ptd@@QEAPEAU1@@Z 000000018001af0c     libucrt:mbctype.obj
 0002:00008f34       $unwind$?setmbcp_internal@@YAHH_NQEAU__acrt_ptd@@QEAPEAU__crt_multibyte_data@@@Z 000000018001af34     libucrt:mbctype.obj
 0002:00008f44       $unwind$?setSBUpLow@@YAXPEAU__crt_multibyte_data@@@Z 000000018001af44     libucrt:mbctype.obj
 0002:00008f60       $unwind$??$?RV<lambda_efdfa57d1f175319df784efa44bb7b81>@@AEAV<lambda_5f0a4c1567f8adc6734073e5d1e1b35c>@@V<lambda_2e8a7d3640ea6ccb4c2413664c2db6fd>@@@?$__crt_seh_guarded_call@X@@QEAAX$$QEAV<lambda_efdfa57d1f175319df784efa44bb7b81>@@AEAV<lambda_5f0a4c1567f8adc6734073e5d1e1b35c>@@$$QEAV<lambda_2e8a7d3640ea6ccb4c2413664c2db6fd>@@@Z 000000018001af60     libucrt:mbctype.obj
 0002:00008f84       $unwind$?x_ismbbtype_l@@YAHPEAU__crt_locale_pointers@@IHH@Z 000000018001af84     libucrt:ismbbyte.obj
 0002:00008f94       $unwind$__GSHandlerCheckCommon 000000018001af94     LIBCMT:gshandler.obj
 0002:00008f94       $unwind$__acrt_WideCharToMultiByte 000000018001af94     libucrt:widechartomultibyte.obj
 0002:00008f9c       $unwind$__acrt_initialize_winapi_thunks 000000018001af9c     libucrt:winapi_thunks.obj
 0002:00008fa4       $unwind$_mbtowc_l          000000018001afa4     libucrt:mbtowc.obj
 0002:00008fa4       $unwind$__acrt_LCMapStringEx 000000018001afa4     libucrt:winapi_thunks.obj
 0002:00008fb8       $unwind$__acrt_initialize_lowio 000000018001afb8     libucrt:ioinit.obj
 0002:00008fd8       $unwind$?initialize_inherited_file_handles_nolock@@YAXXZ 000000018001afd8     libucrt:ioinit.obj
 0002:00008ff4       $unwind$__acrt_uninitialize_locale 000000018001aff4     libucrt:wsetlocale.obj
 0002:00008ff4       $unwind$__acrt_get_sigabrt_handler 000000018001aff4     libucrt:signal.obj
 0002:00008ffc       $unwind$raise              000000018001affc     libucrt:signal.obj
 0002:00009038       $unwind$??$?RV<lambda_450d765d439847d4c735a33c368b5fc0>@@AEAV<lambda_44731a7d0e6d81c3e6aa82d741081786>@@V<lambda_601a2a7da3b7a96e9554ac7215c4b07c>@@@?$__crt_seh_guarded_call@P6AXH@Z@@QEAAP6AXH@Z$$QEAV<lambda_450d765d439847d4c735a33c368b5fc0>@@AEAV<lambda_44731a7d0e6d81c3e6aa82d741081786>@@$$QEAV<lambda_601a2a7da3b7a96e9554ac7215c4b07c>@@@Z 000000018001b038     libucrt:signal.obj
 0002:0000905c       $unwind$?common_flush_all@@YAH_N@Z 000000018001b05c     libucrt:fflush.obj
 0002:00009064       $unwind$??$?RV<lambda_842d9ff0dc9ef11c61343bbaebe7f885>@@AEAV<lambda_c5860995281e5c4ce005b3de8f5874ee>@@V<lambda_d90129c13df834fdcbf8d2b88dafcf2d>@@@?$__crt_seh_guarded_call@X@@QEAAX$$QEAV<lambda_842d9ff0dc9ef11c61343bbaebe7f885>@@AEAV<lambda_c5860995281e5c4ce005b3de8f5874ee>@@$$QEAV<lambda_d90129c13df834fdcbf8d2b88dafcf2d>@@@Z 000000018001b064     libucrt:fflush.obj
 0002:00009088       $unwind$??$?RV<lambda_886d6c58226a84441f68b9f2b8217b83>@@AEAV<lambda_ab61a845afdef5b7c387490eaf3616ee>@@V<lambda_f7f22ab5edc0698d5f6905b0d3f44752>@@@?$__crt_seh_guarded_call@X@@QEAAX$$QEAV<lambda_886d6c58226a84441f68b9f2b8217b83>@@AEAV<lambda_ab61a845afdef5b7c387490eaf3616ee>@@$$QEAV<lambda_f7f22ab5edc0698d5f6905b0d3f44752>@@@Z 000000018001b088     libucrt:fflush.obj
 0002:000090b0       $unwind$??$?RV<lambda_410d79af7f07d98d83a3f525b3859a53>@@AEAV<lambda_3e16ef9562a7dcce91392c22ab16ea36>@@V<lambda_38119f0e861e05405d8a144b9b982f0a>@@@?$__crt_seh_guarded_call@X@@QEAAX$$QEAV<lambda_410d79af7f07d98d83a3f525b3859a53>@@AEAV<lambda_3e16ef9562a7dcce91392c22ab16ea36>@@$$QEAV<lambda_38119f0e861e05405d8a144b9b982f0a>@@@Z 000000018001b0b0     libucrt:wsetlocale.obj
 0002:000090d8       $unwind$__acrt_update_thread_locale_data 000000018001b0d8     libucrt:locale_refcounting.obj
 0002:000090fc       $unwind$qsort              000000018001b0fc     libucrt:qsort.obj
 0002:00009114       $chain$4$qsort             000000018001b114     libucrt:qsort.obj
 0002:00009138       $chain$5$qsort             000000018001b138     libucrt:qsort.obj
 0002:00009148       $unwind$fallbackMethod     000000018001b148     libucrt:strpbrk.obj
 0002:00009158       $unwind$_mbsdec_l          000000018001b158     libucrt:mbsdec.obj
 0002:00009164       $unwind$__acrt_GetStringTypeA 000000018001b164     libucrt:getstringtypea.obj
 0002:0000918c       $unwind$__acrt_LCMapStringA 000000018001b18c     libucrt:lcmapstringa.obj
 0002:0000919c       $unwind$?__acrt_LCMapStringA_stat@@YAHPEAU__crt_locale_pointers@@PEB_WKPEBDHPEADHHH@Z 000000018001b19c     libucrt:lcmapstringa.obj
 0002:000091c4       $unwind$__acrt_lowio_destroy_handle_array 000000018001b1c4     libucrt:osfinfo.obj
 0002:000091d4       $unwind$__acrt_lowio_ensure_fh_exists 000000018001b1d4     libucrt:osfinfo.obj
 0002:00009200       $unwind$_close             000000018001b200     libucrt:close.obj
 0002:00009200       $unwind$_commit            000000018001b200     libucrt:commit.obj
 0002:00009208       $unwind$??$?RV<lambda_a37b2b86f63e897a80ea819b0eb08c01>@@AEAV<lambda_38ce7e780aa69e748d6df282ebc68efe>@@V<lambda_99fb1378e971ab6e7edea83e3a7a83a2>@@@?$__crt_seh_guarded_call@H@@QEAAH$$QEAV<lambda_a37b2b86f63e897a80ea819b0eb08c01>@@AEAV<lambda_38ce7e780aa69e748d6df282ebc68efe>@@$$QEAV<lambda_99fb1378e971ab6e7edea83e3a7a83a2>@@@Z 000000018001b208     libucrt:commit.obj
 0002:0000922c       $unwind$_write             000000018001b22c     libucrt:write.obj
 0002:0000925c       $unwind$_write_nolock      000000018001b25c     libucrt:write.obj
 0002:00009274       $unwind$?write_double_translated_ansi_nolock@@YA?AUwrite_result@?A0x17268360@@HQEBDI@Z 000000018001b274     libucrt:write.obj
 0002:00009298       $unwind$?write_text_ansi_nolock@@YA?AUwrite_result@?A0x17268360@@HQEBDI@Z 000000018001b298     libucrt:write.obj
 0002:00009298       $unwind$?write_text_utf16le_nolock@@YA?AUwrite_result@?A0x17268360@@HQEBDI@Z 000000018001b298     libucrt:write.obj
 0002:000092b8       $unwind$?write_text_utf8_nolock@@YA?AUwrite_result@?A0x17268360@@HQEBDI@Z 000000018001b2b8     libucrt:write.obj
 0002:000092dc       $unwind$_fcloseall         000000018001b2dc     libucrt:closeall.obj
 0002:00009300       $unwind$?__mbsrtowcs_utf8@__crt_mbstring@@YA_KPEA_WPEAPEBD_KPEAU_Mbstatet@@@Z 000000018001b300     libucrt:mbrtowc.obj
 0002:00009318       $unwind$__acrt_locale_free_monetary 000000018001b318     libucrt:initmon.obj
 0002:00009320       $unwind$__acrt_locale_free_time 000000018001b320     libucrt:inittime.obj
 0002:00009330       $unwind$_putwch_nolock     000000018001b330     libucrt:putwch.obj
 0002:00009338       $unwind$fclose             000000018001b338     libucrt:fclose.obj
 0002:0000935c       $unwind$?__mbrtoc32_utf8@__crt_mbstring@@YA_KPEA_UPEBD_KPEAU_Mbstatet@@@Z 000000018001b35c     libucrt:mbrtoc32.obj
 0002:00009378       $xdatasym                  000000018001b378     libucrt:log10.obj
 0002:00009384       $unwind$??$?RV<lambda_751a882b2c74d4b022dec766aa51a29a>@@AEAV<lambda_628dfdc04ba53c8bfc02c9951375f3f5>@@V<lambda_f6c7be5f7998530c34de24c7437d6b54>@@@?$__crt_seh_guarded_call@H@@QEAAH$$QEAV<lambda_751a882b2c74d4b022dec766aa51a29a>@@AEAV<lambda_628dfdc04ba53c8bfc02c9951375f3f5>@@$$QEAV<lambda_f6c7be5f7998530c34de24c7437d6b54>@@@Z 000000018001b384     libucrt:close.obj
 0002:000093a8       $unwind$_call_matherr      000000018001b3a8     libucrt:libm_error.obj
 0002:000093b0       $unwind$_handle_error      000000018001b3b0     libucrt:libm_error.obj
 0002:000093d0       $unwind$__acrt_initialize_fma3 000000018001b3d0     libucrt:fma3_available.obj
 0002:000093d8       $unwind$_log_special_common 000000018001b3d8     libucrt:log_special.obj
 0002:000093e8       $xdatasym                  000000018001b3e8     libucrt:fpsr.obj
 0002:000093f0       $unwind$_raise_exc_ex      000000018001b3f0     libucrt:fpexcept.obj
 0002:00009404       $unwind$_ctrlfp            000000018001b404     libucrt:fpctrl.obj
 0002:0000942c       $unwind$_IsNonwritableInCurrentImage 000000018001b42c     LIBCMT:pesect.obj
 0002:00009450       $xdatasym                  000000018001b450     LIBCMT:chkstk.obj
 0002:00009458       $xdatasym                  000000018001b458     libvcruntime:memcmp.obj
 0002:00009640       .edata                     000000018001b640     FileCase.exp
 0002:00009668       rgpv                       000000018001b668     FileCase.exp
 0002:00009678       rgszName                   000000018001b678     FileCase.exp
 0002:00009688       rgwOrd                     000000018001b688     FileCase.exp
 0002:00009690       szName                     000000018001b690     FileCase.exp
 0002:0000969d       $N00001                    000000018001b69d     FileCase.exp
 0002:000096ac       $N00002                    000000018001b6ac     FileCase.exp
 0002:000096bb       $N00003                    000000018001b6bb     FileCase.exp
 0002:000096c1       $N00004                    000000018001b6c1     FileCase.exp
 0002:0000998c       .idata$6                   000000018001b98c     kernel32:KERNEL32.dll
 0003:00000030       ?__vcrt_flsindex@@3KA      000000018001c030     libvcruntime:per_thread_data.obj
 0003:00000050       ?__acrt_flsindex@@3KA      000000018001c050     libucrt:per_thread_data.obj
 0003:00000054       ?errno_no_memory@@3HA      000000018001c054     libucrt:errno.obj
 0003:00000058       ?doserrno_no_memory@@3KA   000000018001c058     libucrt:errno.obj
 0003:00000290       _mbctypes                  000000018001c290     libucrt:mbctype.obj
 0003:000003a0       _mbcasemaps                000000018001c3a0     libucrt:mbctype.obj
 0003:000004a0       ?__rgctypeflag@@3PADA      000000018001c4a0     libucrt:mbctype.obj
 0003:000004b0       ?__rgcode_page_info@@3PAUcode_page_info@@A 000000018001c4b0     libucrt:mbctype.obj
 0003:000009c0       ?__dcrt_lowio_console_output_handle@@3PEAXEA 000000018001c9c0     libucrt:initcon.obj
 0003:000009d0       ?dazSupported@?1??_ctrlfp@@9@9 000000018001c9d0     libucrt:fpctrl.obj
 0003:00000bb0       ?__proc_attached@@3HA      000000018001cbb0     LIBCMT:dll_dllmain.obj
 0003:00000bc0       GS_ExceptionRecord         000000018001cbc0     LIBCMT:gs_report.obj
 0003:00000c60       GS_ContextRecord           000000018001cc60     LIBCMT:gs_report.obj
 0003:00001160       ?is_initialized_as_dll@@3_NA 000000018001d160     LIBCMT:utility.obj
 0003:00001161       ?module_local_atexit_table_initialized@@3_NA 000000018001d161     LIBCMT:utility.obj
 0003:00001168       ?module_local_atexit_table@@3U_onexit_table_t@@A 000000018001d168     LIBCMT:utility.obj
 0003:00001180       ?module_local_at_quick_exit_table@@3U_onexit_table_t@@A 000000018001d180     LIBCMT:utility.obj
 0003:000011c0       ?__vcrt_startup_thread_ptd@@3U__vcrt_ptd@@A 000000018001d1c0     libvcruntime:per_thread_data.obj
 0003:00001288       ?heap@@3V_HeapManager@@A   000000018001d288     libvcruntime:undname.obj
 0003:000012b0       __vcrt_lock_table          000000018001d2b0     libvcruntime:locks.obj
 0003:000012d8       __vcrt_locks_initialized   000000018001d2d8     libvcruntime:locks.obj
 0003:000012e0       ?module_handles@@3PAPEAUHINSTANCE__@@A 000000018001d2e0     libvcruntime:winapi_downlevel.obj
 0003:000012f8       ?function_pointers@@3PAPEAXA 000000018001d2f8     libvcruntime:winapi_downlevel.obj
 0003:00001320       ?__acrt_invalid_parameter_handler@@3V?$dual_state_global@P6AXPEB_W00I_K@Z@__crt_state_management@@A 000000018001d320     libucrt:invalid_parameter.obj
 0003:00001328       ?__acrt_new_handler@@3V?$dual_state_global@P6AH_K@Z@__crt_state_management@@A 000000018001d328     libucrt:new_handler.obj
 0003:00001330       ?c_termination_complete@@3JA 000000018001d330     libucrt:exit.obj
 0003:00001338       ?thread_local_exit_callback_func@@3P6AXPEAXK0@ZEA 000000018001d338     libucrt:exit.obj
 0003:00001350       ?program_name@?1???$common_configure_argv@D@@YAHW4_crt_argv_mode@@@Z@4PADA 000000018001d350     libucrt:argv_parsing.obj
 0003:000014b0       ?__acrt_lock_table@@3PAU_RTL_CRITICAL_SECTION@@A 000000018001d4b0     libucrt:locks.obj
 0003:000016e0       ?__acrt_locks_initialized@@3IA 000000018001d6e0     libucrt:locks.obj
 0003:00001700       ?fSystemSet@@3HA           000000018001d700     libucrt:mbctype.obj
 0003:00001704       ?initialized@?1??__acrt_initialize_multibyte@@9@4_NA 000000018001d704     libucrt:mbctype.obj
 0003:00001740       ?module_handles@@3PAPEAUHINSTANCE__@@A 000000018001d740     libucrt:winapi_thunks.obj
 0003:000017e0       ?encoded_function_pointers@@3PAPEAXA 000000018001d7e0     libucrt:winapi_thunks.obj
 0003:00001d08       ?ctrlc_action@@3V?$dual_state_global@P6AXH@Z@__crt_state_management@@A 000000018001dd08     libucrt:signal.obj
 0003:00001d10       ?ctrlbreak_action@@3V?$dual_state_global@P6AXH@Z@__crt_state_management@@A 000000018001dd10     libucrt:signal.obj
 0003:00001d18       ?abort_action@@3V?$dual_state_global@P6AXH@Z@__crt_state_management@@A 000000018001dd18     libucrt:signal.obj
 0003:00001d20       ?term_action@@3V?$dual_state_global@P6AXH@Z@__crt_state_management@@A 000000018001dd20     libucrt:signal.obj
 0003:00001d28       ?user_matherr@@3V?$dual_state_global@P6AHPEAU_exception@@@Z@__crt_state_management@@A 000000018001dd28     libucrt:matherr.obj
 0003:00001d58       ?internal_state@?1??_mbtowc_l@@9@4U_Mbstatet@@A 000000018001dd58     libucrt:mbtowc.obj
 0003:00001d64       ?__acrt_global_new_mode@@3V?$dual_state_global@J@__crt_state_management@@A 000000018001dd64     libucrt:new_mode.obj
 0003:00001d70       ?__acrt_app_type@@3W4_crt_app_type@@A 000000018001dd70     libucrt:report_runtime_error.obj
 0003:00001d78       ?internal_pst@?1??__mbrtoc32_utf8@__crt_mbstring@@YA_KPEA_UPEBD_KPEAU_Mbstatet@@@Z@4U3@A 000000018001dd78     libucrt:mbrtoc32.obj
 0003:00002458       ?ResetButtonID@@3HA        000000018001e458     filecvt.obj
 0003:0000245c       ?WordDivEditID@@3HA        000000018001e45c     filecvt.obj
 0003:00002460       ?dummy@?9??ProcessName@@YAXPEB_WK@Z@4PA_WA 000000018001e460     ProcessName.obj
 0003:00002468       ?PluginMenuStrings@?1??GetPluginInfoW@@9@4PAPEB_WA 000000018001e468     FileCase.obj
 0005:00000000       MsetTab                    0000000180021000     libvcruntime:memset.obj
 0005:00000050       MoveSmall                  0000000180021050     libvcruntime:memcpy.obj
 0005:00000090       MoveSmallYmm               0000000180021090     libvcruntime:memcpy.obj
 0005:000000b4       MoveSmallYmmNT             00000001800210b4     libvcruntime:memcpy.obj
 0005:000000d8       MoveSmallXmm               00000001800210d8     libvcruntime:memcpy.obj
 0006:00000060       $R000000                   0000000180022060     FileCase.res
